:020000040800F2
:1000000000000110F9EB03086DA6020825D80008CE
:10001000FDEC0308FDEC0308FDEC03080000000004
:10002000000000000000000000000000B9AC020861
:10003000B5AC020800000000B1AC020819EE0008DF
:10004000FDEC0308FDEC0308FDEC0308FDEC0308E0
:10005000FDEC0308FDEC03085D9A0008899B00088D
:100060004D9B0008119B0008D59A0008E5BC0008CC
:10007000D5BC0008C5BC0008B5BC0008A5BC00087C
:1000800091BC00087DBC0008FDEC0308FDEC0308F2
:10009000FDEC0308FDEC0308FDEC0308999A000849
:1000A000CDDE0008FDEC0308FDEC0308FDEC0308C1
:1000B0001DDF00080DDF0008FDEC030801C5000886
:1000C00009C50008F5C40008FDC40008FDEC0308DC
:1000D000FDEC0308818F0008FDEC0308DDEF00084C
:1000E000219A0008FDEC0308A9AE0208FDEC030804
:1000F000DDDE0008FDEC0308EDDE000869BC000849
:10010000FDEC0308FDEC0308FDDE0008FDEC030830
:1001100041EF0008FDEC0308A1CD010885CD0108E1
:1001200055BC000841BC00082DBC000819BC0008E3
:1001300005BC0008FDEC0308FDEC0308FDEC03081A
:10014000FDEC0308FDEC0308FDEC030871A60208B2
:10015000F1BB0008DDBB0008C9BB0008A5EE000824
:10016000E9C40008F1C40008FDEC0308FDEC030835
:10017000FDEC0308FDEC0308FDEC0308FDEC0308AF
:08018000FDEC0308FDEC03088F
:1001880002020300C01F0020BC1F00200000000066
:100198000000000016000800C41F0020CC1F00202B
:1001A80000000000240600081D0001009C23002018
:1001B8002C240020000000002C0600082700040062
:1001C800BC23002030240020000000002E06000878
:1001D80003000100F4250020FC2500200000000099
:1001E800000000000101040040260020C83900205A
:1001F8000000000000000000080209000639002085
:10020800CC390020000000002982000806020C00FA
:100218007C390020D839002000000000B18D00088A
:1002280007020200B0390020E43900200000000075
:1002380032060008FF010100C6390020E839002015
:100248000000000034060008FA010200C43900204A
:10025800EC3900200000000015C6000802000C0060
:1002680088390020F039002000000000000000005C
:10027800F701060000390020FC39002000000000CA
:10028800360600080A020A00D0260020043A002098
:10029800000000003C060008031233009F3C0020C9
:1002A8006C3C0020000000004806000825005A00A9
:1002B800B83B0020123C00200000000000000000B5
:1002C800F6110C00AC3B0020A03B00200000000011
:1002D8007C06000801200800AC3D0020F83D002005
:1002E80000000000880600081A000800903D002061
:1002F800003E002000000000900600080B201000BF
:1003080038460020704600200000000098060008CB
:100318001F000E00A84300208046002000000000B7
:10032800A806000805020100FC43002090460020B2
:1003380000000000B60600080002050094460020F0
:100348000C4A002000000000000000001E0004000D
:10035800D4470020144A002000000000B806000816
:1003680022000C0054470020184A0020000000001A
:10037800BC06000804008000805D0020005F0020AB
:100388000000000000000000F9010400446500209E
:10039800DC7F0020000000001182000818102C00EB
:1003A80014650020E07F00200000000019A0030869
:1003B800FB010100D86400200C8000200000000030
:1003C800FDC50008FC010900A4630020108000207E
:1003D80000000000C9C500080A1012007863002058
:1003E8001C80002000000000C80600080600160057
:1003F800486000203080002000000000CD14020872
:1004080003010600FC860020388700200000000059
:10041800DA06000829005000D88900202C8A00201C
:10042800000000000000000014000200D489002031
:100438007C8A002000000000E0060008100003008D
:10044800C8890020808A002000000000E206000819
:1004580028000C00BC890020848A002000000000CD
:10046800E606000823001000AC890020908A0020CE
:10047800000000006DE6020819000500A4890020AC
:10048800A08A002000000000F2060008F811010010
:10049800A0890020A88A002000000000F8060008B3
:1004A800000104009C890020AC8A002000000000A4
:1004B800FA0600082F00110088890020B08A002061
:1004C80000000000FE060008050006000A8C002057
:1004D8001499002000000000100700080E20EA0010
:1004E800EE8A00201C99002000000000AD140208CC
:1004F80013000400248C0020089A0020000000004B
:100508001807000802010300D98A00200C9A00206D
:100518000000000071C301081B00F400189A0020B5
:10052800B89C002000000000B566020826000E00F6
:10053800BC9D0020AC9D0020000000002D47030852
:1005480009020100CC9F002024A000200000000028
:100558001C07000812100C00859F002028A000200E
:10056800000000001E0700080C002400989F0020CF
:1005780034A000200000000049C301083400100026
:10058800A0A70020FCA900200000000025B2030855
:100598000D003C0064A700200CAA00200000000009
:1005A80059360208FD01240080A0002048AA002036
:1005B80000000000A1810008FE0108006CA00020D6
:1005C8006CAA00200000000005C600082C001000DE
:1005D80008AC0020F8AB002000000000959D03083F
:1005E8002B0024003CAC002018AC002000000000C8
:1005F800659D03082A006000B8B3002058B30020A6
:1006080000000000FDB103081500700090AD002047
:0C06180018B400200000000000000000EA
:10062400C409000019012828000020030000013C2F
:10063400000031010000000000004A01B400D601AE
:1006440000000000000000000000000000000000A6
:100654000000000000000000000000000000000096
:100664000000000000000000000000000000000086
:100674000000000000000100000000000000000075
:1006840000000000E8036400040A00017E05EA0596
:10069400B40532002B21231E640102000000010076
:1006A4000A0129000000000000000100000000050C
:1006B4000000000000000100C800141E01006400D6
:1006C4002C01280000300100005A000000009001B5
:1006D4002C01C800640004010100000003000001B3
:1006E4000500000000010000000000000000000000
:1006F4002801000004009001000000000000000038
:1007040000000000000000000000000020000200C3
:10071400010000000800000037000000000100058F
:06072400424A46340000C9
:10072A005001000007000000020000000000803FA6
:10073A000000803F0000803F000000000000000031
:10074A00010203040607080901010000E048040841
:10075A00A87304080000000000000000F048040824
:10076A00F84804080000000001200000FC480408C2
:10077A000449040800000000014000000849040878
:10078A00B45D0408000000000120000014490408B8
:10079A00204904080000000004000000244904085D
:1007AA00304904080000000004000000344904082D
:1007BA00CC71040800000000010000000201FF00E3
:1007CA000000803F0000803F701E040805080400F6
:1007DA000000000074420408104204085C1E040869
:1007EA00000000009C1E040805080A000000000022
:1007FA007442040810420408184304080000000068
:10080A00FFFFFFFF0000803F0060024010600240CF
:10081A0000000000000B00000000200000000000A3
:10082A000000000000600240286002400000000052
:10083A00060C00000000200000000000000000007C
:10084A00006002404060024000000000100D0000FD
:10085A0000002000000000000000000000600240CC
:10086A005860024000000000160E00000000200040
:10087A0000000000000000000060024070600240BA
:10088A0000000000200F000000002000000000000F
:10089A000000000000600240886002400000000082
:1008AA0026100000000020000000000000000000E8
:1008BA0000600240A0600240000000003011000009
:1008CA00000020000000000000000000006002405C
:1008DA00B860024000000000362F0000000020002F
:1008EA0000000000000000000064024010640240A2
:1008FA000000000000380000000040000000000076
:10090A000000000000640240286402400000000069
:10091A00063900000000400000000000000000004E
:10092A00006402404064024000000000103A0000E7
:10093A0000004000000000000000000000640240C7
:10094A005864024000000000163B0000000040000E
:10095A0000000000000000000064024070640240D1
:10096A0000000000203C00000000400000000000E1
:10097A000000000000640240886402400000000099
:10098A0026440000000040000000000000000000B3
:10099A0000640240A06402400000000030450000EC
:1009AA000000400000000000000000000064024057
:1009BA00B864024000000000364600000000400013
:1009CA0000000000000000000D6F0308C56E030858
:1009DA00156E030800000000116C0308496D030836
:1009EA00E96D0308B16C0308000000000000000074
:1009FA00056C0308859D0208819D02087D9D0208F9
:100A0A00719D02086D9D0208799D0208759D020874
:100A1A00F99D0208ED9D0208C59D0208D99D0208AC
:100A2A00B19D02089D9D0208899D020801000000EF
:100A3A000000803F010000000403090412010002C3
:100A4A000202004083044057000201020301000031
:100A5A00AD720308AD710308297303086D6C0308AE
:100A6A00A16F03087D6C0308996C0308456C0308A1
:100A7A00356C0308000000000000000001000000BF
:100A8A000101000000010101EDEB02080000000075
:100A9A00000000000100000000FFFF00000000004D
:100AAA00AA5505010000AA5507010000AA5503002E
:100ABA009F00000000000000010203040102030479
:100ACA0006070809AA550B010000AA5509020000E9
:100ADA000000000001000000C01200003030303079
:100AEA002D30312D30315430303A30303A303000F8
:100AFA0001010100807A04080E000000F93303089E
:100B0A00000000000000000054050020447A040898
:100B1A0000000000000000000000000000000000CB
:100B2A00A87304080000000000000000F00500207F
:100B3A0004000000D07904080C000000C939030839
:100B4A00040A002000000000F47804080C000000E9
:100B5A0099390308F809002000000000647A0408A3
:100B6A000800000000000000EC090020040000005A
:100B7A00547A04080C000000B1380308E009002088
:100B8A0000000000E078040803000000695E030822
:100B9A00C8090020000000005C7A04080300000075
:100BAA00695E0308B009002000000000E478040828
:100BBA00010000000000000000000000000000002A
:100BCA00000000000D00000000000000000000000E
:100BDA0000000000447A0408000000000000000041
:100BEA000000000000000000A873040800000000D4
:100BFA0000000000F00500200400000074790408D9
:100C0A000300000055380308980900200800000076
:100C1A00547A04080C000000B1380308E0090020E7
:100C2A0000000000E078040803000000695E030881
:100C3A00C8090020000000005C7A040803000000D4
:100C4A00695E0308B009002000000000E478040887
:100C5A000100000000000000000000000000000089
:100C6A00000000000D00000000000000000000006D
:100C7A00000000006C7A0408000000000000000078
:100C8A000000000000000000A87304080000000033
:100C9A0000000000F0050020040000007C79040830
:100CAA0003000000695E0308100A0020000000002B
:100CBA00E4780408010000000000000000000000C1
:100CCA0000000000000000000D000000000000000D
:100CDA00000000000000000020700020702D72004B
:100CEA0000000001000000000000000000000000F9
:100CFA002D202D2D202D2D2D2D202D2D2D2D00009B
:100D0A0000000000000000000000000000000000D9
:100D1A002D202D2D202D2D2D2D202D2D2D000000A7
:100D2A0000000000000000000000000000000000B9
:100D3A00D28A002088130C1701000000D48A0020F0
:100D4A0088130C1700000000B8780408000000009F
:100D5A00000000000000000000000000C87804083D
:100D6A0008000000000000001C060020040000002B
:100D7A00D4780408080000000000000010060020D3
:100D8A0000000000E0780408040000009538030819
:100D9A000000000000000000E478040801000000E0
:100DAA000000000000000000000000000000000039
:100DBA000D0000000000000000000000000000001C
:100DCA00D08A002088130C1701000000CE8A002068
:100DDA0088130C1700000000247904080E00000094
:100DEA00513403080000000000000000280600201B
:100DFA00228C00200100000034420408CD8A002021
:100E0A0001000000404204082E8700200200000072
:100E1A0048420408465E002000000000000000006E
:100E2A00445E00200000000000000000425E002036
:100E3A000000000000000000405E002000000000EA
:100E4A00000000003E5E00200000000000000000DC
:100E5A003C5E00200000000000000000B8030020F3
:100E6A000000000000000000CC8A00200200000000
:100E7A00544204082C790408000000000000000015
:100E8A000000000000000000C87804080800000004
:100E9A0000000000AC06002004000000D47804081A
:100EAA000800000000000000A0060020000000006A
:100EBA00E078040804000000313403080000000050
:100ECA0000000000E47804080100000000000000AF
:100EDA000000000000000000000000000D000000FB
:100EEA000000000000000000000000003C79040837
:100EFA0000000000000000000000000000000000E8
:100F0A004C7904080C00000039390308E80600206F
:100F1A0004000000587904080C0000007534030826
:100F2A00DC06002004000000647904080C000000BC
:100F3A00F9380308D0060020000000007079040880
:100F4A000300000075380308B806002008000000F6
:100F5A007C79040803000000695E0308100A002077
:100F6A0000000000E478040801000000000000000E
:100F7A000000000000000000000000000D0000005A
:100F8A00000000000000000000000000847904084E
:100F9A000000000000000000000000000000000047
:100FAA008C79040804000000F939030800000000E5
:100FBA0000000000E47804080100000000000000BE
:100FCA000000000000000000000000000D0000000A
:100FDA00000000000000000000000000D8790408AA
:100FEA0000000000000000000000000000000000F7
:100FFA001C6B04080C0000000000000048070020D9
:10100A0004000000E879040808000000000000005D
:10101A003C07002004000000F479040808000000DE
:10102A00000000003007002004000000FC790408DA
:10103A00080000000000000024070020040000004F
:10104A00047A0408080000000000000018070020C5
:10105A00040000000C7A04080800000000000000E8
:10106A000C07002004000000147A0408080000009D
:10107A000000000000070020040000001C7A040899
:10108A000800000000000000F40600200400000030
:10109A00E4780408010000000000000000000000DD
:1010AA0000000000000000000D0000000000000029
:1010BA000000000000000000247A04080E0000006E
:1010CA00413403080000000000000000540700201B
:1010DA002C7A04080E000000000000000000000046
:1010EA0000000000CC070020347A04080E0000003B
:1010FA000000000000000000000000006C08002052
:10110A00218C00200400000060420408C88A0020E4
:10111A00E0150C1700000000CB8A00200800000030
:10112A0010420408CA8A002005000000744204081C
:10113A003C7A04080E0000000000000000000000D5
:10114A0000000000BC08002000000101FFFF0000B1
:10115A00A8680408000000000000000085C3010818
:10116A00A08601000400000000000000000000004A
:10117A000000000000000000000000000000000065
:10118A0000000000EC760408D463040800000000A4
:10119A005D7D01087D0000000600000000000000DF
:1011AA000000000000000000000000000000000035
:1011BA0000000000000000009C7A04080000000003
:1011CA000000000099D40308E803000003000000AF
:1011DA000000000000000000000000000000000005
:1011EA00000000000000000000000000A47A0408CB
:1011FA000000000000000000D515020810270000BA
:10120A0003000000000000000000000000000000D1
:10121A0000000000000000000000000000000000C4
:10122A006C7C040800000000F9ED0208253601086C
:10123A00204E000005000000000000000000000031
:10124A000000000000000000000000000000000094
:10125A00000000001C6A04080000000000000000F2
:10126A0055CF03081027000001000000000000000D
:10127A000000000000000000000000000000000064
:10128A000000000000000000B07A0408000000001E
:10129A000000000095C50008E803000005000000F2
:1012AA000000000000000000000000000000000034
:1012BA00000000000000000000000000BC7A0408E2
:1012CA000000000000000000A9C50108204E00002F
:1012DA000300000000000000000000000000000001
:1012EA0000000000000000000000000000000000F4
:1012FA00CC7A04080000000000000000B1C3010815
:10130A00204E000003000000000000000000000062
:10131A0000000000000000000000000000000000C3
:10132A0000000000DC7A0408000000000000000051
:10133A002D550108400D03000300000000000000C5
:10134A000000000000000000000000000000000093
:10135A0000000000000000005C69040800000000B2
:10136A0000000000A94C020810270000010000003C
:10137A000000000000000000000000000000000063
:10138A00000000000000000000000000F0630408F4
:10139A000000000000000000397702081027000052
:1013AA000300000000000000000000000000000030
:1013BA000000000000000000000000000000000023
:1013CA00EC7A0408000000000000000035E0030881
:1013DA00A0860100010000000000000000000000DB
:1013EA0000000000000000000000000000000000F3
:1013FA0000000000E0630408000000000000000094
:10140A0055DF030850C3000001000000000000007F
:10141A0000000000000000000000000000000000C2
:10142A000000000000000000F47A04080000000038
:10143A0000000000BDDA0308A861000001000000F6
:10144A000000000000000000000000000000000092
:10145A00000000000000000000000000007B0408FB
:10146A000000000000000000E5800208A0860100DC
:10147A000100000000000000000000000000000061
:10148A000000000000000000000000000000000052
:10149A00246A0408000000000000000079F0000837
:1014AA00A00F000001000000000000000000000082
:1014BA000000000000000000000000000000000022
:1014CA00000000000C7B040800000000000000007F
:1014DA00354B03081027000001000000000000003F
:1014EA0000000000000000000000000000000000F2
:1014FA000000000000000000886A040800000000E4
:10150A0000000000C9500208102700000100000076
:10151A0000000000000000000000000000000000C1
:10152A00000000000000000000000000C86304087A
:10153A0000000000000000009D5F03081A4100003F
:10154A000100000000000000000000000000000090
:10155A000000000000000000000000000000000081
:10156A00187B04080000000000000000353602085D
:10157A00400D030000000000000000000000000011
:10158A000000000000000000000000000000000051
:10159A0000000000207B040800000000000000009A
:1015AA00F1350208400D03000000000000000000B1
:1015BA000000000000000000000000000000000021
:1015CA000000000000000000287B04080000000062
:1015DA0000000000B1C70108A08601000300000056
:1015EA0000000000000000000000000000000000F1
:1015FA00000000000000000000000000A8800408AD
:10160A000E000000000000000000000000000000C2
:10161A00C81C0020FFFFFFFFFA00000001000000C5
:10162A0001000000847904080000000000000000A6
:10163A000000000000000000407B040804000000D5
:10164A00E73703080000000000000000E4780408FF
:10165A00010000000000000000000000000000007F
:10166A00000000000D000000000000000000000063
:10167A0000000000EA5E00200100C409000000002A
:10168A00E85E00200100C40900000000E65E0020B8
:10169A000100C40900000000E45E00200100C40942
:1016AA0000000000E05E00200100C4090000000004
:1016BA00E25E00200100C40900000000DE5E002096
:1016CA000100C40900000000DC5E00200100C4091A
:1016DA0000000000607B04080E000000000000000B
:1016EA000000000000000000040F0020F88600201F
:1016FA009CFF2C0100000000D20300200A00000019
:10170A0018430408C48A0020E0150C1700000000E2
:10171A00D10300200800000010420408D003002072
:10172A000500000074420408C68A00200200000076
:10173A0030430408108C00200100FF7F01000000E4
:10174A00088C0020020000003C430408E28A0020C2
:10175A00030000004C430408E18A00200300000053
:10176A004C430408E08B00200000F4010100000053
:10177A00DE8B00200000F40101000000DC8B002059
:10178A000000F40101000000DA8B00200000F401DF
:10179A0001000000D88B002000FF0100F48B00201C
:1017AA00E803D0070A000000F28B00200064010061
:1017BA000A000000F38B0020006401000A00000008
:1017CA00EC8B0020006401000A000000F18B00206D
:1017DA00006401000A000000F08B00200064010090
:1017EA000A000000EF8B0020006401000A000000DC
:1017FA00EB8B002000FF01000A000000EA8B0020AA
:10180A0000FF01000A000000EA8A00200000F4013B
:10181A0001000000E88A00200000F4010100000035
:10182A00E68A00200000F40101000000E48A00209A
:10183A000000F40101000000E78B002000C801004D
:10184A00E68B002000C80100E58B002000C80100DB
:10185A00E48B0020006401000A000000E38B0020F2
:10186A0000FF01000A000000FF8B002000C80100F1
:10187A00FE8B002000C80100FD8B002000C801007B
:10188A00FC8B002000C80100FB8B002000C801006F
:10189A00FA8B002000C80100F98B002000C8010063
:1018AA00F88B002000C80100F78B002000C8010057
:1018BA00687B04080000000000000000000000002F
:1018CA0000000000787B0408090000000000000006
:1018DA00A80F002004000000807B04080900000013
:1018EA00000000009C0F002004000000447F040850
:1018FA000900000000000000900F00200400000012
:10190A00887B04080900000000000000840F002002
:10191A00040000008C7B040809000000000000009D
:10192A00780F002004000000947B040809000000DE
:10193A00000000006C0F0020040000009C7B0408DB
:10194A000900000000000000600F002004000000F1
:10195A00A47B04080900000000000000540F0020C6
:10196A0004000000E4780408010000000000000000
:10197A000000000000000000000000000D00000050
:10198A000000000000000000000000007C7C040849
:10199A00000000000000000000000000000000003D
:1019AA008C7C04080500000000000000E08A00208A
:1019BA0000000000E47804080100000000000000B4
:1019CA000000000000000000000000000D00000000
:1019DA00000000000000000000000000947C0408E1
:1019EA0000000000000000000000000000000000ED
:1019FA00A87304080000000000000000D0050020C1
:101A0A0004000000A07C04080C0000002D38030824
:101A1A000810002000000000D07904080C00000023
:101A2A00A5330308FC0F002000000000F478040826
:101A3A000C00000071330308F00F002000000000C2
:101A4A00647A04080800000000000000E40F002087
:101A5A0004000000547A04080C0000005D330308F7
:101A6A00D80F002000000000A47C04080900000030
:101A7A0000000000CC0F002004000000E0780408F9
:101A8A0003000000695E0308B40F00200000000094
:101A9A00E4780408010000000000000000000000D3
:101AAA0000000000000000000D000000000000001F
:101ABA000000000000000000AC7C040800000000E8
:101ACA00000000000000000000000000BC7C0408C8
:101ADA000C000000000000002010002000000000A0
:101AEA00C47C04080A00000000000000288C0020C2
:101AFA0000000000D07C04080A000000000000007A
:101B0A00308C002000000000D87C04080A00000085
:101B1A0000000000388C002000000000E07C04086F
:101B2A00080000000000000014100020000000005F
:101B3A00E87C040804000000F53C030800000000EB
:101B4A0000000000E4780408010000000000000022
:101B5A000000000000000000000000000D0000006E
:101B6A00000000000000000000000000F47C0408EF
:101B7A00000000000000000000000000000000005B
:101B8A00087D04080C000000000000003810002046
:101B9A0000000000187D040804000000BD3A030894
:101BAA000000000000000000207D04080C00000076
:101BBA00000000002C10002000000000347D040802
:101BCA00040000009D3A0308000000000000000025
:101BDA00E478040801000000000000000000000092
:101BEA0000000000000000000D00000000000000DE
:101BFA0000000000000000003C7D04080000000016
:101C0A00000000000000000000000000507D0408F1
:101C1A00070000000000000074100020000000000F
:101C2A005C7D040808000000000000006810002025
:101C3A0000000000687D04080800000000000000A1
:101C4A005C10002000000000747D040808000000F9
:101C5A00000000005010002000000000807D0408F1
:101C6A0008000000000000004410002000000000EE
:101C7A00E4780408010000000000000000000000F1
:101C8A0000000000000000000D000000000000003D
:101C9A0000000000000000008C7D04080000000025
:101CAA0000000000BB05002000000000987D040829
:101CBA000B00000000000000DC1000200000000003
:101CCA00A07D04080B00000000000000D0100020D6
:101CDA0000000000AC7D04080B00000000000000BA
:101CEA00C410002000000000B87D04080B000000AA
:101CFA0000000000B810002000000000C47D0408A5
:101D0A000B00000000000000AC10002000000000E2
:101D1A00D07D04080B00000000000000A010002085
:101D2A0000000000D87D04080B000000000000003D
:101D3A009410002000000000E47D04080B0000005D
:101D4A00000000008810002000000000F07D040858
:101D5A0008000000000000007C10002000000000C5
:101D6A00E478040801000000000000000000000000
:101D7A0000000000000000000D000000000000004C
:101D8A000000000000000000FC7D040800000000C4
:101D9A00000000000000000000000000107E04089F
:101DAA0008000000000000000C11002000000000E4
:101DBA001C7E04080800000000000000001100203A
:101DCA0000000000287E040808000000000000004F
:101DDA00F410002000000000347E0408080000000F
:101DEA0000000000E810002000000000E478040869
:101DFA0001000000000000000000000000000000D8
:101E0A00000000000D0000000000000000000000BB
:101E1A00000000003C7E04080000000000000000F2
:101E2A00B8050020000000004C7E04080B000000EA
:101E3A00000000003C11002000000000587E040849
:101E4A000B0000000000000030110020000000001C
:101E5A00647E04080700000000000000281100202A
:101E6A0000000000707E0408070000000000000067
:101E7A0020110020000000007C7E040807000000FA
:101E8A00000000001811002000000000E478040897
:101E9A000100000000000000000000000000000037
:101EAA00000000000D00000000000000000000001B
:101EBA0000000000887E0408000000000000000006
:101ECA00B805002000000000947E04080700000006
:101EDA000000000088110020000000009C7E040819
:101EEA000700000000000000801100200000000030
:101EFA00A47E0408070000000000000078110020FA
:101F0A0000000000AC7E040807000000000000008A
:101F1A007011002000000000B47E040807000000D1
:101F2A00000000006811002000000000BC7E0408C8
:101F3A0007000000000000006011002000000000FF
:101F4A00C47E0408070000000000000058110020A9
:101F5A0000000000CC7E040807000000000000001A
:101F6A005011002000000000D47E04080700000081
:101F7A00000000004811002000000000E478040876
:101F8A000100000000000000000000000000000046
:101F9A00000000000D00000000000000000000002A
:101FAA0000000000DC7E04080E00000000000000B3
:101FBA00313503080000000090110020DE8A00205D
:101FCA00170000005C430408DD8A00200A32010081
:101FDA00DC8A002001FA0100D88A002000C801002A
:101FEA00D68A0020E803D00701000000424C55457C
:101FFA004A41594634000000E47E04080E000000FD
:10200A004735030800000000713A03086C120020EB
:10201A00EC7E04080E000000BD3203080000000038
:10202A0000000000BC120020F47E04080E0000002C
:10203A00D53C03088D370308893703089813002015
:10204A00FC7E04080E000000693503080000000049
:10205A00000000004C140020047F04080E00000059
:10206A00F9350308C935030800000000D814002018
:10207A000C7F04080E00000075360308BD360308FD
:10208A000000000078150020E88B00200103010001
:10209A00187F04080E0000009D35030879350308EF
:1020AA000000000068160020207F04080E000000CF
:1020BA0029360308DD3A030800000000F416002060
:1020CA002C7F04080E000000ED360308293B0308A4
:1020DA000000000094170020E28B00200103010099
:1020EA00347F040800000000000000000000000027
:1020FA0000000000407F0408080000000000000003
:10210A00C018002000000000487F040807000000F3
:10211A0000000000B818002000000000587F0408E2
:10212A000700000000000000B018002000000000B6
:10213A00647F04080700000000000000A8180020BF
:10214A0000000000707F04080C000000000000007E
:10215A009C180020000000007C7F04080300000097
:10216A00695E03088418002000000000E47804086F
:10217A000100000000000000000000000000000054
:10218A00000000000D000000000000000000000038
:10219A0000000000847F0408000000000000000026
:1021AA000000000000000000947F04080A000000FC
:1021BA000000000040490408000000009C7F040859
:1021CA000A00000000000000C048040800000000E7
:1021DA00A47F04080A00000000000000008C002010
:1021EA0000000000AC7F04080A00000000000000A4
:1021FA00CC18002000000000E47804080100000068
:10220A0000000000000000000000000000000000C4
:10221A000D000000000000000000000000000000A7
:10222A00B47F040800000000000000000000000065
:10223A0000000000C87F040803000000695E03086C
:10224A000819002000000000D47F040803000000E1
:10225A00695E0308D403002000000000DC7F040844
:10226A0003000000695E0308F01800200000000067
:10227A00E47F040803000000695E0308D818002000
:10228A0000000000E47804080100000000000000DB
:10229A000000000000000000000000000D00000027
:1022AA00000000000000000000000000F07F0408A9
:1022BA000000000000000000000000000000000014
:1022CA00FC7F040807000000753B0308B8190020CA
:1022DA0000000000EC76040803000000695E0308B1
:1022EA00A019002000000000088004080300000074
:1022FA00695E0308881900200000000010800408A5
:10230A0003000000695E0308701900200000000045
:10231A001880040807000000593B030868190020C8
:10232A0000000000EC79040803000000695E03085D
:10233A005019002000000000248004080300000057
:10234A00695E030838190020000000003080040884
:10235A0003000000695E0308201900200000000045
:10236A00E4780408010000000000000000000000FA
:10237A0000000000000000000D0000000000000046
:10238A0000000000000000003C8004080E0000006D
:10239A00F9340308C134030800000000C019002002
:1023AA00448004080E0000005D37030800000000A6
:1023BA0000000000741A0020508004080E0000007B
:1023CA00000000000000000000000000001B0020C8
:1023DA00608004080E00000035370308913B0308AB
:1023EA00000000008C1B0020688004080000000028
:1023FA0000000000000000000000000084720408D1
:10240A0003000000695E0308B01C00200000000001
:10241A005480040803000000695E0308981C002029
:10242A00000000007480040803000000695E0308CD
:10243A00801C0020000000008080040803000000C7
:10244A00695E0308681C00200000000088800408F8
:10245A0002000000815D0308000000000000000087
:10246A009080040802000000815D0308010000005A
:10247A00000000009C80040802000000815D03083F
:10248A000200000000000000000000000D00000033
:10249A0000000000000000000000000009024300E4
:1024AA00020100C0320904000001020201000524F1
:1024BA00001001052401000104240202052406007B
:1024CA0001070582030800FF09040100020A00004F
:1024DA0000070501024000000705810240000000D4
:1024EA00FF000000685E0C004300000000000000CE
:1024FA0000000000000000000000000000000000D2
:10250A00000000000000000043000000000000007E
:10251A0000000000000000000000000000000000B1
:10252A00000000000000000043000000000000005E
:10253A000000000000000000000000000000000091
:10254A00000000000000000043000000000000003E
:10255A000000000000000000000000000000000071
:10256A00000000000000000043000000000000001E
:10257A000000000000000000000000000000000051
:10258A0000000000000000004300000000000000FE
:10259A000000000000000000000000000000000031
:1025AA0000000000000000004300000000000000DE
:1025BA000000000000000000000000000000000011
:1025CA00000000000000000061EF0308A1ED03080D
:1025DA00000000006D8304083B7B0408FB740408B8
:1025EA00FB740408FB740408FB740408FB740408F5
:1025FA00FB740408FB740408FB740408FB740408E5
:10260A00FFFFFFFFFFFFFFFFFFFFFFFFFFFF0000CE
:10261A000100415343494900000000000000000046
:10262A0000000000000000000000000000000000A0
:10263A000000415343494900000000000000000027
:10264A000000000000000000000000000000000080
:10265A0000000000381F00200000000000000000F9
:10266A000000000000000000000000000000000060
:10267A000000000000000000000000000000000050
:10268A000000000000000000000000000000000040
:10269A000000000000000000000000000000000030
:1026AA000000000000000000000000000000000020
:0C26BA0000000000000000000100000013
:1080000070B4EFF31186502383F31288436B1A6820
:10801000D20720D45D686DB9446A826A944217D051
:1080200081691144D9600ED9A21A5A608462002273
:1080300080F858201A6842F00102F1B21A6081F308
:10804000118870BC704701698A1A5A608562EEE730
:10805000012380F85830F3B283F3118870BC704765
:10806000436A8269D154436A0169426B01338B428E
:1080700028BF00234362002A2FD0EFF31182502340
:1080800083F31288436B1968C9072CD470B45E68F7
:108090006EB9456A816A8D4217D084690C44DC60F0
:1080A0000ED9691A59608562002180F85810196844
:1080B00041F00101D2B2196082F3118870BC70479F
:1080C0000469611A59608662EEE7012380F858302E
:1080D000D2B282F3118870BC7047426DD36843F00E
:1080E0008003D3607047D2B282F31188704700BF1B
:1080F000026B10B462B1836CC2684469D11A013B4F
:10810000615C5DF8044B08BF13468364C8B27047D6
:10811000016A4369C4685B5C0131A14228BF114612
:1081200001625DF8044BD8B2704700BF436B13B1D6
:1081300090F858007047836A406A181AB0FA80F0C5
:1081400040097047416A836A99420AD3CB1A416B4E
:10815000026961B14968501E0B4483420AD2C01AB9
:10816000704702691144CB1A416B0029F2D1501EAD
:10817000C01A704700207047036B43B1826C5B6884
:1081800093422FBF981AC0689B1AC0187047C269E3
:10819000036A9A422FBFD01AC0688018C01A70476D
:1081A0000A4B30B503F1180493F900205D78072AD3
:1081B000C8BF143A811804330D7313F8025C855458
:1081C00013F8012C0A76A342EED130BD2C1404081A
:1081D00003682DE9F041DF691FB13B46BDE8F0417E
:1081E0001847002A164611DD04460D460E4400E0ED
:1081F00023689B68204698470028F9D0236815F823
:10820000011B1B6820469847AE42F1D1BDE8F081C2
:1082100010B425212624242200230470417082708A
:10822000C3705DF8044B7047152303701623C370A9
:10823000172383713A2383703B2343713C230372DA
:10824000704700BF30B4846814B12368A5885D838B
:10825000436840F2E93001E0002832D01D8901383E
:1082600015F0020F80B2F7D089B2998140F2E9315E
:1082700001E0002947D01889013910F0010F89B2B7
:10828000F7D0998940F2E93100E059B318890139F2
:1082900010F0020F89B2F8D092B29A8140F2E9321E
:1082A00001E0002A3FD01989013A11F0010F92B282
:1082B000F7D09B8914B12368A2881A83012030BCAF
:1082C000704721498B4204D0A1F574418B42D9D12A
:1082D00002201E4901EB00104189013189B2418120
:1082E0004189CFE7184A934204D0A2F574429342E1
:1082F000E0D10221154B03EB01114B8901339BB2F5
:108300004B814B89D6E71048834203D010498B42FA
:10831000B8D102210D4800EB01114889013080B22B
:1083200048814989AEE708498B4203D0084A934205
:10833000C0D10222054B03EB0212538901339BB2D9
:1083400053815389B6E700BF0030014094B4002048
:10835000003C0040002870B51EDB0928044620DDE3
:10836000012303EB83035B00B0FBF3F2092AF8D887
:108370007BB10E4EB4FBF3F00928CCBF572230225C
:10838000A6FB03E5024403FB1044EB0801F8012BB4
:10839000F0D100230B7070BD2D230B7040420131D2
:1083A000DBE7303001F8010BF3E700BFCDCCCCCCDC
:1083B000884230B44FF001042ED301FB04F4B0FB2B
:1083C000F4F58D42F9D284B1AAB901E0B0FBF4F51D
:1083D000092DCCBF572230222A4404FB150003F894
:1083E000012BB4FBF1F4002CF0D100221A7030BC48
:1083F0007047B0FBF4F5092DCCBF372230222A4458
:1084000004FB150003F8012BB4FBF1F4002CF0D1B0
:1084100000221A7030BC70470546002AEBD1D7E71E
:1084200003685A1C02601970704700BF2DE9F047BD
:10843000089C2578002B804689460CBF4FF0200A07
:108440004FF0300A661C35B3002A29DD334601E0BF
:10845000024698B113F8011B501E0029F8D1971E4F
:1084600060B13D46013D51464046C8476B1C002B5C
:10847000F8DC257827EAE770013055B1041B29465E
:108480004046C847301916F8015B002DF7D1BDE80A
:10849000F087BDE8F087002A04DC2846BDE8F087B5
:1084A0000020EBE7571EDCE783684268D0ED037AD3
:1084B00000EB83010133934281ED040A836004BF22
:1084C0000023836000EB830393ED047A036870EE6E
:1084D000277A9A42C0ED037A77EEC77AC0ED037A25
:1084E0000CDA013307EE103AF8EEC76AB7EE007AFD
:1084F00087EEA60A036030EE070A704707EE102ADF
:10850000B8EEC77A87EE870A704700BF90ED057A0C
:1085100090ED004AD0ED066AD0ED014AD0ED047A24
:1085200090ED035AD0ED025AA4EE007AB0EE406A04
:10853000B0EE470AB0EE667AA6EE247A67EEC07A0D
:10854000A0EE457AE6EE257A80ED057AC0ED067A52
:10855000704700BFD0ED057A90ED013AD0ED003ABA
:10856000D0ED064A90ED024A90ED077A90ED035A5D
:1085700090ED086AD0ED045AC0ED067AF0EE406A3C
:1085800027EE830AC0ED056AA3EEA60A80ED087AFD
:10859000A4EE240AA5EE470AA5EEC60A80ED070A56
:1085A000704700BFD0ED007A90ED017A30EE670A97
:1085B000E7EE007AB0EE670AC0ED007A704700BFC0
:1085C000704700BF0A44914214D030B40139551E9F
:1085D00041F2210211F8014F082380EA042004042B
:1085E0004CBF82EA40004000013B80B2F7D18D428F
:1085F000F0D130BC704700BF2DE9F04FDFF8F8C173
:10860000DFF8F8E1BCF80A70DEF80060BCF80C3066
:10861000BCF808A03C028BB0361B4FF00004CDE93B
:108620000034009CBCF806304FEA17654FF0000795
:1086300067EB0507B946B046A4FB06670024CDE901
:108640000634009C002304FB09770024CDE90034A4
:10865000AAFB0823CDE90223039AF30D00930AFB3A
:1086600009230393009B43EA47230093029B4FEAAD
:10867000D31AFB150193039B4AEA436ADDE9002301
:1086800044464D46CDE90845069C12F5FA62A4FB26
:10869000086743F1000304FB0977CDE90623BCF822
:1086A0000440039BBCF802204FEAE31B230C059314
:1086B00023040493340A44EA07643D12DDE90467A5
:1086C0004FEAC23816EB0A0647EB0B0718EB040813
:1086D000DDE906344FEA524949EB0509B3F5FA6F73
:1086E00074F10004B246BB463CDADDE90067BC0029
:1086F000B20044EA9673B41847EB030522463C46A1
:108700002B4602FB04F406FB0344A2FB062323448E
:10871000940844EA83749D105B104FEA3202B8EB70
:10872000040869EB0509BAEB020A6BEB030BDDE900
:108730000623304C4FF0FF35A242AB412CDBDDE984
:108740000856A5FB052305FB06F403EB4403D40FF1
:1087500044EA4304DD17DDE90623121B63EB05033E
:10876000CDE90623DEF80440A4FB082304FB09330B
:10877000540D44EAC3245D15B4EB0A0A65EB0B0BF8
:108780004FEADA3343EA4B4300B1036009B1069B79
:108790000B600BB0BDE8F08F40F6AC52B4184FF050
:1087A000000347EB03052246A2FB022304FB05F46A
:1087B00003EB4403941843EB0305A4185D414FEA0F
:1087C000850CA6004CEA947CB41A6CEB0305DF0020
:1087D000D6006D104FEA340447EA5277921B63EBE0
:1087E0000703B8EB040869EB05091AEB020A4BEB27
:1087F000030BA4E724FAFFFF708600209C1F0020D3
:1088000050F8043C012280F84520103803B1184785
:10881000704700BF4FF40063838270474FF40063DA
:1088200083827047BFF34F8F0549064BCA6802F435
:10883000E0621343CB60BFF34F8F00BFFDE700BF83
:1088400000ED00E00400FA05F8B5057B4669036811
:108850001F2D29D9A5F120045F682021A1400F42D6
:108860002A4613D01022A240D960DA605A68E2404A
:10887000D10703D5012202FA04F4DC600446304635
:10888000FFF7BEFB227B23681F2A20D9A2F120001C
:1088900008215A688140114200D0D96004225968E9
:1088A00082400A4221D1F8BD20211C68A9400C4217
:1088B0002A460CD01022AA4099609A601A68EA40B1
:1088C000D207DBD5012202FA05F59D60D6E7082123
:1088D00018689140014200D099600421186801FA9B
:1088E00002F2024203D09A60F8BDDA60F8BDF8BD2A
:1088F00070B4037B04681F2B08D9203B20216268D9
:1089000001FA03F31A421CD170BC7047202122687F
:1089100001FA03F31A42F7D042691449582000FBC8
:10892000021251685689CD680868296821F0010152
:108930002960828992B222EA06028281A36070BC19
:10894000704742690949582000FB02125168568954
:10895000CD680868296821F001012960828992B2F6
:1089600022EA06028281E36070BC704770600020DA
:1089700030B4094B1C786CB1084A002502EBC404E2
:10898000116893884D628889083203439BB2A242E2
:108990008B81F5D130BC70473063002034630020F8
:1089A00010B4037B01681F2B09D9203B20224C689F
:1089B00002FA03F31C4214D15DF8044B70472022E5
:1089C0000C6802FA03F31C42F6D00C4A40680024FB
:1089D000147002685DF8044B22F0010202608B60A3
:1089E0007047064A40680024147002685DF8044B22
:1089F00022F001020260CB60704700BF1B9B002089
:108A0000F0B5C40022189200AE498B585B689D8A6D
:108A1000ADB2EEB2F7070A445CD4B70732D5BFF364
:108A20005F8F167EF6B2012E00F0C780A64D1A8B1E
:108A3000BFF35F8F221801EB8202167E022E00F038
:108A4000D580221801EB8202167E032E00F088806A
:108A50009A8895F9086092B242F480629A8022184E
:108A600001EB8202127E013296425BD1AA7A002685
:108A70006E72002A40F09580204401EB80000023B4
:108A80004375F0BD77074ED416F0400600F0C9805C
:108A90008D4D1E8A95F908E0176AF6B207F80E6048
:108AA0005FFA8EFE0EF1010C4FFA8CFC177E85F8F2
:108AB00008C00CF103029742664600F01C812218A0
:108AC00001EB8202127E9445C9D10EF1020676B204
:108AD0002E72C4E71E887C4D26F400663604360CE0
:108AE0001E801E88B6B246F480661E80967E0027E1
:108AF0002F72002E48D06E7A002E42D0221801EB41
:108B000082020126127E6E72022A00F0B9802218BB
:108B100001EB8202927D42F001021A82204401EBB5
:108B20008000037EF0BD684D967E0127AF72002E57
:108B300073D06E7A002E7BD1221801EB8202527E16
:108B4000002A00F0A3801A882E7A92B2013642F4ED
:108B5000007276B21A802E721A88D205FCD47EE793
:108B6000927E002A3FF474AF6A7A002A3FF470AF15
:108B70009A8895F9086022F480621204120C9A8097
:108B80006DE7D27DFF2AB9D0221801EB8202967DD3
:108B900006F0FE061E82D37DFF2BBFD0FF232B7273
:108BA000BCE79A8822F4407212042044120C01EBB4
:108BB00080009A8000234375F0BD927E424D002ACA
:108BC0003FF435AF6A7A002A3FF431AF1A8822F4B5
:108BD00080621204120C1A80BFF35F8F1A8B1A88FE
:108BE000AE7292B242F400721A8031E7927E002A8D
:108BF0003FF427AF6A7A002A3FF423AF1A8895F929
:108C0000086022F480621204120C1A809A8822F4FE
:108C100080621204120C9A8021E76A7A002A8BD0B3
:108C200091E715F0800F284D3AD195F9086016E7C5
:108C3000167ED2F820E01F88022E95F9086045D9EB
:108C400027F480673F043F0C1F801F8AFFB20EF895
:108C500006701F88D2F820E0BFB247F400771F806B
:108C6000F2B21F8A561C76B2FFB20EF806709F88C9
:108C7000961CBAB276B242F480622E729A806BE78A
:108C80001A8892B242F400621A8040E71A8895F975
:108C9000086092B242F4807201271A806F725BE71B
:108CA00095F90870B7F1FF3F2CD0D669F65D1E82AA
:108CB00092F818E001377AB2964516462A727FF488
:108CC000CEAEA3E7103900209C1F0020BFB247F4AE
:108CD00000771F801F8AFFB20EF80670F6B21F8A57
:108CE000D2F820E0721C52B20336FFB276B20EF810
:108CF00002702E7230E79A8822F480621204120CFD
:108D00009A80DCE6D77D1F822E72957E1DB9127E79
:108D1000002A7FF403AF9A8822F480621204120CB6
:108D20009A80FBE670B5044682B01430E56D0623E8
:108D30006A464321A847B0B19DF804009DF8006041
:108D40009DF801109DF802509DF803209DF8053014
:108D500041EA062143EA002342EA0522A187E2878D
:108D6000A4F84030012002B070BD00BF70B50446C9
:108D700082B00830656A06236A463B21A847A8B13D
:108D80009DF804009DF800609DF801109DF80250C8
:108D90009DF803209DF8053041EA062143EA0023AF
:108DA00042EA0522E18222836383012002B070BD82
:108DB0000023036043608360282303702923C3706A
:108DC0000123837143727047F8B50468C4F30D043E
:108DD00005460E4604B32F6828F06AF8092840F0CB
:108DE0008880454C236923F440732361236943F44D
:108DF00000732361236943F0010323613E6028F07F
:108E000057F82369092823F00103236171D12B68E6
:108E100004332B600020F8BD384B394A93422BD9DC
:108E200002F58042934226D902F5804293422AD924
:108E300002F58042934228D902F58032934226D926
:108E400002F50032934224D902F50032934222D92E
:108E500002F50032934220D902F5003293421ED926
:108E600002F5802293421CD9B3F1016F1BD3052078
:108E700005F06CFAFBE7082428F01AF8092814D04A
:108E80004FF0FF30F8BD1024F6E71824F4E7202453
:108E9000F2E72824F0E73024EEE73824ECE740241A
:108EA000EAE74824E8E75824E6E7134F3B6923F450
:108EB00040733B613B6943F400733B613B6923F0C2
:108EC000F8033B613B6943F002031C433C613B698F
:108ED00043F480333B6127F0EBFF3B6923F002034F
:108EE0003B613B69092823F0F8033B613FF473AF12
:108EF000C6E76FF00100F8BD003C024000400008EA
:108F0000FF3F0008F8B504460D468E180027B5420D
:108F100001D12069F8BDE368591CE160234415F8CC
:108F2000012B1A720429F2D1206918B9A1682046D0
:108F3000FFF74AFF2061E760E9E700BF70B582B044
:108F40000446694614302FF0FDFDB0B19DF80500D0
:108F50009DF801609DF802109DF803509DF80420D3
:108F60009DF8063041EA062143EA002342EA052241
:108F7000A187E287A4F84030012002B070BD00BF95
:108F800038B5254B1C68236B73B1636D626BCAB136
:108F9000998A1A88C90592B201D5D20700D438BD82
:108FA0004FF6F7721A8038BD636D99891A88890661
:108FB00092B2EBD59206E9D5E26ACAB1988880B23E
:108FC0009047E2E799891A880D0692B2E0D510061B
:108FD000DED5A26A616A8A4219D0A1692569885CD6
:108FE00098800132B2FBF5F105FB1122A262CFE7B6
:108FF0009B88E2696169DBB28B54E269E068636D6A
:109000000132B2FBF0F100FB1122E261BEE7DA6847
:1090100022F08002DA60BBE7E838002003685B6A70
:1090200003B11847704700BF03681B6A03B11847B4
:10903000704700BF03682DE9F041DF691FB13B466F
:10904000BDE8F0411847002A164611DD04460D46DA
:109050000E4400E023689B68204698470028F9D01A
:10906000236815F8011B1B6820469847AE42F1D1D2
:10907000BDE8F08103689B69184700BF03685B691E
:10908000184700BF03681B69184700BF0368DB6807
:10909000184700BF03689B68184700BF03685B68F8
:1090A000184700BF03681B68184700BF014B1868CA
:1090B000F8E700BF28BD002038B50C46097849B153
:1090C000054601342B6828461B68984714F8011B95
:1090D0000029F7D138BD00BF064B53F820302BB123
:1090E0001A689B8851690B4201D1138370475383DF
:1090F000704700BFB0BC002003682DE9F04F03F1BA
:109100003F4404F57E04604EA40A0125345D04F05A
:109110001F066409032C05FA06F500F0AF80042C45
:1091200000F0A780022C54D08588B5FA85F0C0F1F4
:109130001F0080B2C40803EB840400F00700266A15
:1091400080000F27874026EA07062662276A01F07B
:10915000030602FA00F0721E3843012AC1F3810CA3
:10916000C1F300182062C1F3411137D9002422460F
:1091700001274FF0030E03E0102A04F1020426D069
:1091800007FA02F0A84302F10102F5D1D3F800C0BA
:109190000EFA04F0C04300EA0C0CC3F800C0D3F888
:1091A000008006FA04FC4CEA080CC3F800C0D3F8AF
:1091B0000CC000EA0C00D860D3F80CC001FA04F02F
:1091C00040EA0C00102AD86004F10204D8D1BDE8AE
:1091D000F08F2E4C666C35436564A5E7002002468F
:1091E0004FF0010E4FF0030904E00132102A00F1A4
:1091F00002003CD00EFA02F737EA0504F5D1D3F8A5
:1092000000A009FA00F4E4430AEA040AC3F800A043
:10921000D3F800B006FA00FA4AEA0B0AC3F800A035
:10922000D3F808A004EA0A0AC3F808A0D3F808B0E3
:109230000CFA00FA4AEA0B0AC3F808A0D3F804A013
:109240002AEA07075F60D3F804A008FA02F747EAA2
:109250000A075F60DF683C40DC60DF6801FA00F409
:1092600001323C43102ADC6000F10200C2D1BDE8AB
:10927000F08F064C266B3543256355E7034C266C6F
:109280003543256450E700BF90460408003802408B
:10929000026802F13F4303F57E032DE9F04F9B0A7C
:1092A000544DEB5C03F01F055B090124032B04FA0A
:1092B00005F400F09980042B00F09180022B3ED041
:1092C00001F00306731E012BC1F3810CC1F30018DA
:1092D0008588C1F3411137D90024234601274FF077
:1092E000030E03E0102B04F1020426D007FA03F06A
:1092F000A84303F10103F5D1D2F800C00EFA04F03F
:10930000C04300EA0C0CC2F800C0D2F8008006FA94
:1093100004FC4CEA080CC2F800C0D2F80CC000EA09
:109320000C00D060D2F80CC001FA04F040EA0C0046
:10933000102BD06004F10204D8D1BDE8F08F2E4B81
:109340005D6C2C435C64BBE7002003464FF0010ECC
:109350004FF0030904E00133102B00F102003CD070
:109360000EFA03F737EA0504F5D1D2F800A009FA9E
:1093700000F4E4430AEA040AC2F800A0D2F800B0FC
:1093800006FA00FA4AEA0B0AC2F800A0D2F808A0CE
:1093900004EA0A0AC2F808A0D2F808B00CFA00FAE7
:1093A0004AEA0B0AC2F808A0D2F804A02AEA070782
:1093B0005760D2F804A008FA03F747EA0A07576093
:1093C000D7683C40D460D76801FA00F401333C43CD
:1093D000102BD46000F10200C2D1BDE8F08F064B23
:1093E0001D6B2C431C636BE7034B1D6C2C431C64EF
:1093F00066E700BF904604080038024010B5040933
:10940000013C032C17D80D4B33F8142000F00F004B
:1094100042FA00F313F001030DD0012303FA00F028
:109420000138104035F0D4FB054A064B125D10445C
:1094300003EBC00010BD002010BD00BFC0440408F5
:10944000C844040870A800202DE9F04F4A484B4951
:109450004B4B4C4C4FF0010A4FF002094FF00408FF
:109460004FF0080C4FF0100E20274026802530F8D2
:10947000022B12F0010F03D01960A3F804A00833E7
:1094800012F0020F03D01960A3F80490083312F011
:10949000040F03D01960A3F80480083312F0080FFA
:1094A00003D01960A3F804C0083312F0100F03D0E2
:1094B0001960A3F804E0083312F0200F02D01960FD
:1094C0009F80083312F0400F02D019609E8008334D
:1094D00012F0800F02D019609D80083312F4807F53
:1094E00005D04FF4807B1960A3F804B0083312F460
:1094F000007F05D04FF4007B1960A3F804B0083357
:1095000012F4806F05D04FF4806B1960A3F804B09B
:10951000083312F4006F05D04FF4006B1960A3F804
:1095200004B0083312F4805F05D04FF4805B1960FB
:10953000A3F804B0083312F4005F05D04FF4005BC9
:109540001960A3F804B0083312F4804F05D04FF42B
:10955000804B1960A3F804B00833D20B04D04FF449
:10956000004219609A80083301F58061A1427FF4BE
:109570007EAFBDE8F08F00BFC04404080000024089
:1095800070A800200010024000286AD003682DE96E
:10959000F04F03F13F4404F57E045F4EA40A012519
:1095A000345D04F01F066409032C05FA06F559D052
:1095B000042C00F0AC80022C59D08588B5FA85F0D7
:1095C000C0F11F0080B2C40803EB840400F0070060
:1095D000266A80000F27874026EA07062662276A48
:1095E00001F003068240701E3A430128C1F3810C4A
:1095F000C1F300182262C1F341113DD90024224673
:1096000001274FF0030E03E0102A04F1020426D0D4
:1096100007FA02F0A84302F10102F5D1D3F800C025
:109620000EFA04F0C04300EA0C0CC3F800C0D3F8F3
:10963000008006FA04FC4CEA080CC3F800C0D3F81A
:109640000CC000EA0C00D860D3F80CC001FA04F09A
:1096500040EA0C00102AD86004F10204D8D1BDE819
:10966000F08F70472D4C266C35432564A5E72B4CB5
:10967000666C35436564A0E7002002464FF0010E9A
:109680004FF0030904E00132102A00F102003CD03F
:109690000EFA02F737EA0504F5D1D3F800A009FA6B
:1096A00000F4E4430AEA040AC3F800A0D3F800B0C7
:1096B00006FA00FA4AEA0B0AC3F800A0D3F808A099
:1096C00004EA0A0AC3F808A0D3F808B00CFA00FAB2
:1096D0004AEA0B0AC3F808A0D3F804A02AEA07074D
:1096E0005F60D3F804A008FA02F747EA0A075F6050
:1096F000DF683C40DC60DF6801FA00F401323C4383
:10970000102ADC6000F10200C2D1BDE8F08F034CEA
:10971000266B3543256350E7904604080038024025
:10972000002855D0026802F13F4303F57E032DE97E
:10973000F04F9B0A544DEB5C03F01F055B090124BD
:10974000032B04FA05F444D0042B00F09780022B7D
:1097500044D001F00306731E012BC1F3810CC1F349
:1097600000188588C1F341113DD900242346012703
:109770004FF0030E03E0102B04F1020426D007FA89
:1097800003F0A84303F10103F5D1D2F800C00EFAAB
:1097900004F0C04300EA0C0CC2F800C0D2F800800C
:1097A00006FA04FC4CEA080CC2F800C0D2F80CC05F
:1097B00000EA0C00D060D2F80CC001FA04F040EAD4
:1097C0000C00102BD06004F10204D8D1BDE8F08F5A
:1097D00070472E4B1D6C2C431C64BAE72B4B5D6C01
:1097E0002C435C64B5E7002003464FF0010E4FF0B8
:1097F000030904E00133102B00F102003CD00EFA03
:1098000003F737EA0504F5D1D2F800A009FA00F40D
:10981000E4430AEA040AC2F800A0D2F800B006FA4B
:1098200000FA4AEA0B0AC2F800A0D2F808A004EA3B
:109830000A0AC2F808A0D2F808B00CFA00FA4AEAFC
:109840000B0AC2F808A0D2F804A02AEA070757605A
:10985000D2F804A008FA03F747EA0A075760D76866
:109860003C40D460D76801FA00F401333C43102B2C
:10987000D46000F10200C2D1BDE8F08F034B1D6B34
:109880002C431C6365E700BF904604080038024083
:1098900038B5044690F8590000285AD104F114054F
:1098A000236E80226B2128469847642005F016FA23
:1098B000236E0722682128469847642005F00EFA97
:1098C000236E00226B2128469847642005F006FA93
:1098D000236E01226B21284698470F2005F0FEF9E0
:1098E00094F85320236E032A8CBF1A2218221B21BE
:1098F000284698470F2005F0F1F9236E18221C2105
:10990000284698470F2005F0E9F9236E94F8522075
:109910001A21284698470F2005F0E0F9236E94F8A5
:109920005420192128469847642005F0D7F9236E62
:1099300010223721284698470F2005F0CFF92846F6
:10994000236E0122382198470F20BDE8384005F0EA
:10995000C5B9FFF753FD0546D0B12023002183711F
:10996000C171FFF7DDFE21460F4B41F8103F28463D
:1099700033F07CFAAB88B3FA83F3C3F11F030122FF
:1099800012FA03F38AD009490A6813430B6085E78A
:109990000146FFF7C5FE2146034B41F8103F28461C
:1099A00033F064FA7AE700BF01880008003C014008
:1099B00010B1036882885A83704700BF10B10368F2
:1099C00082881A83704700BF18B10368828809B97A
:1099D0005A8370471A83704710B40A4B0A4A1C789E
:1099E00001238340234052F8200029B9B3FA83F1C0
:1099F00049095DF8044BE7E7191C18BF01215DF820
:109A0000044BE1E7ACBC0020B0BC002030B10368DF
:109A100082881B691A4214BF01200020704700BFD2
:109A20002DE9F0410B4E346873691C400FD0DFF80C
:109A300028800127B4FA84F3C3F11F0307FA03F562
:109A400058F8230003689847AC437561F2D1BDE82C
:109A5000F08100BF003C0140E0BC00202DE9F04156
:109A60000B4E346873691C400FD0DFF82880012743
:109A7000B4FA84F3C3F11F0307FA03F558F823007F
:109A800003689847AC437561F2D1BDE8F08100BF2F
:109A9000003C0140E0BC00202DE9F0410B4E346851
:109AA00073691C400FD0DFF828800127B4FA84F3D3
:109AB000C3F11F0307FA03F558F82300036898471A
:109AC000AC437561F2D1BDE8F08100BF003C0140BC
:109AD000E0BC00202DE9F0410B4E346873691C4056
:109AE0000FD0DFF828800127B4FA84F3C3F11F03F5
:109AF00007FA03F558F8230003689847AC437561EB
:109B0000F2D1BDE8F08100BF003C0140E0BC002084
:109B10002DE9F0410B4E346873691C400FD0DFF81B
:109B200028800127B4FA84F3C3F11F0307FA03F571
:109B300058F8230003689847AC437561F2D1BDE83B
:109B4000F08100BF003C0140E0BC00202DE9F04165
:109B50000B4E346873691C400FD0DFF82880012752
:109B6000B4FA84F3C3F11F0307FA03F558F823008E
:109B700003689847AC437561F2D1BDE8F08100BF3E
:109B8000003C0140E0BC00202DE9F0410B4E346860
:109B900073691C400FD0DFF828800127B4FA84F3E2
:109BA000C3F11F0307FA03F558F823000368984729
:109BB000AC437561F2D1BDE8F08100BF003C0140CB
:109BC000E0BC0020084A094808B5536C43F48043C0
:109BD00053640021402237F074FB054B4FF0FF32F5
:109BE0001A60C3F8032008BD00380240E0BC002022
:109BF00020BD002003685B6A184700BF2DE9F041D3
:109C0000044618460D461646984634F037FB27683A
:109C1000E6722844A07229467D69434632462046B2
:109C2000AC46BDE8F0416047036810B504461B68C8
:109C30009847236820469B689847A37B0133A3730A
:109C400010BD00BF10B5036804469B689847FF230A
:109C500001226373227310BD08B5FFF7CFFB38B143
:109C60002C2282710022C2712021BDE8084057E5F4
:109C700008BD00BF40F2E93300E0A3B10289013B17
:109C800012F0020F9BB2F8D089B2818140F2E93321
:109C900000E043B10289013B12F0010F9BB2F8D002
:109CA0008089C0B27047094A904205D0084B98425B
:109CB00001D0FF2070470223064A02EB03135A89A2
:109CC000013292B25A815889C0B2704700300140C7
:109CD000003C004094B4002010B5014600BF064B84
:109CE000DC68A068FFF764FE6068FFF7C3FFA06848
:109CF000FFF764FE00BF10BD9C1F0020144B98426C
:109D000024D003F58063984220D0028822F04002DC
:109D10001204120C0280028822F038031B041B0C70
:109D200059B141F48071002991FAA1F2B2FA82F19D
:109D300008BF4FF0FF310139C9000B439BB20380CC
:109D400003889BB243F04003038070474908DCE777
:109D50000038004010B5802104468069FFF7CEFF2F
:109D6000012004F061FF2046FFF792FD10226A21D6
:109D700004F11400FEF766FA642004F0AFFFA06956
:109D80000421FFF7BBFF0120BDE8104004F04CBFE9
:109D9000F0B484894FF6FF764FF47A7443B3002908
:109DA00038D00F78013101E0B4421AD00589013C66
:109DB00015F00205A4B2F7D0BCB284814FF47A74D6
:109DC00002E0BCB2B4420CD0058915F0010504F1E3
:109DD000FF37F6D08589ADB20AB115700132013B6B
:109DE000DCE70D4B984207D0A3F57443984202D0AC
:109DF0000120F0BC70470225084B03EB05156B8969
:109E000001339BB26B81688980B2003018BF01209A
:109E1000F0BC7047FF27C9E70030014094B4002030
:109E200070B50546806810B104688088608341F091
:109E30008001686840F2E93400E0E4B10689013C41
:109E400016F0020FA4B2F8D089B2818140F2E93154
:109E500000E009B30489013914F0010F89B2F8D088
:109E600081890021FFF794FFAB6813B11A689B88C2
:109E70001383012070BD1049884204D0A1F57441BC
:109E80008842EED102240D4901EB041461890131AD
:109E900089B261816189E4E7074CA04203D0084997
:109EA0008842DED10221054C04EB01114C890134BA
:109EB000A4B24C814989D4E70030014094B4002019
:109EC000003C0040F8B50501684C694B62596119C6
:109ED0009A4204EB050704BF01230B730646387A48
:109EE00032F06EFB3B7A03F01F015B090122032B6A
:109EF00002FA01F26DD0042B66D0022B5CD06319FC
:109F000001361879FFF77AFAF6B2074610B1122334
:109F1000C671837163195879FFF770FA10B1132372
:109F2000C671837163199879FFF768FA10B1142329
:109F3000C671837166190A21F2793846FFF724FB4E
:109F40007079FFF75BFAF2790A21FFF71DFBB07910
:109F5000FFF754FAF2790A21FFF716FB6359454AD5
:109F6000934247D0444A934250D0414A934259D0F9
:109F7000424A934262D0424A93426BD0414A934252
:109F80002CD02C44227BE2B901200222198801F452
:109F9000415141F445710A4302431A809A8B22F4DD
:109FA00000621204120C07219A8319821A8892B255
:109FB00042F040021A80F8BD334B596A0A435A6294
:109FC0009DE700200246E1E72F4B19690A431A6119
:109FD00095E72D4B196A0A431A6290E702F564422D
:109FE0004FF40010536A43F40013536226F058FEF6
:109FF0006359C6E702F584324FF48050536A43F444
:10A000008053536226F04CFE6359BAE702F50032E2
:10A010004FF48040136A43F48043136226F048FEF5
:10A020006359AEE702F5FE324FF40040136A43F481
:10A030000043136226F03CFE6359A2E702F5823228
:10A040004FF40050536A43F40053536226F028FE45
:10A05000635996E702F568424FF48010536A43F45F
:10A060008013536226F01CFE63598AE794B40020E3
:10A07000003C004000300140003800400034014006
:10A08000005001400054014000380240427A02B9B9
:10A09000704710B504460368406804F10A01984708
:10A0A0000023637210BD00BF437A5A1C0344D2B22E
:10A0B00042729972037A934200D802B9704710B580
:10A0C00004460368406804F10A019847002363725C
:10A0D00010BD00BF302827D0312827D0322827D004
:10A0E000332827D0342827D0352827D0202827D038
:10A0F000212827D0102827D0112827D0122827D090
:10A10000132827D0142827D0152827D0162805D0A3
:10A11000172808BF0F2202D0002070470E22104BD4
:10A1200003EB4203587E70470022F8E70122F6E76E
:10A130000222F4E70322F2E70422F0E70522EEE729
:10A140000622ECE70722EAE70822E8E70922E6E729
:10A150000A22E4E70B22E2E70C22E0E70D22DEE729
:10A160002C14040870B5448806460D46C4F30B044D
:10A1700022460021284637F0A4F83369094A934261
:10A1800009D3094A934206D2224628461946BDE819
:10A19000704034F017BE23B121462846BDE8704018
:10A1A000184770BD240600082A070008064B074917
:10A1B0008B4202D30023184670471A88C2F30B0261
:10A1C0009042F8D01433F3E7880100082406000811
:10A1D000024A136823EA000010607047248C0020B4
:10A1E000F8B5174D2B78A32B28D16B78BE2B25D132
:10A1F000022229464FF6FF70FEF7E4F9114FAC1C1E
:10A2000022884AB1A618BE4218D2052A16D921467C
:10A21000FEF7D8F93446F3E721460222FEF7D2F9D9
:10A220000222A118FEF7CEF90634074B641B1C80EE
:10A2300041F60F53C31A58425841F8BD0020F8BDEB
:10A2400000400008008000081A3B00202DE9F04F74
:10A25000DFF84C914D4F8BB00326A7EB090718226E
:10A26000002104A837F02DF8494BCDF81090059740
:10A270001A69002A04DA474A5A6002F188325A60A1
:10A2800001228DF82420F322DA60434B434C1B88D3
:10A29000ADF800300222694604A8FEF733FE022220
:10A2A00069464FF6FF70FEF78DF9DFF8F8A080469B
:10A2B0004FF0000B544539D30AAC002524F8245D37
:10A2C0000222214604A8FEF71DFE02222146404636
:10A2D000FEF778F940BAC043ADF80800022202A99F
:10A2E00004A8FEF70FFE079878B106ABC0F1040290
:10A2F0002946184436F0E5FF089818B9069904A8CD
:10A30000FEF762FD0023089007939DF82430089A19
:10A3100023B11F490B6943F000430B61013E2DD06F
:10A32000002A9CD1FFF75CFF50B32CE065888DF8C4
:10A330000DB0C5F30B05AB1DADF808302388C3F392
:10A340000B02ADF80A201B0B062202A904A88DF807
:10A350000C30FEF7D7FD062202A94046FEF732F97F
:10A36000616880462A4604A8FEF7CCFD6168404635
:10A370002A46FEF727F9143480469BE7002AD1D0FD
:10A38000052003F0E3FF0BB0BDE8F08F008000086C
:10A39000003C02402301674564140408880100085A
:10A3A00000400008240600080378202B024600F134
:10A3B0000100F9D0092BF7D02D2B2CD02B2B03BF6C
:10A3C0005378B7EE000A0246B7EE000AA3F1300157
:10A3D000C8B209289FED467A10D8F2EE046A07EE5B
:10A3E000901AF8EEE77A12F8013FE7EE267AA3F129
:10A3F0003001C8B20928B0EE677AF0D92E2B4CD0C4
:10A4000003F0DF03452B0BD0F7EE007A67EE276AE7
:10A4100020EE260A70475378BFEE000A0246D5E7C1
:10A4200010B451782D2959D02B290ABF9178501C8E
:10A43000901C0024A1F13003092B53D8002303EB17
:10A44000830301EB430310F8011FA1F13002092A35
:10A45000A3F13003F3D9B3F59A7F28BF4FF49A7371
:10A46000072B42D9DFED236A1A46F7EE007A083A45
:10A47000072A67EEA67AFAD803F007032BB1F2EEAB
:10A48000046A013B67EEA67AFBD124B3C7EE276AC4
:10A490005DF8044B20EE260A70475378A3F1300193
:10A4A000C8B2092802F10102AAD8F2EE046AF0EE5D
:10A4B000665A07EE901AF8EEE77A12F8013F87EE37
:10A4C000A66AA3F13001C8B2092866EEA56A37EE84
:10A4D000067AEED994E767EE276AD9E7901C91785F
:10A4E0000124A7E7F7EE007ACFE7F7EE007AC5E799
:10A4F0000000000020BCBE4CB5EEC00ADFED317A92
:10A50000F1EE10FACCBF30EE270A30EE670ADFED2D
:10A510002E7A20EE270A30B5FDEEC07A87B017EE0E
:10A52000904A054684EAE470002303A9A0EBE47096
:10A5300001930093029323F001FE002CACBF202373
:10A540002D2303A88DF8003033F098FE012803A9CD
:10A5500024D002282DD0032805BF30236846684642
:10A560008DF8013036F0D3FE684633F087FE0338AD
:10A57000C4B222466946284636F027FF00232B55F1
:10A58000284633F07BFE2E22431C2A540DEB040197
:10A59000E81836F0D9FE284607B030BD30236846AB
:10A5A0008DF801308DF802308DF8033036F0AFFEB3
:10A5B000DAE7302368468DF801308DF8023036F046
:10A5C000A6FED1E76F12033A00007A442DE9F0416C
:10A5D000064615460846B6FBF2F43CB905FB146482
:10A5E000124B1B5D00F8013BBDE8F081B4FBF2F7B4
:10A5F00067B90E4B05FB174705FB1464DA5D00F8DD
:10A60000012B1B5D00F8013BBDE8F081B7FBF2F8C0
:10A61000B8F1000F02D04046FFF7D8FF05FB1878CD
:10A62000024B13F8082000F8012BE3E77C480408EC
:10A6300030B402681146531C036011F8024B0160EC
:10A64000D31C517803609378151D05601B0443EA01
:10A650000123D078234343EA006030BC704700BF39
:10A660000368591C1A46016012F8021B02605878F0
:10A6700041EA0020704700BF03685A1C0260187846
:10A68000704700BF38B504460068154634F09AFBA1
:10A6900022682A44226038BD036810B40A0E5C1C8C
:10A6A00004601A7003680A0C5C1C04601A7003686A
:10A6B0000A0A5C1C04601A7003685A1C0260197054
:10A6C0005DF8044B704700BF036810B40A0A5C1CB5
:10A6D00004601A7003685A1C026019705DF8044B1C
:10A6E000704700BF03685A1C026010B419700368F9
:10A6F0000A0A5C1C04601A7003680A0C5C1C046083
:10A700001A700368090E5A1C026019705DF8044B38
:10A71000704700BF03685A1C026019700368090A79
:10A720005A1C0260197070472DE9F047002488B068
:10A7300080460F461E46A14605AD531C0393117873
:10A7400039B3252933D1931CCDF810900393507859
:10A7500030284ED04FF0000AA0F13003DBB2092BB5
:10A7600042D96C2819D0642800F0938024D8252879
:10A770001CD063D9582876D063281BD13178404645
:10A78000B847039A531C0393117804360134002907
:10A79000D7D1204608B0BDE8F087039B5A1C03922E
:10A7A0001B78642B7CD02AD8252B54D125214046F8
:10A7B0000134B847039AC0E7732833D044D97528C9
:10A7C0004FD106F1040E30682B4600220A2176464E
:10A7D000FDF7EEFD049A0095534639464046FDF7D5
:10A7E00025FE039A0444A8E704AA03A923F082FCE7
:10A7F000B7E7D31C039390784FF0010AACE7732BB3
:10A8000010D05BD9752B3AD0782B96D1A3F1580292
:10A81000B2FA82F2306852092B4610210436FDF755
:10A82000C7FDD7E73368049A0093394600234046B2
:10A83000FDF7FCFD04360444039A7EE70028B9D1F5
:10A84000204608B0BDE8F0876E28B3D1039A33687C
:10A8500004361C6071E72AD9582BD7D0632B8DD0D2
:10A860006BE77828A6D1A0F15802B2FA82F23068DC
:10A8700052092B461021FDF79BFD0436AAE706F18D
:10A88000040E30682B4600220A217646FDF790FD23
:10A89000A0E7331D306829461E46FDF75BFD99E7AA
:10A8A000331D306829461E46FDF754FD92E7002B04
:10A8B0007FF443AF204608B0BDE8F0876E2BC6D0CA
:10A8C0003BE700BF0EB400B584B005AB019053F870
:10A8D000042B0649039301A8FFF726FF019B0022E2
:10A8E0001A7004B05DF804EB03B0704721840008CF
:10A8F0000FB430B583B006AB0A490B4853F8042BAC
:10A90000096800680193FFF70FFF084C05462068AF
:10A91000FEF7B4FB0028FAD0284603B0BDE830406B
:10A9200004B07047DC380020E038002028BD00204B
:10A93000DFED2B7AB4EEE70AF1EE10FA4ADDDFED37
:10A94000296A9FED297A01E0B0EE670AB4EEC70AE2
:10A95000F1EE10FA70EE667AF6DC9FED247AF4EEF2
:10A96000C77AF1EE10FA38D5DFED1E6A9FED207A36
:10A9700001E0F0EE407AF4EEC77AF1EE10FA37EE2D
:10A98000A60AF6D4DFED1B7AB4EEE70AF1EE10FA70
:10A9900014DDDFED137A37EEC00A60EE006A9FED3A
:10A9A000166A9FED167ADFED167AA6EE867A20EE0D
:10A9B000266AE6EE877AA6EE270A7047DFED117A5F
:10A9C000B4EEE70AF1EE10FA44BFDFED087A37EE95
:10A9D000C00AE2E7F0EE407ABFE7B0EE670AD1E7DF
:10A9E000DB0F4940DB0FC940E4CB1641DB0F49C008
:10A9F000E4CB16C1DB0FC93F92E741B99730083C61
:10AA000015A82ABEDB0FC9BF80EAE073A3EBE07391
:10AA10008B4205DB002801DD401A704702D17047E8
:10AA2000002070470844704709B909E0194690FBB7
:10AA3000F1F301FB13030846002BF7D108467047DA
:10AA40000146FBE7F0EEC07AB0EEE07AB4EEE77ACA
:10AA5000F1EE10FAB4BFB0EE676AB0EE476AB5EE39
:10AA6000406AF1EE10FA46D0B4EEE77AF1EE10FA51
:10AA70008CBFF0EE675AF0EE475AC5EE866A9FED3E
:10AA80001F3A9FED1F6A9FED1F4A9FED1F5ADFED92
:10AA90001F3ADFED1F4ADFED1F5AA6EEC36AE6EE4E
:10AAA000A34AA6EE864AB7EE006AA6EE845AA6EE40
:10AAB000A46AE6EE855AC5EE866AB4EEE77AF1EE50
:10AAC00010FA48BFDFED147AF5EEC00A48BF77EE02
:10AAD000E66AF1EE10FA48BFDFED107AB5EEC00A73
:10AAE00048BF77EEE66AF1EE10FA48BFF1EE666A0B
:10AAF000B0EE660A7047DFED076ADEE739094E3DC2
:10AB0000E3B59E3E88FA163E45FE7F3F99FB243F03
:10AB100069A2163EA7DFA834DB0FC93FDB0F49400F
:10AB2000DFED317A30EE277AFDEEC76A16EE903A05
:10AB30002033402B02D99FED2D0A7047B4EEE70A6F
:10AB4000F1EE10FA4DDD9FED2A6ADFED2A6A01E091
:10AB5000B0EE677AB4EEE67AF1EE10FA77EE467A66
:10AB6000F6DC9FED257AF4EEC77AF1EE10FA35D5D2
:10AB7000DFED1F6A9FED217A01E0F0EE407AF4EEFE
:10AB8000C77AF1EE10FA37EEA60AF6D4DFED167AA0
:10AB9000B4EEE70AF1EE10FA1BDCDFED197AB4EE41
:10ABA000E70AF1EE10FA44BFDFED137A37EEC00A80
:10ABB00060EE006A9FED136A9FED137ADFED137A62
:10ABC000A6EE867A20EE266AE6EE877AA6EE270AB9
:10ABD0007047DFED0F7A37EEC00AE9E7B0EE670A9B
:10ABE000D4E7F0EE477ABCE7DB0FC93F0000000076
:10ABF000DB0FC940E4CB1641DB0F49C0E4CB16C1E3
:10AC0000DB0FC9BF92E741B99730083C15A82ABEAF
:10AC1000DB0F4940FDEEC07A17EE903A2033402B0F
:10AC200051D8DFED2D7AB4EEE70AF1EE10FA50DDDF
:10AC3000DFED2A6A9FED2A7A01E0B0EE670AB4EEF2
:10AC4000C70AF1EE10FA70EE667AF6DC9FED257A0F
:10AC5000F4EEC77AF1EE10FA38D5DFED206A9FEDF9
:10AC6000227A01E0F0EE407AF4EEC77AF1EE10FAC3
:10AC700037EEA60AF6D4DFED1D7AB4EEE70AF1EE60
:10AC800010FA1BDCDFED1A7AB4EEE70AF1EE10FAE7
:10AC900044BFDFED147A37EEC00A60EE006A9FED24
:10ACA000156A9FED157ADFED157AA6EE867A20EE0D
:10ACB000266AE6EE877AA6EE270A7047DFED067A67
:10ACC00037EEC00AE9E79FED0E0A7047B0EE670A5B
:10ACD000D1E7F0EE407AB9E7DB0F4940DB0FC9401E
:10ACE000E4CB1641DB0F49C0E4CB16C1DB0FC93FF3
:10ACF000DB0FC9BF92E741B99730083C15A82ABEBF
:10AD00000000000010B507EE901A2DED028BB8EE92
:10AD1000678ADFED217A28EE008A044628EE278A2A
:10AD2000B0EE480A34F00EFAF0EE408AB0EE480A6F
:10AD300034F06AF9F7EE007A9FED187AF0EE675A70
:10AD4000E8EE875A0023A361B0EE676AC7EEA56AF2
:10AD500063612362E361A8EEC76ABDEC028B77EE04
:10AD6000C07AB6EE007AF8EE005A27EE877A20EE27
:10AD7000250A27EE267A26EE266A67EEA67A20EEC8
:10AD8000260A84ED046AC4ED017A84ED007A84ED2C
:10AD9000027A84ED030A10BD27D4D236F304353F7E
:10ADA00010B44C09012250F8243001F01F0102FABE
:10ADB00001F10B4340F824305DF8044B704700BFAD
:10ADC0004B0901F01F0150F82320012303FA01F180
:10ADD000114214BF18460020704700BF38B5392013
:10ADE000FEF70CFB044618B1272201238271C371C0
:10ADF000204631F051FC002019F0DEFD18B100882A
:10AE000010F020000DD10021144D2B78052B08BF28
:10AE100081F001012046FEF7D7FD2B78032B09D0E6
:10AE200038BD0F4B5B79002BEDD10E4B1968C1F388
:10AE30008021E9E72720FEF7E1FA044631F02CFCF7
:10AE40002046FEF7BBFD1F20FEF7D8FA044631F07E
:10AE500023FC2046BDE83840FEF7B0BDE5380020B1
:10AE6000A84300209C6300200F4B1B785A1E012A28
:10AE700009D9042B00D070470C490D4B0020142237
:10AE800088705A70704730B40A490B4D0B4C03223E
:10AE90002720012B2A70A270087002D1034B0022D8
:10AEA0009A7030BC704700BFE53800200A8C002043
:10AEB0006CA000200039002078630020AC890020BD
:10AEC00038B52C20FEF79AFA044618B11122012356
:10AED0008271C37120462021FEF722FC31F08EFBE7
:10AEE0002046FEF793FDC8B91B4D03232D202B7080
:10AEF000FEF784FA044618B1112202238271C3714D
:10AF000020462021FEF70CFC2046FEF77FFDC8B14D
:10AF10002B7813B902232B7038BD38BD2D20FEF7D6
:10AF20006DFA0546A8B1112202238271C37131F076
:10AF3000B3FB2B68AA885A832046FEF767FD20B131
:10AF4000054DE5E705232B7038BD034B04221A702D
:10AF500038BD31F0A1FBEFE7E5380020074A084B88
:10AF600010781B78074A834296BFC31AC3F1800347
:10AF70000020126818441044704700BF049F00204E
:10AF8000809E00207C9E0020064A074B10781B788C
:10AF900083428ABFC3F18003C01AC018C0F17F008A
:10AFA000704700BF049F0020809E002030B543788A
:10AFB0004E4C013B5BB2022293422274DBBF1B0169
:10AFC0004B4A0023D3586361007804F1100183B029
:10AFD000E16008B903B030BDFEF710FAA06118B106
:10AFE0001A2200238271C3710921FEF799FBA0691F
:10AFF000FEF7E4FC00BF04216069FEF77FFE002538
:10B000009F2332208DF800308DF801508DF80250CA
:10B010008DF8035003F062FE8DF8055000BFE5681F
:10B02000A868FEF7C5FC01AA694604236868FEF714
:10B03000AFFEA868FEF7C2FC00BF9DF806309DF881
:10B0400005009DF807102B4A1B0243EA00430B43FF
:10B05000934244D00FDD284A934238D026DD274A58
:10B0600093422DD00132934223D1254B4FF480726D
:10B070001A809A8110E0234A934221D001329342F0
:10B08000F3D0A2F51A42033A934212D11C4B20216D
:10B090004FF4807219809A815A881988120202FB33
:10B0A00001F101205A609960207793E7023A9342B8
:10B0B00006D0134B0020188098815860986089E76B
:10B0C0000F4B80214FF4807219809A81E4E70C4B7A
:10B0D0004FF400714FF4807219809A81DCE7084BBD
:10B0E00040214FF4807219809A81D5E79C1F00207F
:10B0F00094B400201620C2001920C2001740EF00AF
:10B10000C005002017BA200030B5134C237F83B050
:10B110001BB90120237703B030BD052200238DF831
:10B1200000208DF8013000BFE568A868FEF740FCFC
:10B1300001AA694602236868FEF72AFEA868FEF79E
:10B140003DFC00BF9DF8053003F0010383F00100D2
:10B15000237703B030BD00BF9C1F002070B5064CA4
:10B160000646256803E023685B1BB34203D8FFF75C
:10B17000CBFF0028F7D070BD8CB400202DE9F04F34
:10B1800089B0B2F1000A02900491039340F3AB80BE
:10B190000B46002201EB8A0153F8040B8B42024458
:10B1A000FAD1039B0592002B00F09580059B002BA4
:10B1B00067D0514B059A1B6800920099DAB251187A
:10B1C000B1F5807F8CBFC2F58072009A01924B4A24
:10B1D00092689A426AD9190C1A0A4FF002040620A2
:10B1E0008DF81F308DF81E208DF81D108DF81C4035
:10B1F000FFF7B4FF0620FEF76FFD414A01231377E6
:10B2000000BFD2F80C90D9F80800FEF7D1FBD9F8AE
:10B21000040007A904230022FEF7BAFD0024049DC0
:10B22000029E019FA34629684FEA840800220B462C
:10B23000013469B1B94228D23168D9F80400FEF767
:10B24000A7FD2A68336813443360BF1AC5F800B0FD
:10B25000A24505F1040506F10406E4D1D9F8080079
:10B26000FEF7ACFB00BF244B019900981B68421A03
:10B270000092214A0B441360039A22B3009A002AD9
:10B280009BD1059809B0BDE8F08F029CD9F8040065
:10B2900054F808103B46FEF77BFD54F808202B6855
:10B2A0003A44DF1B44F808202F60D7E70598009C3C
:10B2B0001449154A001B0590059800230B70137064
:10B2C00009B0BDE8F08F059B009A9B1A059305987D
:10B2D00009B0BDE8F08FFFF717FF00287FF466AFD5
:10B2E000039B0593CDE7039C1CB9FFF70DFF059465
:10B2F000C7E700230593C4E77C9E0020C00500201B
:10B300009C1F0020049F0020809E002070B5104DDF
:10B31000104E2B7831788B4284B016D00E4A0392AF
:10B320001A4402928CBF0C46CA1A04A98CBFC3F1FE
:10B3300080020024012341F8102D02A8022201946A
:10B34000FFF71CFF002333702B7004B070BD00BFEB
:10B35000809E0020049F0020849E002070B5194C20
:10B36000194D23782978994284B027D0174A03923F
:10B370001A44029234BF0E46CA1A04A934BFC3F15C
:10B3800080020026002341F8102D02A80222019617
:10B39000FFF7F4FE23781844C0B203062B7848BFA9
:10B3A00080F080008342207002D0002004B070BD85
:10B3B000002301202B70237004B070BD012004B065
:10B3C00070BD00BF809E0020049F0020849E00204E
:10B3D00008B545F20820FFF7C1FE0620FEF77CFC09
:10B3E000064B0122C7201A77FEF776FC0448054970
:10B3F000054A002303700B70136008BD9C1F0020DA
:10B40000049F0020809E00207C9E00202DE9F041BA
:10B4100082B00346060C050A032406208DF8073087
:10B42000884617468DF805608DF806508DF8044063
:10B43000FFF794FEB0B100BF0C4BDC68A068FEF7CC
:10B44000B7FA01A9606804230022FEF7A1FC3B467D
:10B45000424600216068FEF79BFCA068FEF7AEFA4A
:10B4600000BF384602B0BDE8F08100BF9C1F00203D
:10B47000F0B5124B9D6885B00DB905B0F0BDED0A71
:10B4800014D0002704AE7C196410E0021022694633
:10B49000FFF7BCFF0F2809DD6B4653F8042B013280
:10B4A0000AD1B342F9D12546AF42ECDBFFF72EFFBC
:10B4B000034BED021D60E0E7671CF5E7C0050020C7
:10B4C0007C9E00200C4B984213D0A3F580639842D9
:10B4D0000FD003F5804398420BD003F58063984268
:10B4E00007D003F58063984203D0044B18684008E6
:10B4F0007047024B1868704700040140F8A900200B
:10B50000F0B5774B774A87B01968914200AF00F0E9
:10B51000DB800023744A3B607B60136843F4803314
:10B52000136003E03B68B3F5A04F09D0136803F440
:10B5300000337B603B6801333B607B68002BF1D0BC
:10B54000694B1B6813F4003318BF01237B607B68D1
:10B55000012B7BD0654D644B654AEA606549586FA5
:10B56000654A0860AA605E6B644C654A654826F0CF
:10B5700080065E635E6F46F080765E67196B0C43F3
:10B580001C63596B5963996B9963196C41F05B515A
:10B5900041F47B1141F41F6141F00F011964596CB2
:10B5A00007F118040A4348F2FF715A6444F8101D69
:10B5B000002621460123FB733E737E73BE7325F084
:10B5C0003BFA21464FF6FF734F48BB6025F034FA33
:10B5D0004FF6FF7321464D48BB6025F02DFA2146FA
:10B5E0004B4825F029FA21464A4825F025FA2146FC
:10B5F000494825F021FA2146484825F01DFA214600
:10B60000474825F019FA2146464825F015FA204604
:10B6100025F004FC444B454C1B68BA684448454936
:10B62000A4FB03439B09A0FB0202013B920CB3F174
:10B63000807F0A6007D2404AF0200721536085F8D6
:10B640002300966011601C37BD46F0BD264B3B4D74
:10B650001A6C3B4842F080521A642C684268816838
:10B6600044F440442C609C689C609C6844F4004412
:10B670009C609C6844F4A0549C600068120642EAF6
:10B68000801242F48002490842F00802013942EA7D
:10B6900001425A601A6842F080721A601A68920178
:10B6A000FCD52849104A40F205700860996821F0DD
:10B6B00003019960996841F002019960936803F071
:10B6C0000C03082BFAD145E700221A6062B61E4B24
:10B6D0001B6883F308881D4B1B689847FEE700BF73
:10B6E000FCFF0120EFBEADDE0038024000ED00E0BF
:10B6F0000005FA054065002000000008FF91670082
:10B70000335F0700000002400004024000080240CE
:10B71000000C0240001002400014024000180240D9
:10B72000001C024000200240F8A90020D34D621006
:10B7300083DE1B4390B4002010E000E00070004066
:10B7400000000020003C02400000FF1F0400FF1F1B
:10B7500008B5054B1B6803B19847044B044A1A60AF
:10B7600072B6FDF75FF800BFA0820020FCFF012049
:10B77000EFBEADDE08B5034B1B6803B1984772B648
:10B78000FDF750F8A0820020084B10B507281B6871
:10B79000C8BF143818440C46007EFDF72FFE20B1B8
:10B7A0002146BDE81040FEF70FB910BD7CA0002077
:10B7B00030B50446406D61718389A26823F400535B
:10B7C0001B041B0C838185B0A379009213F0040243
:10B7D00030D04FF4805213F00203ADF804205CD156
:10B7E000ADF806304FF480630022ADF8083011F058
:10B7F0000103ADF80C2028D1ADF80A3008238D07DD
:10B80000694648BFADF80A3025F09EFBA279636D0A
:10B81000D10724D412F0080F9A8A1BD122F0080213
:10B820001204120C9A829A8992B242F400529A81BE
:10B8300005B030BD13F00203ADF804202AD04FF458
:10B8400000551346ADF80650CEE70423ADF80A3094
:10B850000C23D4E792B242F008029A82E3E710493F
:10B860008B4215D0A1F548418B420FD001F5806184
:10B870008B4209D00B498B42CCD105200121FFF727
:10B8800083FFA279636DC5E70320F7E70220F5E7A0
:10B890000020F3E7ADF80630A6E74FF400539FE72A
:10B8A000001001400014014010B50446406DA16035
:10B8B000838923F400531B041B0C8381A37984B078
:10B8C00013F00402009135D04FF4805213F00203BC
:10B8D000ADF804205CD1ADF806304FF48063627996
:10B8E000ADF80830D1074FF00003ADF80A30ADF8DD
:10B8F0000C3045BF0423ADF80A3008230C236946F9
:10B90000920748BFADF80A3025F01EFBA279636D9F
:10B91000D1071FD412F0080F9A8A16D122F008021C
:10B920001204120C9A829A8992B242F400529A81BD
:10B9300004B010BD13F00203ADF8042025D04FF47D
:10B9400000511346ADF80610C9E792B242F0080262
:10B950009A82E8E710498B4215D0A1F548418B4205
:10B960000FD001F580618B4209D00C498B42D1D1B7
:10B9700005200121FFF708FFA279636DCAE70320C4
:10B98000F7E70220F5E70020F3E7ADF80630A6E779
:10B990004FF400539FE700BF001001400014014026
:10B9A00038B50C4B07281B68CCBFA0F11404044623
:10B9B00023440546187EFDF721FD50B101342722AE
:10B9C000C471827130F068FE28460021BDE838401D
:10B9D000DAE638BD7CA00020064A00235168814287
:10B9E00002F11C0204D00133102BF7D10020704764
:10B9F000D8B27047E800002070B50F4C0F4DC0EB77
:10BA0000C00004EB8004286B26693043286382B0B1
:10BA10009209667BA1600025012101A863618DF870
:10BA200004608DF805208DF806508DF8071025F07C
:10BA300053FA02B070BD00BFE80000200038024099
:10BA4000074BC0EBC00030B403EB8000054C056928
:10BA5000236B2B4323630176427630BC704700BFD3
:10BA6000E8000020003802402DE9F04F534C54F814
:10BA7000204083B0002C00F09C80E56D002D00F08C
:10BA80009A8017464E4A9846064604F16203286992
:10BA9000226004F262226361A2614FF400736A685B
:10BAA000A160E36023616265A24668B1FFF794FF7D
:10BAB000721CD2B20C21FFF7C3FF636DA9682A691B
:10BAC00022630433A1632365E868A0B1FFF784FF14
:10BAD000721C8146D2B20B21FFF7B2FF2346EA7FE8
:10BAE00038494846FFF788FF636DA968EA686263D2
:10BAF0000433E163E36494F86100FDF77FFC814661
:10BB000094F86000FDF77AFC8346287F00284DD129
:10BB100018F0080F36D1BA070DD5B9F1000F0AD0C9
:10BB20000B22731C89F8062089F8073048466A7F83
:10BB30002221FDF729FDFB0715D4A36B7BB995F8EE
:10BB40002020A97F8DF8063001A8930901228DF8E5
:10BB500005308DF804108DF8072025F0BDF950460A
:10BB600003B0BDE8F08FBBF1000FE6D001360C2327
:10BB70008BF807608BF8063058466A7F2221FDF764
:10BB800003FDDAE70136F6B2B9F1000F04D00B235A
:10BB900089F8076089F8063018F0100F484614BF7E
:10BBA000022112216A7FFDF7EFFCC6E730F008FDA5
:10BBB000AEE7A246D3E7AA46D1E700BFE8380020A7
:10BBC00068140408498800080348D0F8AC3113B160
:10BBD00000F5D27018477047E80000200348D0F8FD
:10BBE000903113B100F5C47018477047E800002089
:10BBF0000348D0F8743113B100F5B6701847704798
:10BC0000E80000200348D0F8583113B100F5A870BF
:10BC100018477047E80000200348D0F83C3113B1C2
:10BC200000F59A7018477047E80000200348D0F8E4
:10BC3000203113B100F58C7018477047E8000020E0
:10BC40000348D0F804310BB1FC301847704700BFEF
:10BC5000E80000200348D0F8E8300BB1E030184786
:10BC6000704700BFE80000200348D0F8CC300BB18B
:10BC7000C4301847704700BFE80000200348D0F8E0
:10BC8000B0300BB1A8301847704700BFE800002063
:10BC90000348D0F894300BB18C301847704700BF80
:10BCA000E80000200248836F0BB1703018477047DE
:10BCB000E80000200248C36D0BB1543018477047AC
:10BCC000E80000200248036C0BB138301847704779
:10BCD000E80000200248436A0BB11C301847704747
:10BCE000E80000200248836803B11847704700BF8E
:10BCF000E8000020431C00F00E812DE9F04F4FEAD0
:10BD0000C00808EB00039B00DFF8E8A25AF803B074
:10BD100087B00AEB0304BBF1000F00F0F980143385
:10BD20000AEB03010022DBF804704AF803204A60A2
:10BD30008A60CA600346A56801900133D4F80C906C
:10BD4000DBB2002D00F0E8801522EB71AA71B9F189
:10BD5000000F00F0FA80162289F8062089F80730D3
:10BD60009BF80E0030F02CFCBB8823F440731B04BE
:10BD70001B0CBB802846FDF721FE4846FDF71EFE42
:10BD800011212846FDF784FA11214846FDF780FA73
:10BD90000826642403E03CB130F030FC013C284626
:10BDA000FDF734FE0028F6D02846FDF701FE30F0FE
:10BDB00025FC2846FDF702FE30F020FC013EEED1C6
:10BDC0004846FDF7F5FD30F019FC2846FDF7F0FD7B
:10BDD00030F014FC2846FDF7F1FD30F00FFC48462A
:10BDE000FDF7ECFD019B08EB03040AEB84042846F5
:10BDF000637C002B0CBF122132210422FDF7C4FB0F
:10BE0000637C002B0CBF1221322148460422FDF72F
:10BE1000BBFB704B9F4200F0B7806F4B9F4200F01E
:10BE2000BD806E4B9F4200F0A580BB8801996C4A93
:10BE30006C4C23F440731B041B0CBB803B88884470
:10BE40000AEB880A9BB243F001039AF810103B807A
:10BE5000BD8802A8002918BF144624F0DFFF049A09
:10BE60006148B2FBF4F325F03F05A0FB02122D045C
:10BE7000900C2D0C0543BD805C4C39884FF49672B4
:10BE800002FB00F284FB02409BB2D217002BC2EBF4
:10BE9000A01221F0010108BF01230904013243F47B
:10BEA0000043090C92B239803A84BB833B889BB231
:10BEB00043F001033B803B8823F4816323F00203BA
:10BEC0001B041B0C43F480634FF480423B803A8197
:10BED0003B8823F080031B041B0C3B809BF8103035
:10BEE0008DF808300024012302A88DF80B308DF85E
:10BEF00009408DF80A4024F0EFFF9BF80F308DF8D1
:10BF0000083002A88DF809408DF80A4025F00AF89B
:10BF100007B0BDE8F08F7047B9F1000F48D0162286
:10BF200089F8073089F806209BF80E0030F048FBAE
:10BF3000BB8823F440731B041B0C2846BB80FDF711
:10BF40003DFD4846FDF73AFD1EE79BF80E0030F038
:10BF500037FBBB8823F440731B041B0CBB802846B3
:10BF6000FDF72CFD4846FDF729FD11212846FDF778
:10BF70008FF90DE71E4A136A43F4000313624FF46E
:10BF8000000024F095FE50E7194A136A43F40013A9
:10BF900013624FF4001024F08BFE46E7144A136A34
:10BFA00043F4800313624FF4800024F081FE3CE7E9
:10BFB0009BF80E0030F004FBBB8823F440731B0495
:10BFC0001B0C4846BB80FDF7F9FC4846FDF7F6FC24
:10BFD000DEE600BF0054004000580040005C004016
:10BFE000009F2400804F120083DE1B43D34D62105C
:10BFF0000038024010390020F8B54FEAC00E274F34
:10C00000069C0EEB000507EB85056E68002E42D0FE
:10C010004900C9B2A9754FF0000C0121EA7585F8F5
:10C0200019C0A9762B76697585F814C0B3882C627F
:10C030009905EC6114D43388DA050CD44FF480549C
:10C0400001E0013C1ED033889B05FAD433889BB2B3
:10C0500043F480733380B3889BB243F44073B3805E
:10C060000EEB000107EB81024FF4805401E0013C2C
:10C0700008D0537D002BFAD107EB81073C7D84F07B
:10C080000100F8BD064A138801339BB21380FFF705
:10C0900031FE2046F8BD3046F8BD00BF1039002003
:10C0A000183B002070B590F904506C1C82B00AD087
:10C0B000032D08DC16460A46417900962846FFF70C
:10C0C0009BFF02B070BD002002B070BD00B50378C8
:10C0D000012B83B004D1032301AA0021FFF7E2FF63
:10C0E0009DF805309DF804209DF806001B0243EAE8
:10C0F0000243184303B05DF804FB00BF08B5FFF727
:10C10000E5FF014B586008BD9C1F002008B5FFF7F4
:10C11000DDFF014B186008BD9C1F0020F0B585B005
:10C1200002AB04460093032206231E210020FFF7E2
:10C1300063FF00283CD09DF808509DF809109DF839
:10C140000A709DF80B209DF80C609DF80D3041EAB7
:10C15000052142EA072243EA062309B212B21BB2C2
:10C16000144D06EE901A07EE102A07EE903AF8EEFC
:10C17000E66A95ED035AD5ED055A95ED046AB8EED9
:10C18000C77AF8EEE77A66EE856A27EE257A67EEDB
:10C19000867AFDEEE66ABDEEC77AFDEEE77A16EE28
:10C1A000901A17EE102A17EE903A2180A280638031
:10C1B00005B0F0BD0000002000B583B00020009263
:10C1C0000A466821FFF718FF03B05DF804FB00BFC3
:10C1D000F0B5C60033189B00254DEA585468A28A72
:10C1E00083B092B20192019A2B4412F4706F1CBF7B
:10C1F00001221A75019B13F4E06F07460CD1A38A44
:10C200003E4423F4706305EB86051B041B0C0022DF
:10C21000A3826A7503B0F0BD238BA38823F48063E7
:10C220001B041B0CA380019B9B05E8D42388980565
:10C23000E5D42388D9050ED52388DA05FCD42388D4
:10C240009BB243F40073238023889B05FCD43846BB
:10C25000FFF750FDD3E723889BB243F4007323809C
:10C26000A38823F440731B041B0CA380C7E700BF03
:10C2700010390020F0B583B0441C8DF8073001D090
:10C28000032802DD002003B0F0BDC700244E3B1898
:10C2900006EB83035D68002DF4D04900C9B299759F
:10C2A00001240021DA755C7699761C765C75197527
:10C2B000A9880DF107028905DA611A6214D42B8866
:10C2C000DA050CD44FF4805401E0013C1ED02B88D9
:10C2D0009B05FAD42B889BB243F480732B80AB88E8
:10C2E0009BB243F44073AB80074406EB87024FF4E4
:10C2F000805401E0013C09D0537D002BFAD106EBBC
:10C3000087073C7D84F0010003B0F0BD054A138827
:10C3100001339BB21380FFF7EDFC2046B3E700BF6B
:10C3200010390020183B00202DE9F043322083B063
:10C3300002F0D4FC0022104611231E21FFF79AFFC1
:10C34000602301221E210020FFF794FF642002F0E9
:10C35000C5FC6846FFF7E2FE0024DFF8548125465D
:10C3600026460A27012302221E210020FFF782FF12
:10C37000322002F0B3FC6846FFF7D0FEBDF902E0C0
:10C38000BDF90410BDF900208E457346A8BF0B46C9
:10C390009342A8BF134643454FF0010075440C4437
:10C3A000164479DBFCF798FE013FDBD14FF0010921
:10C3B0000022104612231E21FFF75CFFDFF8F080F9
:10C3C0000A27012302221E210020FFF753FF3220FB
:10C3D00002F084FC6846FFF7A1FEBDF902E0BDF95A
:10C3E0000410BDF900208E457346A8BF0B4693424A
:10C3F000A8BF134643454FF00100A5EB0E05A4EB83
:10C400000104A6EB02064ADBFCF766FE013FD8D129
:10C4100007EE906AF8EEE76A07EE905AB8EEE77A10
:10C4200007EE904ADFED1F5A9FED1F5A1F4EF8EEA0
:10C43000E77A85EEA66A0022104670231E21C5EE1B
:10C44000876A85EE277AB0EEC66AF0EEE66AF0EE0D
:10C45000C77A86ED036AC6ED046AC6ED057AFFF772
:10C4600009FF202301221E210020FFF703FF0023E4
:10C47000184602221E21FFF7FDFE642002F02EFC6A
:10C48000B9F1000F04D14FF07E53F3603361736153
:10C49000012003B0BDE8F0834FF0000988E74FF0BA
:10C4A0000009B5E700406F4601C05E46000000206D
:10C4B00001F0FFFF0378012B00D07047417990F91C
:10C4C00004005822D6E600BF0378012B00D0704745
:10C4D000417990F904004822CCE600BF13460020C1
:10C4E0000A466821C6E600BF0220FCF789BA00BFF1
:10C4F00002206DE60120FCF783BA00BF012067E649
:10C500000020FCF77DBA00BF002061E61549164BFC
:10C5100016480A6810B48C681549B2FBF4F203FBA4
:10C5200002F30360D1F88820124B134C42F47002DE
:10C53000C1F888201A68002042F001021A60986051
:10C540001A6822F0847222F480321A605C601A68E1
:10C550004FF0006422F480221A60D8608C605DF88D
:10C56000044B70470000002040420F00F8A9002053
:10C5700000ED00E00038024010300024044B4FF47E
:10C58000F0700A21022283E80700FFF7BFBF00BF57
:10C590000000002038B50B4C23688BB15A68821A12
:10C5A000002A054604DA0CE05A68AA1A002A07DBBA
:10C5B0009A68226018461A6890472368002BF3D1C6
:10C5C00038BD38BDD08500200B4B002210B402725C
:10C5D00003F1A804012102E0072A09DC99798907FF
:10C5E00002D51979815401329C4203F11803F3D129
:10C5F0005DF8044B704700BF004404083723037004
:10C60000704700BF01233321322241704271037011
:10C61000037170472722032302704370704700BFE5
:10C6200008B516F019FBFFF7A5F800BF024A034B47
:10C63000127819782CF022B8982200209922002034
:10C64000038A2DE9F0478589ADB21D4029D00F46F8
:10C6500006464FF000484FF00009B5FA85F328FA76
:10C6600003F2D24391B21B3B15403182042B16D802
:10C67000DFE803F03129211903007B6A002B32D057
:10C6800003F1FF3A1FFA8AFAC7F824903C6A34B1E2
:10C6900023682046514698476468002CF8D1002D45
:10C6A000DBD1BDE8F0873868716B036889B29847C1
:10C6B000002DD2D1F5E77868B16B036889B298474D
:10C6C000002DCAD1EDE7B868F16B036889B29847CD
:10C6D000002DC2D1E5E7F868316C036889B298474C
:10C6E000002DBAD1DDE7F36A1FFA83FACEE700BF67
:10C6F0002DE9F04F2DED028BA0F10A0389B00C4615
:10C70000E72B00F24E87DFE813F01C014C074C07C3
:10C710004C074C074C074C074C074C074C074C0781
:10C720004C074C074C074C074C074C074C074C0771
:10C730004C074C074C074C074C0780014C074C0733
:10C740004C0771014C074C074C0764014C078102F0
:10C750004C0769024C0739024C0731024C070C02A6
:10C760004C07E0014C074C074C07DA01D3014C079A
:10C77000C7054C074C07BF054C0796054C074C07EF
:10C780004C0779054C074C074C074C07F6024C0741
:10C79000FC004C07F305CF054C074C074C074C0732
:10C7A0004C074C074C07B2064C0783064C0717078B
:10C7B0004C0719064C076E064C074C074C074C07F4
:10C7C0002805ED04E604C502E800AB049704CF0495
:10C7D0008B044C07540438044C074C074C074C0797
:10C7E0002D044C074C070C044C074C074C07FE0368
:10C7F000E703AC036A034C074C074C075B03440395
:10C80000350315034C074C074C074C074C074C07E6
:10C810004C074C074C074C074C074C074C074C0780
:10C820004C0728054C074C074C074C074C074C0796
:10C830004C074C074C074C074C074C074C072D0185
:10C840004C074C074C074C074C074C074C074C0750
:10C850004C074C074C074C074C074C074C074C0740
:10C860004C074C074C074C074C074C074C074C0730
:10C870004C074C074C074C074C074C074C074C0720
:10C880004C074C074C074C074C074C074C074C0710
:10C890004C074C074C074C074C074C074C074C0700
:10C8A0004C074C074C074C074C074C074C074C07F0
:10C8B0004C074C074C074C074C074C074C074C07E0
:10C8C0004C074C074C074C074C074C074C074C07D0
:10C8D0004C074C074C079E01A901AE4E337853B16B
:10C8E000AD4F002537F8021F2046FDF713FF3378C0
:10C8F0000135AB42F6DC012009B0BDEC028BBDE88E
:10C90000F08FA44E3378002BF5D0A44F0025B84605
:10C91000236817F81520591C21601A7098F8011027
:10C9200001EB810101EB810101F2EE2189B2204688
:10C93000FDF7F0FE33780135AB4208F10208E7DC81
:10C94000D9E7974D284631F099FC0028D3DD2B46D6
:10C950000544226813F8011B501C9D422060117091
:10C96000F7D1C8E70B68DFF870C2591C9CF80020AB
:10C9700021601A709CF80030002BBCD0894E8A4D83
:10C980008A488B490023226816F8017F02F1010EC4
:10C99000C4F800E01770226815F8017F02F1010E5B
:10C9A000C4F800E01770226810F8017F02F1010E50
:10C9B000C4F800E01770226811F8017F02F1010E3F
:10C9C000C4F800E017709CF8002001339A42DADCCA
:10C9D00091E70B68774A581C11782060197023681A
:10C9E0005278591C216001201A7085E7724D084663
:10C9F0002988FDF78FFEA9882046FDF78BFE20468B
:10CA00002989FDF787FE012076E76C4D05F1500678
:10CA1000287831F039F82368027A591C21601A709D
:10CA200023686A78591C21601A702368AA78591CF7
:10CA300021601A702368EA780435591CAE422160DF
:10CA40001A70E5D157E75E4D0846E989FDF762FEA9
:10CA50002046A989FDF75EFE01204DE7594B03F101
:10CA6000700522681978501C20601170226859786E
:10CA7000501C2060117022689978501C2060117041
:10CA80002268D978501C2060117022681979501CD6
:10CA90002060117022685979501C20601170226842
:10CAA00099790733501C9D4220601170D9D122E73B
:10CAB0000B6801229918216010461A701CE708467D
:10CAC0000021FDF70FFE012016E73F4D05F1380765
:10CAD00003E00835AF423FF40EAF95F902603046EF
:10CAE00016F0B6FE0028F4D023685A1C22601E708F
:10CAF00029882046FDF70EFE2368EA78591C21603C
:10CB00001A7023682A79591C21601A702368AA793F
:10CB1000591C21601A7023686A79591C21601A70A7
:10CB2000D7E72A4B03F15A0522685979501C206037
:10CB3000117022681978501C206011702268597891
:10CB4000501C2060117022689978501C2060117070
:10CB50002268D978501C2060117022681979063338
:10CB6000501C9D4220601170DED1C4E60B68184A4B
:10CB7000591C527D216001201A70BDE6154D05F14A
:10CB8000800655F8041F2046FDF7ACFDAE42F8D1F3
:10CB9000B1E600BFBC9F0020DA5E00203CAC002064
:10CBA00088890020EF470020FF4700201F48002011
:10CBB0000F480020D489002088390020D88900201F
:10CBC000AC89002090AD002064A70020B83B002075
:10CBD00014650020149A0020ED470020AB4D05F1AC
:10CBE0004006B5F880102046FDF794FD236895F8BF
:10CBF0008220591C21601A70236895F8832004351F
:10CC0000591CB54221601A70EBD174E6A04D0B6837
:10CC10002A7A591C21601A70A98B2046FDF77AFDEB
:10CC2000298B2046FDF776FD698B2046FDF772FDC6
:10CC30002368EA7C591C21601A70A98C2046FDF7F4
:10CC400069FDE98C2046FDF765FD2368AA7F591C24
:10CC500021601A70236895F82020591C21601A70F1
:10CC6000698C2046FDF756FD2368EA7A591C21603D
:10CC70001A70E9682046FDF735FD23682A7C591CA7
:10CC800021601A70236895F82120591C2160012029
:10CC90001A7031E67F4D804E9FED808ADFF830823A
:10CCA000DFED7F8A05F120070EE0FCEEE77ACDED9F
:10CCB000017ABDF8041020460435FDF72BFDAF4284
:10CCC00006F118063FF417AE717C0029F3D0754BBE
:10CCD000D5ED007A1B78012BE7D1734B1B68DB0481
:10CCE00040F10285F5EE407AF1EE10FA40F033851E
:10CCF00040F2DC51DFE70B686C4D591C2A7921604A
:10CD00001A7023686A79591C21601A702988204694
:10CD1000FDF700FD2368AA79591C21601A70698803
:10CD20002046FDF7F7FC2368EA79591C21600120B1
:10CD30001A70E1E50B685E4F591C3A7821601A7051
:10CD40003B78002B3FF4D7AD0025EEB2304618F00B
:10CD5000DDFD23684278591C216030461A7018F0B6
:10CD6000D5FD01892046FDF7D5FC3B780135AB4266
:10CD7000EBDCC0E54F4B5049B3F9003081FB032198
:10CD8000DB17C3EBA101204689B2FDF7C3FC0120EC
:10CD9000B2E50A68494B501C19782060117022686E
:10CDA0005978501C2060117022689978501C2060BE
:10CDB00011702268DB78511C2160012013709BE503
:10CDC0003F4D0846298AFDF7A5FC698A2046FDF7F4
:10CDD000A1FC2046A98AFDF79DFC01208CE5DFF827
:10CDE000F4E00027FEB2714600232268501C206048
:10CDF00016702268501C20601370226811F8010F11
:10CE00000133551C062B25601070EED10137062F1B
:10CE10000EF1060EE6D12B4900232268501C20603B
:10CE200017702268501C20601370226811F8010FDF
:10CE30000133551C0B2B25601070EED12368134A6B
:10CE4000581C07212060197023680021581C20609D
:10CE50001970236892F8F020591C216001201A7083
:10CE60004AE50B68184A19491078124A5D1C25607A
:10CE7000187023688978581C20601970236892788C
:10CE8000591C216001201A7036E500BF189A002055
:10CE900014650020AC870020885F0020000040421D
:10CEA00000E082446C6000209C630020AC3D0020C8
:10CEB00011430020BC89002067666666D4470020C5
:10CEC00048600020FB9A002078630020AC89002095
:10CED000DB9B9141D79A00200A68B14BB149187881
:10CEE000551C2560107022685878551C25601070FC
:10CEF00022689B78501C206013702046C988FDF77B
:10CF000009FC0120F8E4A74D08462988FDF702FC3A
:10CF100069882046FDF7FEFBA9882046FDF7FAFB4D
:10CF2000E9E4A14D05F16006A9882046FDF7F2FB72
:10CF3000E9882046FDF7EEFB29892046FDF7EAFB4C
:10CF40002368AA7A591C21601A702368EA7A591C4E
:10CF500021601A7055F80C1B2046FDF7C3FBAE424A
:10CF6000E2D1C8E4914952232268501C206013701A
:10CF700011F8013F002BF7D1BDE48D480023226852
:10CF8000056803EB4301561C6D5C26601570026852
:10CF900025680A446E1C527826602A70026825684B
:10CFA0000A4401339278691C0A2B21602A70E6D169
:10CFB000A1E4804D0B682A68591C127821601A7010
:10CFC0002B6822689978531C2360002311702A680B
:10CFD00021681A4401335279481C032B20600A70DF
:10CFE000F5D123682A68591C127A21601A702368C7
:10CFF0002A68591CD27821601A7023682A68591C43
:10D00000127921601A702B6820465989FDF782FB3E
:10D010002A682368527A591C21601A702A68DEE453
:10D02000654B08461968FDF75DFB644B204619887F
:10D03000FDF770FB01205FE4614B08461988FDF79E
:10D0400069FB604B20461988FDF764FB5E4B226844
:10D050001B78511C03F001032160012013704BE485
:10D060005A4B0A681B785A4D511C03F00203216089
:10D07000137023682A7D591C21601A702968204684
:10D08000FDF730FB69682046FDF72CFB2989204617
:10D09000FDF740FBE9892046FDF73CFB2046298A45
:10D0A000FDF738FB012027E44A4D08462988FDF7A3
:10D0B00031FB69882046FDF72DFBB5F90430464A5F
:10D0C000D91782FB0323C1EBA301204689B2FDF7E8
:10D0D00021FB012010E4084610224049FDF7D2FA56
:10D0E000012009E43E4B9B8AB3F5006F00F20583F3
:10D0F000B3F5806F00F22D83B3F5007F34BF0127B5
:10D100000227384D05F10C0655F8041B91FBF7F189
:10D11000204689B2FDF7FEFAAE42F5D1324D334FCB
:10D1200005F10C06B5EC010AD7ED087A80EE270A66
:10D1300031F0BCFF81B22046FDF7ECFAAE42F1D1EE
:10D140002B4D05F10C0655F8041B204689B2FDF75E
:10D15000E1FAAE42F7D1FFF7CEBB00258146DFF8FA
:10D160009480DFF894B00595049506950795012104
:10D170004FF6FF7A05E001350B2D00F0158218F906
:10D18000011F4F1C4AFA05F3F5D0DE07F3D5BBF8B3
:10D1900000302B41D807EED506A8FDF701FEEAE7DF
:10D1A000A4890020903D0020B8B30020901404080A
:10D1B000949F0020244A00202C4600202046002076
:10D1C0000447002006470020B846002050460020B3
:10D1D0005446002030460020676666669C87002023
:10D1E000D84500201046002090630020C4B40020E1
:10D1F000E0490020C01404084A9B0020FDF784FF8A
:10D200002368BC4D002803F101010CBF0222032258
:10D2100021601A7029882046FDF764FAA968204623
:10D22000FDF760FAFDF79AFE01462046FDF75AFA2F
:10D230000120FFF761BB0B68AF4AB04D1178B04ACF
:10D24000581C2060197011682046FDF74BFA2368BE
:10D25000AC4A591C127A21601A7029882046FDF7C1
:10D2600059FAA9882046FDF755FA29892046FDF785
:10D2700051FA00212046FDF74DFA20460021FDF726
:10D2800049FA0120FFF738BB084608229D49FDF7FF
:10D29000F9F90120FFF730BB0B689B4A581C9178C5
:10D2A00020601970FFF79BBB0B68984E01255A1C34
:10D2B0000A601D700B68B278591921601A7024F049
:10D2C0000DFD2368924A93495F1927601870B1F9E0
:10D2D0000010B2F90000FDF7A7FB23685A1922607D
:10D2E000187031882046FDF715FA2846FFF704BB71
:10D2F0000B68894D01269A190A601E7029F000FFFB
:10D30000002840F00882854B2268511C2160107073
:10D31000226841F2B410511C185C216041F278116E
:10D32000107059582046890AFDF7DCF9A96A204691
:10D330004908FDF7D7F90120FFF7DEBA00212046A2
:10D34000FDF7E8F900212046FDF7E4F90021204629
:10D35000FDF7E0F92368724D00265A1C22601E700A
:10D3600023682A68591C92F82C2021601A702368BF
:10D370002A68591C92F8362021601A7023682A689E
:10D38000591C92F8372021601A7023685A1C2260B9
:10D390001E7023685A1C22601E7023685A1C22606B
:10D3A0001E702B682046598FFDF7B4F92B68204674
:10D3B000198FFDF7AFF923682A68591C92F82E20BF
:10D3C00021601A7023685A1C22601E702B68204648
:10D3D000598EFDF79FF92B682046998EFDF79AF933
:10D3E0000120FFF789BA0B684E4A4F49D0784F4A5F
:10D3F0005D1C2560187023684979581C20601970DD
:10D400002368D278591C216001201A70FFF774BA82
:10D41000474EF378002B00F072810B680822591CEC
:10D4200021601A7023680122991821601A702368FC
:10D43000404D591C2A7921601A702368AA78591C1A
:10D4400021601A7029882046FDF764F9E989204691
:10D45000FDF760F92368F279591C21601A7023687E
:10D46000EA78591C216001201A70FFF745BA2BF0A9
:10D47000E9F8FF28064600F0558108A9002501F8C3
:10D48000125D0DF10D008DF80D502BF0BBF808A8C2
:10D4900000F8115D2BF0AAF808A800F8105D2BF039
:10D4A00099F808A820F8085D2BF088F823685A1C22
:10D4B00022601E7023689DF80D20591C21601A708F
:10D4C00023689DF80E20591C21601A7023689DF86E
:10D4D0000F20591C21601A7023689DF81020591CD8
:10D4E00021601A702046BDF81810FDF713F90120CD
:10D4F000FFF702BAC0050020D48900208839002037
:10D50000248C002014650020C88900200A8C00208B
:10D510000688002008880020305D0020B86D0020BB
:10D52000949F0020AC890020BC9D0020BC89002075
:10D530007863002048600020AD4E0B687279AD4DD5
:10D54000591C21601A702B682046198CFDF7E2F8EF
:10D550002B682046D98BFDF7DDF871892046FDF751
:10D56000D9F8B1892046FDF7D5F82B682046598CAB
:10D57000FDF7D0F82B682046998CFDF7CBF8F189A0
:10D580002046FDF7C7F8318A2046FDF7C3F82A6820
:10D59000236892F82620591C216001201A70FFF799
:10D5A000ABB90020FFF7A8B9DFF874A200254FF04F
:10D5B00008080135C5F1200208FA02F2A5F120039E
:10D5C0002AFA05F6164328FA03F31E43252D06F022
:10D5D00001024FF000030BD01343EAD0E8B21BF076
:10D5E0000BFF0028E5D0294606A8FDF7D9FBE0E7A8
:10D5F000814B1B78DA0700F19C8000257F4E2F4677
:10D6000002E00135252D0DD029463046FDF7D8FB27
:10D610000028F6D0294606A8FDF7D2FB00285ED1E7
:10D620000137EEE7764B774DB3F850102046FDF703
:10D6300071F8754B1988204689B2FDF76BF8734B6A
:10D6400019684B0103F02002C1F340031343C1F3F7
:10D65000800243EA4203C1F3C00243EA8203C1F3FA
:10D66000401243EAC20301F0100119432046FDF7BE
:10D6700051F804A904222046FDF704F8236829780C
:10D68000634A581C2060197011886429A8BF64215E
:10D690002046FDF73FF8B9F1960F4FD00021204604
:10D6A000FDF738F82168B7F1190348BFA7F1120355
:10D6B000A3F3C4034A1C226020461A460B7005A936
:10D6C000FCF7E0FF2368534A581C102120601970B2
:10D6D00020461188FDF706F80120FFF70DB93946FD
:10D6E00004A8FDF75DFB9BE7F4EEC87AF1EE10FAB3
:10D6F00056DA4FF47A71FFF7DEBA082701E50B68B6
:10D70000B178454A581C2060197023681278591C5A
:10D7100021601A708BE695F82420404B002A37D1FF
:10D720003046F1E523685A1C226001201E70FFF785
:10D73000E3B8069B43F0010306935EE723680322E8
:10D74000591C21601A7023686A78591C21601A706C
:10D75000A8E70427D5E4F4EEC87AF1EE10FA3FF515
:10D76000C7AAF4EEE87AFDEEE77AF1EE10FA17EECA
:10D77000901A2DD86FF4F973303903FB01F140F2A0
:10D78000E73391FBF3F101F2DB5189B2FFF793BA72
:10D790005978022917D003290CBF04203046B3E57D
:10D7A000FDEEE77A40F2E73217EE903A303B02FBAB
:10D7B00003F388FB0312D917C1EB622101F2E931AF
:10D7C00089B2FFF778BA042A34BF022003209BE510
:10D7D00040F2F313A1F5836103FB01F140F2E7335B
:10D7E00091FBF3F101F2DD5189B2FFF764BA00BF9A
:10D7F00078630020949F0020C1860020A0BD0020F7
:10D80000300A0020859F0020183B00204C46002055
:10D810001C3B0020789B0020A0890020B86D0020D0
:10D8200090E33FF408B501210220FCF7D5F8094B3D
:10D830001B7803F00503052B08D000210120FCF71D
:10D84000CBF800210846FCF7C7F8FEE715F096FA7A
:10D85000F3E700BFE4380020022828BF022010B4FC
:10D86000084C094B207000EB8002C0EBC202074954
:10D870005DF8044B013003EB4203C0B20B6017F0BC
:10D88000E5BA00BF859F0020EE8A0020949F00200B
:10D8900008B522F093FEFCF7D9FCBDE8084022F061
:10D8A00075BE00BF38B5484B5A899989914224BF4B
:10D8B00000225A81198ADA89914224BF0022DA8132
:10D8C000DA78CAB1072A41496AD091F85700404D29
:10D8D000012400210A282C709C70D9715DD00C287D
:10D8E00007D0002A6CD0DFED3B7A072A0ED00A2839
:10D8F00062D0DFED397A09E0344A92F857000A28FD
:10D9000056D00C285BD1D979DFED347A344C9FEDB9
:10D91000350AA278002918BFF0EE407A062A04D80A
:10D92000314901EB820191ED0F0A217979B1013A78
:10D93000032A0BD8F7EE007A87EE800A31F0B6FBA7
:10D940002388984228BF1846208038BD38BD9B7870
:10D950001F4A07EE103A1178B8EEC77A67EE277AB9
:10D9600007EE101AB8EEC77A27EE277AB4EEC70A88
:10D97000F1EE10FAEADD80EE277AFDEEC77A17EEB7
:10D98000903A102BA8BF1023012BB8BF0123DBB2A4
:10D990008B4238BF0B46137038BDDFED147AA4E715
:10D9A00091F857000A2803D00C28ACD0D9799AE70F
:10D9B000D979DFED0E7AA9E7DFED0D7AA6E7D979FF
:10D9C000DFED047AA2E700BF78630020C4B4002032
:10D9D000A08900206F1203396F12833A0AD7A33946
:10D9E000486000206F120338901404085304E9388B
:10D9F0000F506E3A38B50D4C0D4DAC4206D26168F1
:10DA000020461434FCF7AEFBAC42F8D3FDF72CFAF9
:10DA1000084A094B094C1460002209491A705A70CF
:10DA200008480860BDE838401AF00EBA88010008BE
:10DA300024060008949F0020859F0020EE8A002085
:10DA4000244A0020989F002008B5FFF7D3FF22F05A
:10DA5000B5FDFCF7FBFBBDE8084022F097BD00BF19
:10DA6000F0B50C2934D8DFE801F0893333335E3365
:10DA70003333343333330700048C9689B2F802E031
:10DA80001788734D24F480542404240C0484038CDC
:10DA90008488818B23F4005321F4E6411B0409049C
:10DAA0001B0C46EA0E06090C43EA063341EA07213D
:10DAB000A8429BB2A4B289B200F09E8005F58065B1
:10DAC000A84200F099809268848081830264038474
:10DAD000F0BD048C9589B2F802C0B2F800E05C4F4A
:10DAE00024F480742404240C0484038C8688818BA1
:10DAF00023F400731B0421F073011B0C45EA0C0492
:10DB0000090443EA0423090CB8429BB2B6B241EAC5
:10DB10000E015CD04F4CA04259D092688680818320
:10DB2000C2630384F0BD048C9589B2F802C0B2F8D8
:10DB300000E0474E24F010042404240C0484038CD9
:10DB40008788018B23F0200321F4E6411B0409049C
:10DB50001B0C45EA0C04090C43EA041341EA0E21AC
:10DB6000B0429BB2BFB289B25DD03A4CA0425AD00B
:10DB700092688780018382630384F0BD048C978957
:10DB8000B2F802E01688324D24F001042404240C7B
:10DB90000484038C8488018B23F002031B0421F08E
:10DBA00073011B0C47EA0E0709043B43090CA8420A
:10DBB0009BB2A4B241EA060125D005F58065A842D2
:10DBC00021D092688480018342630384F0BDD589AB
:10DBD000148A578A23F4006343EA05254FF6FF337E
:10DBE0002B40958826F440563C4343EA052346EAF9
:10DBF00004169BB2B6B290E7158A24F4804444EA36
:10DC00008514A4B25FE7D689158A578A23F00803E2
:10DC1000334324F4407496883D4323F004032C439B
:10DC20003343A4B2CDE7D489158A568A23F0800302
:10DC300043EA04134FF6BF741C40938827F44067EF
:10DC4000354344EA031347EA85079BB2BFB28FE727
:10DC500000000140000401402DE9F04FC8220021DE
:10DC600083B08A488A4CDFF84C928A4D8A4E8B4F9B
:10DC7000DFF8448233F025FB89488A49DFF83CE22B
:10DC8000DFF83CC200221359834200F0D580B3F183
:10DC9000804F00F0E580AB4200F0E480B34200F03A
:10DCA000E380BB4200F0E280734500F0E180634511
:10DCB00000F0E080434500F0DF80DFF808A2534524
:10DCC00000F0DC800AF5806A534500F0D9800AF53F
:10DCD000806A534500F0D680AAF5983A534500F083
:10DCE000D3800AF5806A53457BD00AF5806A534594
:10DCF00008BF0D2376D01832C02AC4D1644C6A4EB6
:10DD00006A4F6B4D04F1C00802E01834A04565D09D
:10DD1000A379002BF9D023794FEA131909F1FF39C0
:10DD2000B9F1030F03F00F03EFD836F8190040FAEA
:10DD300003F2D207E9D54FF0010A0AFA03F3013BD7
:10DD4000184030F045FF17F80930184415EBC002B1
:10DD5000DBD055F83000DFF870E1217A00F13F4365
:10DD600003F57E039B0A1EF8033003F01F0E5B09C8
:10DD7000032B0AFA0EFA61D0042B68D0022B52D082
:10DD800093880093B3FA83F3C3F11F039BB2DA08BD
:10DD900000EB820203F00703D2F820E09B004FF073
:10DDA0000F0C0CFA03FC2EEA0C0EC2F820E0D2F89D
:10DDB00020E001FA03F343EA0E03136269460023ED
:10DDC000022218348DF804208DF805308DF80630C5
:10DDD0008DF8073022F030FEA04599D103B0BDE8A0
:10DDE000F08F0C2309EBC3034FF0010A93F85C306A
:10DDF00003F01F0B5B09032B0AFA0BFA09D0042B63
:10DE00000CD0022B7FF477AF4B6C4AEA03034B64D0
:10DE100071E70B6C4AEA03030B646CE70B6B4AEA8D
:10DE200003030B6367E7DFF87CE0DEF844304AEA7F
:10DE30000303CEF84430A3E70023D3E7DFF864E020
:10DE4000DEF840304AEA0303CEF8403098E7DFF8C6
:10DE500054E0DEF830304AEA0303CEF830308FE782
:10DE60000123BFE70223BDE70323BBE70423B9E790
:10DE70000523B7E70623B5E70723B3E70823B1E790
:10DE80000923AFE70A23ADE70B23ABE7A4A00020EB
:10DE9000004404080004004000080040000C00405A
:10DEA0000000014000380240C0440408C84404088F
:10DEB00070A80020901404080004014000100040E5
:10DEC0000014004000400140904604080149024807
:10DED000FEF7B6BB44A100200040014001490248C2
:10DEE000FEF7AEBB1CA1002000040140014902481E
:10DEF000FEF7A6BB1CA10020000401400149024816
:10DF0000FEF79EBBF4A00020000C0040014902482F
:10DF1000FEF796BBCCA000200004004002494FF061
:10DF20008040FEF78DBB00BFA4A00020F0B50468C0
:10DF3000474DA30AAB426ED009D8B3F5801F66D017
:10DF4000023DAB4258D14FF0480E012608E0414D4A
:10DF5000AB4264D00F35AB424FD14FF0C00E042618
:10DF60004779B0004FEA970C00295CD0634602273E
:10DF7000A5899F4083190CEB43032F4303F1040C45
:10DF8000354DBFB245F8231045F82C20A781EFF39B
:10DF90001181502282F31288821905EBC2021369A3
:10DFA00063B313620433821905EBC202576917B1D8
:10DFB0001F6053690433821905EBC202976917B1D8
:10DFC0001F6093690433821905EBC202D76917B148
:10DFD0001F60D36904330027CAB21F6082F311881F
:10DFE000304405EBC000036A5BB9A38923F0010349
:10DFF0001B041B0CA381F0BDF0BDF0BD05EB0E03AF
:10E00000D1E7A3899BB243F00103A381F0BD4FF098
:10E01000200E0026A4E74FF0700E0226A0E74FF076
:10E02000980E03269CE70223BF0803FA07F7A3898B
:10E03000094D9BB223EA070387190CEB470CA38118
:10E040000CF1040345F82C1045F823209FE700BF8E
:10E050000300100041001000A4A0002010B50368C8
:10E0600083480139834282B089B200F0CB80A0F5A9
:10E070008060834200F0C68000F58040834200F05B
:10E08000B88000F58060834200F0B38000F58060C6
:10E09000834200F0AE80774C188824686408B4FB93
:10E0A000F2F4013CA4B282B2B3F1804F0AD07248BC
:10E0B000834207D000F58060834203D000F5806082
:10E0C000834202D122F0700292B26C48834200F087
:10E0D000A28000F58060834200F0A78022F44072A5
:10E0E00000F56C4092B283421A80D9621C854FD0F1
:10E0F0005F4A93424CD001229A821A8892B242F02F
:10E1000001021A80B3F1804F00F099805A4A93427D
:10E1100000F0978002F58062934200F0948002F54F
:10E120008062934200F0918002F58062934200F099
:10E130008E8002F58062934200F08B8002F570427F
:10E14000934200F0888002F57052934200F085807F
:10E1500002F58062934200F0828002F58062934271
:10E160007FD0A2F5983293427DD002F5806293422F
:10E170007BD002F58062934208BF0D2215D002A821
:10E180004FF0012340F8043D22F0A6FE02B010BD7E
:10E190000122002119869A821A88394892B242F0E7
:10E1A000010283421A80ADD10A46364B03EBC2030B
:10E1B00001A893F85D408DF80440012300228DF8FA
:10E1C00005308DF807308DF8062022F085FE1B2CD7
:10E1D00008D02E2CDAD12C4B019301A822F07CFE22
:10E1E00002B010BD294B019301A822F075FE02B0C8
:10E1F00010BD204C18882468B4FBF2F4013CA4B292
:10E2000082B251E71B4C18882468B4FBF2F4013C3D
:10E21000A4B282B256E701201A80D9621C85988286
:10E220001A8892B202431A8070E701201A80D962DC
:10E230001C8598821A8892B202431A8062E70122F2
:10E24000B3E70222B1E70322AFE70422ADE70522DC
:10E25000ABE70622A9E70722A7E70822A5E70922DC
:10E26000A3E70A22A1E70B229FE70C229DE700BF4C
:10E2700000040140F8A90020000400400010004004
:10E2800000000140901404082C0100011901000154
:10E290002C4B98423DD0B0F1804F3CD0A3F57C434D
:10E2A00098423AD003F58063984238D003F58063F2
:10E2B000984236D003F58063984234D003F58063EA
:10E2C000984232D003F57043984230D003F5705332
:10E2D00098422ED003F5806398422CD003F58063DA
:10E2E00098422AD0A3F59833984228D003F580634A
:10E2F000984207D003F58063984208BF0D2202D0F0
:10E30000002070470C22104B03EBC20393F85C0013
:10E3100070470022F7E70122F5E70222F3E7032224
:10E32000F1E70422EFE70522EDE70622EBE70722FB
:10E33000E9E70822E7E70922E5E70A22E3E70B22FB
:10E34000E1E700BF00000140901404082DE9804877
:10E35000013085B0C3B203938A4D8B4F8B4C8C4EEA
:10E360000A230293DFF82C922EF000FC4FF4FA7A85
:10E370004FF0100C4FF47A70D9F80430C3F308034F
:10E38000002B40F0C180EFF31183002B40F0BC80E4
:10E390002968A26800BF2B689942F9D1D7F800E03C
:10E3A00000FB0EF39B1AB3FBFEF300FB01314FF0B1
:10E3B000010E0191D9F80430C3F30803002B40F09B
:10E3C0008780EFF31183002B40F082802B68A168D7
:10E3D00000BF2A689342F9D1D7F800B000FB0BF2D6
:10E3E000521AB2FBFBF200FB0323019A9B1AB3F50E
:10E3F0007A7FDFD3BAF1010ABED1039B002B40F034
:10E40000BD804FF47A7ADFF88C9150464FF0100CB3
:10E41000D9F80430C3F30803002B40F09280EFF3E7
:10E420001183002B40F08D802968A26800BF2B6803
:10E430009942F9D1D7F800E000FB0EF39B1AB3FB29
:10E44000FEF300FB01314FF0010E0191D9F80430C9
:10E45000C3F3080303BBEFF31183EBB92B68A16887
:10E4600000BF2A689342F9D1D7F800B000FB0BF245
:10E47000521AB2FBFBF200FB0323019A9B1AB3F57D
:10E480007A7FE3D3BAF1010AC2D1029B013B029326
:10E490007FF468AFFDF75CF9EFF311888CF3128815
:10E4A000A1682368DB0344BFC6F800E0A1682B68BD
:10E4B00032685FFA88F888F31188D7F800801A4428
:10E4C00000FB08F35B1AB3FBF8F300FB0233D4E75D
:10E4D000EFF311888CF31288A1682368DB0344BF33
:10E4E000C6F800E0A1682B6832685FFA88F888F304
:10E4F0001188D7F800801A4400FB08F35B1AB3FBBD
:10E50000F8F300FB023370E7EFF311828CF312880B
:10E51000D4F808E02368D90303D501233360D4F885
:10E5200008E02B683168D2B282F311883A68194446
:10E5300000FB02F3A3EB0E03B3FBF2F300FB01318C
:10E5400035E7EFF311828CF31288D4F808E02368E2
:10E55000D90303D501233360D4F808E02B68316870
:10E56000D2B282F311883A68194400FB02F3A3EB9C
:10E570000E03B3FBF2F300FB013164E718462EF003
:10E5800069F93EE78CB4002090B4002010E000E070
:10E5900088B4002000ED00E02DE9F047B14FB24E05
:10E5A00022F00CF8BE421ED2DFF85083DFF8509301
:10E5B0004446258862197DB14A450DD2052D0BD9F7
:10E5C00033886188C3F30B03994200F0FA80144644
:10E5D00025886219002DEFD1716830461436FBF79B
:10E5E000C1FDBE42E4D3A14A1378A3F11701022969
:10E5F0000FD99F4911F83300002840F08381D800DB
:10E600000144497829B19B4911F833300BB91823DB
:10E610001370994C6378022B84BF002363702378B6
:10E62000022B84BF00232370944B9A78042A00F0B5
:10E630000F8132B91A88B2F5F07F84BF4FF4F072BF
:10E640001A808F4D8F4A2B681A40002A00F0638190
:10E65000D80700F1F880590400F1F0801A0700F1A2
:10E66000E8809B0400F1DE80874D2B685A8C998CE2
:10E67000914224BF00225A84FFF714F91FF068F872
:10E68000002800F0C0804FF40070FBF7A1FD4FF4AC
:10E690008020FBF79DFD4FF40010FBF799FD4FF034
:10E6A0000070FBF795FD4FF08060FBF791FD774B15
:10E6B0001B78042B00F0AB80012B00F0A88063785E
:10E6C000022B06D8724A734903EB430302EB830320
:10E6D0000B602378022B07D803EB83016E4AC3EB50
:10E6E000C10302EB43032B601AF0FEFE002130222F
:10E6F0006A4832F0E6FD28682DF096FC684B2D68DC
:10E7000003F1500102E0043399427AD01A78002ACA
:10E71000F9D19C78D8788442F5D26249624B0A706C
:10E7200028461D6029F0E2FE604B614A1E7961496E
:10E730006148624B1160C825642212FB0652604C8E
:10E74000406B31F8061C5A60002221809A60DA6022
:10E750001A615A619A61DA6183F8202083F82120D6
:10E7600008B121F0F1FD574B9FED575A1B88574ACE
:10E770009FED576A5579574C57495848086006EE3F
:10E78000903AF8EEE66A1388C5EE265A07EE103A7C
:10E7900053881279C4ED005A07EE903AB8EEC77A62
:10E7A0004F4BF8EEE77A1D725A7227EE067A67EE43
:10E7B000867ABDE8F04783ED017AC3ED007A21F057
:10E7C000E5BE63799B077FF402AF716894F804A0FB
:10E7D0003046FBF7C7FC3388BAEB133F04D014363E
:10E7E000BE42FFF4E5AEFEE673887068AA1FC3F36D
:10E7F0000B039A4204F10601A8BF1A4630F0E2FA70
:10E80000EDE7012289E7374814F026FF3BE7364B56
:10E810009A78022A04BF00229A706378022B7FF64E
:10E8200051AF56E73148FBF7D3FC4020FBF7D0FC53
:10E830001AE72F48FBF7CCFC2B6812E72D48FBF7B3
:10E84000C7FC2B680AE72C48FBF7C2FC2B6802E7E1
:10E850009A8AB2F57A7FBFF4F4AE4FF47A729A8254
:10E86000EFE600BF2406000888010008D4890020D4
:10E8700000370408F4440408859F00204860002005
:10E88000248C002009600002949F0020E5380020BD
:10E89000989F0020244A0020EE8A00204C2300206C
:10E8A000D88900201403002080230020AC3D0020E4
:10E8B00078BD0020B2890020D8450020549B00205C
:10E8C0002C820020BC230020C0C9FB48C41F0020AC
:10E8D00017B7D138C0230020843B00203661023DA9
:10E8E000603B002064A700200A8C00200940000241
:10E8F00001600002092000020860000202400008D6
:10E9000000800008D8000C186468002C7FF478AEF2
:10E910001724147074E643F008032B6098E600BFD8
:10E9200008B521F04BFEFBF791FC21F02FFEFFF71D
:10E9300033FE0120BDE8084016F088BA2DE9F04FFB
:10E94000013085B0C3B203930B4602918B4C8C4EC1
:10E95000002B00F099808B4D8B4FDFF830922EF01A
:10E9600005F94FF4FA7A4FF0100C4FF47A70D9F899
:10E970000430C3F30803002B40F0DE80EFF3118373
:10E98000002B40F0D9802968A26800BF2B6899420B
:10E99000F9D1D7F800E000FB0EF39B1AB3FBFEF3AE
:10E9A00000FB01314FF0010E0191D9F80430C3F39F
:10E9B0000803002B40F08780EFF31183002B40F019
:10E9C00082802B68A16800BF2A689342F9D1D7F8EA
:10E9D00000B000FB0BF2521AB2FBFBF200FB032368
:10E9E000019A9B1AB3F57A7FDFD3BAF1010ABED13F
:10E9F000039B002B40F0BD804FF47A7ADFF88C91B6
:10EA000050464FF0100CD9F80430C3F30803002B24
:10EA100075D1EFF31183002B71D12968A26800BF73
:10EA20002B689942F9D1D7F800E000FB0EF39B1A4E
:10EA3000B3FBFEF300FB01314FF0010E0191D9F859
:10EA40000430C3F3080313BBEFF31183FBB92B6846
:10EA5000A16800BF2A689342F9D1D7F800B000FB43
:10EA60000BF2521AB2FBFBF200FB0323019A9B1A32
:10EA7000B3F57A7FE3D3BAF1010AC4D1029B013B1B
:10EA80000293002B7FF467AF05B0BDE8F08FEFF382
:10EA900011888CF31288A1682368DB0344BFC6F891
:10EAA00000E0A1682B6832685FFA88F888F3118863
:10EAB000D7F800801A4400FB08F35B1AB3FBF8F3A5
:10EAC00000FB0233D2E7EFF311888CF31288A168C0
:10EAD0002368DB0344BFC6F800E0A1682B683268F6
:10EAE0005FFA88F888F31188D7F800801A4400FB91
:10EAF00008F35B1AB3FBF8F300FB023370E7EFF3A4
:10EB000011828CF31288D4F808E02368D90303D566
:10EB100001233360D4F808E02B683168D2B282F365
:10EB200011883A68194400FB02F3A3EB0E03B3FB10
:10EB3000F2F300FB01317FE7EFF311828CF31288CF
:10EB4000D4F808E02368D90303D501233360D4F84F
:10EB500008E02B683168D2B282F311883A68194410
:10EB600000FB02F3A3EB0E03B3FBF2F300FB013156
:10EB700018E718462DF06EFE3EE700BF10E000E0FB
:10EB800088B400208CB4002090B4002000ED00E098
:10EB9000204B5B68C3F3080330B4BBB9EFF31183B8
:10EBA000A3B91D4B1D4C1868A16800BF1A6890429C
:10EBB000F9D11B4B1C684FF47A7202FB04F3591A0B
:10EBC000B1FBF4F130BC02FB00107047EFF311828F
:10EBD000102383F3128811498C680B6813F4803F6B
:10EBE000104B02D0012018608C680B49D2B20D681E
:10EBF000186882F311880A4B19684FF47A72284416
:10EC000002FB01F31B1B30BCB3FBF1F302FB003032
:10EC1000704700BF00ED00E08CB4002010E000E081
:10EC200090B4002088B400202DE9F84F8046FFF70B
:10EC3000AFFF254E2549DFF8A0E0254A254D844643
:10EC400010274FF47A740120DEF80430C3F3080370
:10EC5000D3B9EFF31183BBB90B68D2F808A000BF9A
:10EC6000D1F800904B45F7D1D6F800B004FB0BF972
:10EC7000A9EB0A09B9FBFBF904FB0393A3EB0C0313
:10EC80004345E1D3BDE8F88FEFF3118A87F312888B
:10EC9000D2F808B01368DB0344BF2860D2F808B08C
:10ECA0000B68D5F800905FFA8AFA8AF31188D6F8D3
:10ECB00000A0994404FB0AF3A3EB0B03B3FBFAF3A4
:10ECC00004FB0933DAE700BF90B400208CB40020C5
:10ECD00010E000E088B4002000ED00E02DE9F04FE6
:10ECE000DFF830C1474A4849484E494D8046102711
:10ECF00018F1FF38C0F08480DCF80430C3F3080357
:10ED0000002B5CD1EFF31183002B58D10B68946872
:10ED100000BF08688342F9D1D6F800904FF47A70AA
:10ED200000FB09FEAEEB040EBEFBF9FE00FB03EE9A
:10ED3000DCF80430C3F308034FF47A740120FBB904
:10ED4000EFF31183E3B90B68D2F808A000BFD1F844
:10ED500000904B45F7D1D6F800B004FB0BF9A9EBB6
:10ED60000A09B9FBFBF904FB0393A3EB0E03B3F50C
:10ED70007A7FBDD2DCF80430C3F30803002BDFD068
:10ED8000EFF3118A87F31288D2F808B01368DB0317
:10ED900044BF2860D2F808B00B68D5F800905FFA3D
:10EDA0008AFA8AF31188D6F800A0994404FB0AF382
:10EDB000A3EB0B03B3FBFAF304FB0933D5E7EFF343
:10EDC000118487F31288D2F808901368D80303D50A
:10EDD00001232B60D2F808900B682868E4B284F312
:10EDE0001188D6F800A04FF47A7400EB030E04FBF0
:10EDF0000AF3A3EB0903B3FBFAF304FB0E3E97E718
:10EE0000BDE8F08F10E000E08CB4002090B400204A
:10EE100088B4002000ED00E030B4EFF3118310223D
:10EE200082F312880649074C0A6807480132002518
:10EE30000A602560DBB2026883F3118830BC70473A
:10EE40008CB4002088B4002010E000E00F4B1B8839
:10EE5000014643B90E4B0F4A1B7810680BB981F07D
:10EE60000101FAF7B1BD0C4B5A691AB118B91A6809
:10EE7000106058747047094A18681188084A92FB54
:10EE8000F1F2012102605974704700BFBCBC002040
:10EE9000BEBC0020C0BC0020C4BC0020DCBC0020E4
:10EEA00020A1070038B5254B5C69236B73B1636DF6
:10EEB000626BCAB1998A1A88C90592B201D5D20784
:10EEC00000D438BD4FF6F7721A8038BD636D99894A
:10EED0001A88890692B2EBD59206E9D5E26ACAB1E0
:10EEE000988880B29047E2E799891A880D0692B215
:10EEF000E0D51006DED5A26A616A8A4219D0A169FE
:10EF00002569885C98800132B2FBF5F105FB11227E
:10EF1000A262CFE79B88E2696169DBB28B54E26948
:10EF2000E068636D0132B2FBF0F100FB1122E26197
:10EF3000BEE7DA6822F08002DA60BBE7E83800203A
:10EF400038B5254BDC68236B73B1636D626BCAB156
:10EF5000998A1A88C90592B201D5D20700D438BD62
:10EF60004FF6F7721A8038BD636D99891A88890641
:10EF700092B2EBD59206E9D5E26ACAB1988880B21E
:10EF80009047E2E799891A880D0692B2E0D51006FB
:10EF9000DED5A26A616A8A4219D0A1692569885CB6
:10EFA00098800132B2FBF5F105FB1122A262CFE796
:10EFB0009B88E2696169DBB28B54E269E068636D4A
:10EFC0000132B2FBF0F100FB1122E261BEE7DA6828
:10EFD00022F08002DA60BBE7E838002038B5254B24
:10EFE0009C68236B73B1636D626BCAB1998A1A888E
:10EFF000C90592B201D5D20700D438BD4FF6F772D9
:10F000001A8038BD636D99891A88890692B2EBD54A
:10F010009206E9D5E26ACAB1988880B29047E2E7E1
:10F0200099891A880D0692B2E0D51006DED5A26A3B
:10F03000616A8A4219D0A1692569885C9880013289
:10F04000B2FBF5F105FB1122A262CFE79B88E269D2
:10F050006169DBB28B54E269E068636D0132B2FB37
:10F06000F0F100FB1122E261BEE7DA6822F08002D3
:10F07000DA60BBE7E83800202DE9F04F2DED028B78
:10F0800095B0804626F044FA8E4B1D7825B115B018
:10F09000BDEC028BBDE8F08F8B4B1B685905F6D594
:10F0A0008A4BDFF880B21B686BB1894ADBF800102D
:10F0B0001368CB1A7C2B06D986481160037801337C
:10F0C000037016F0B9FF844B1B78002B6DD0834C76
:10F0D000834AD4F81031A8EB0303934201F227834B
:10F0E00094F81891B9F1000F32D17E4F3868F9F7D2
:10F0F000D5FFC0B201280FD902287B4E42F0138001
:10F100003378002B42F00881D4F81C31A8EB0303BC
:10F11000B3F57A6F82F0CE82D4F82031002B44D040
:10F1200094F81831BBB9714B1B689B7801211E3BC9
:10F1300000228B4284F8181184F82C2142F26C8250
:10F1400038680221043016F029FF94F8243110E0C9
:10F15000D4F820314BB3D4F8283140F6B732A8EBBD
:10F160000303934221D994F82431002B01F0D9866E
:10F170005C4F013BDBB284F82431002B01F00A84A0
:10F18000D4F8206194F82C2116F8011B94F82D3145
:10F190003868C4F820610A44013384F82C2184F8CB
:10F1A0002D31F9F77FFFC4F82881514BDBF800605F
:10F1B0001B7843B14F4F386828B14F4B1B78013B48
:10F1C000012B41F2F6834D4B1B786BB14C4F3B68E2
:10F1D00053B1DBF80030414C03931A46D4F8443164
:10F1E000D31A632B01F29381464F3B78022B01F037
:10F1F00078863D4E96F87430032B01F0B683424B6F
:10F200001B7873B1414D2B685BB1344CFFF7C0FCE8
:10F21000D4F85031039044F61F62C31A934200F2AF
:10F2200031813B4B1B78002B7ED13A4B1B7843B18D
:10F230002A4CD4F8A03203F5C333A033984581F0AB
:10F240003782354B1B78002B3FF421AF234E334CD4
:10F25000334D06F2C1272068F9F720FF00283FF45C
:10F2600016AF2068F9F712FF2B7880465A1E33B18B
:10F2700020682A70F9F712FF0028F2D107E703226D
:10F280003946781E32F003F896F8C03296F8C1225B
:10F2900086F8C38283F47F4383F0FF039B1A1FFA2F
:10F2A00088F89BB2B8EB132FD5D196F8C222DBB207
:10F2B0009A42D0D1781E16F0A3FB2B781844287000
:10F2C000C9E700BFC44900209C630020B843002068
:10F2D0002846002024460020169C0020D41F002031
:10F2E0003F0D0300D045002028000020D445002019
:10F2F000189C0020C0430020209C0020289C002057
:10F30000C845002066AB0020309C0020349C0020C3
:10F31000A09C0020B19C00203A9C0020409C002032
:10F32000449C00208CB40020484C2278A2B1484B69
:10F330009B7A53B1FFF72CFC464B1B68C31AA3F50D
:10F340007A73B3F5FA6F07D82278434B43491868AC
:10F35000F9F770FE00232370414CD4F8983203F57E
:10F36000C333A0339845FFF460AF3E4DC4F8988294
:10F370002B78002B41F010873B4D2B78002B41F070
:10F380006B8694F89C2239498D5CEA0702F107806C
:10F39000AF0701F1C787680701F188872A0748D5B9
:10F3A000334B344E0D9314AA1146A3F13D0241F89C
:10F3B000202D0020A3F140020D4603F8400C0591DA
:10F3C000022311215170937028463168FBF764F9CC
:10F3D00028467168FBF760F9F389274903EBC303FB
:10F3E0009B00053381FB0321DB17C3EBA1012846FA
:10F3F00089B2FBF769F9338A03EB8303590089B2B9
:10F400002846FBF761F91D4B059D1B789B0743BF01
:10F41000318901F57A7189B24FF47A712846FBF788
:10F4200053F90C9B327D591C0C9128461A7025F01B
:10F43000FFFF134A94F89C321178013393FBF1F2E9
:10F4400001FB123384F89C32EFE600BF089C0020D9
:10F450001465002008860020A49C0020C89B002082
:10F46000D41F0020A89C0020A99C0020AC9C002058
:10F47000C89B002054460020676666665046002000
:10F48000B09C002094F85631002B41F0CB85D34B33
:10F490001A6802F00803002B48F603414AF60B40B5
:10F4A0004BF60F4349F6074604BF03460E4612F0DB
:10F4B000040F4FF0190118BF1E46970684F8561125
:10F4C00003D546F4804646F02006C54B5F79C6F367
:10F4D0000909002F42F013819B79002B42F01E8214
:10F4E0001F4664204FF0FF3A4FF0000E0C960D9629
:10F4F000ADF83E70ADF83CE0CDF842E0CDF846E026
:10F50000CDF84AE0CDF83890ADF840A08DF84E0027
:10F510000CAE0FCEB34F84F805E00FC796E80F008E
:10F5200007C727F8023B39464FF0010E1B0CFE2699
:10F530001F20C82201F81E39A670A27184F807E0C6
:10F54000E07094F86601207180F0F10383EA031300
:10F55000DAB2130983F0E70343EA022383EAC20322
:10F560001BB283EA0312D2B2C3F3072383EA121356
:10F5700043EA022383EAC2031BB283F0C80282EA91
:10F580000212D2B2C3F3072383EA121343EA02231F
:10F5900083EAC2031BB283EA0E0686EA0616F6B2B7
:10F5A000C3F3072282EA161242EA062200EB0E0398
:10F5B00082EAC60607EB0E0084F86631268011F851
:10F5C000013B734083EA0313DBB21A0982EA162275
:10F5D00042EA032282EAC3031BB29EB28142268022
:10F5E000EDD183F07C0383EA0313DBB24FEA131EF1
:10F5F0008EEA162E8EEA032E8EEAC30E0FFA8EFEC8
:10F600001FFA8EFC784FA4F800C05FFA8EFE4FEA16
:10F610001C2C84F828C084F827E007F5C77904F18A
:10F62000220A38687968BA68FB684E460FC61037F8
:10F630005745B146F5D1386830606C4E3B7989F852
:10F64000043006F1270784F8B5E184F8B6C116F84E
:10F65000011F2868F9F726FDB742F8D194F8573111
:10F66000002B41F0E4846249DBF8002009780A208D
:10F6700084F85701002901F000865E4E0129308888
:10F68000079042F2518170880690022902F04F8063
:10F69000B0880590032902F05E81F0880490042967
:10F6A00002F054810529308902F04C810629B6F810
:10F6B0000A9002F044810729B6F80CC000D0F38903
:10F6C00094F866110C920F4687F0300282EA02121B
:10F6D000D2B216094849089786F07A0646EA022609
:10F6E0000988277186EAC202444EC1EB012186FBDC
:10F6F000017A079E4FF0000E66F30F0E069E12B2BF
:10F7000066F31F4E8A44059ECDF834E0C917C1EB5D
:10F710006A2A002782EA0211C9B266F30F07C2F310
:10F720000722002682EA111260F30F0600200792DA
:10F730006CF30F00049A8DF845A063F31F40079BFC
:10F74000109062F31F4769F31F464FF000090E97B0
:10F750000F968DF8449043EA01220DF1300E82EAB3
:10F76000C106BEE80F0036B286F0C80C8CEA0C1C4D
:10F770001C4F84F805905FFA8CFCC6F307260FC770
:10F7800086EA1C1646EA0C239EE8030083EACC03B3
:10F790001BB283F0230247F8040B82EA0212D2B2B2
:10F7A000C3F30723089E83EA1213384643EA022371
:10F7B00083EAC20206F1010E20F814194FF0230C5F
:10F7C0001621FE26C82384F866E102372280E17004
:10F7D00084F807C0A670A371114611E04C460020C2
:10F7E00038460020DC1F0020D61F002063210020A7
:10F7F000BC9F0020DC5E0020489B00200308208086
:10F8000010F8013B4B4083EA0313DBB21A0982EA8A
:10F81000112242EA032282EAC3031BB299B2B84220
:10F820002180EDD183F0F40383EA0313DBB24FEAC6
:10F83000131E8EEA112E8EEA032E8EEAC30E0FFAE5
:10F840008EFE1FFA8EF7C84E27804FEA172C5FFAFC
:10F850008EFE84F81EE084F81FC07168B2683068BC
:10F86000F36806F5C7770FC730697169B26904F2AA
:10F870008F1607C704F2AD1784F8ADC184F8ACE168
:10F8800016F8011F2868F9F70DFCB742F8D194F873
:10F890005A31002B41F0DB83B44B06931B681922CD
:10F8A000980684F85A2140F1EA82B14BB14E1B7898
:10F8B000990741F12187337D042B8CBF0327022751
:10F8C000FFF766F9338A32890C9003EB83035B0000
:10F8D000ADF84A304FF47A7033688DF84C700E935F
:10F8E000F18996F814E073688DF84DE000FB02F2A0
:10F8F0004FF0000C0CAF4FF0FF30CDF834C0109239
:10F900000F93ADF848101190BE46BEE80F00059762
:10F91000994F0FC79EE80F0007C73A46182122F8F3
:10F920001C39E17194F8661184F805C081F0780300
:10F9300083EA0313D8B2030983F0F60343EA0023F2
:10F9400083EAC0031BB283EA0310C0B2C3F30723E8
:10F9500083EA101343EA002383EAC0031BB283F057
:10F96000C80080EA001E5FFA8EFEC3F3072080EA1B
:10F970001E1040EA0E2080EACE0000B280F018038C
:10F9800083EA0313DBB2C0F3072080EA131040EAD6
:10F99000032080EAC30301F1010EFE204FF01E0C8C
:10F9A0004FF0C809A0700237217184F866E1238006
:10F9B00084F803C084F80690184612F8011B4140F1
:10F9C00081EA0111C9B20B0983EA102343EA01233A
:10F9D00083EAC10109B288B2BA422080EDD181F038
:10F9E000180181EA0111C9B20A0982EA102383EAE7
:10F9F000012383EAC1031BB29AB25B490491DBB2D3
:10FA00004FEA122C2280079384F827C084F826300E
:10FA10000F4601F5C77A04F1220938687968BA6897
:10FA2000FB68D646AEE80F0010374F45F246F4D1DA
:10FA30003868CEF80000DFF84C919DF81C3084F84F
:10FA4000B43109F1260784F8B5C1CA461AF8011F76
:10FA50002868F9F727FB5745F8D1FFF799F8069B77
:10FA600071681B683289069113F0140F4FF47A7194
:10FA7000D6F800E001FB02F141F00B860E4694F847
:10FA800066A10C908AF06A003C4B3D4FB3F904200C
:10FA9000CDF834E080EA0010C0B2030983F0D5034A
:10FAA00043EA002383EAC0031BB283EA0310C0B217
:10FAB000C3F3072383EA101343EA002383EAC00356
:10FAC0001BB287FB0207D2174FF0000CC2EBA70254
:10FAD0000698DDF814E0109683F0C8070E900F9199
:10FAE000ADF84A20ADF844C0ADF846C0ADF848C006
:10FAF00087EA0717FFB2C3F30726BEE80F0086EABE
:10FB0000171646EA072686EAC7071B4E84F804A0A4
:10FB10003FB20FC687F021039EE8070083EA031374
:10FB2000DBB2C7F3072787EA13170AF1010E47EA8A
:10FB3000032786E8070087EAC30384F866E14FF0ED
:10FB4000210A4FF0FE0E1C27C8220C3684F805C08F
:10FB500084F807A084F802E0A6F11C01E7701846BB
:10FB6000A271238010E000BFD61F00204C46002069
:10FB70005046002054460020DC1F00203046002064
:10FB8000676666666321002011F8012B424082EA15
:10FB90000212D2B2130983EA102343EA022383EA52
:10FBA000C20212B290B2B1422080EDD182F068025E
:10FBB00082EA0212D2B24FEA121A8AEA102383EAC8
:10FBC000022A8AEAC20A0FFA8AFA1FFA8AF3D74E81
:10FBD00023804FEA132C5FFA8AFA04F1220384F897
:10FBE00025C084F824A006F5C77E0693F368306824
:10FBF0007168B26877460FC7069B10369E42BE46B4
:10FC0000F4D13388CA4E3B804F4684F8B2A184F8C1
:10FC1000B3C117F8011F2868F9F744FABE42F8D1BA
:10FC200094F866E1C34AC44E84F804E08EF0EB0316
:10FC300083EA0313D9B20B0983F0C50343EA012316
:10FC400083EAC1031BB283EA0310C0B2C3F30721E6
:10FC500081EA101141EA002181EAC0010CCA09B20F
:10FC600081F0C80787EA0717FFB24FF0000C0C922B
:10FC7000C1F30721059A0D93CDF838C081EA171317
:10FC800043EA072307CA83EAC7031BB283F031079D
:10FC900086E8070087EA0717FFB2C3F3072383EA62
:10FCA000171343EA072383EAC703277A607AA17A06
:10FCB000E27A267B84F805C01BB25F4087EA07170B
:10FCC000FFB2C3F3072383EA171343EA072383EA48
:10FCD000C7031BB2584080EA0010C0B2C3F3072329
:10FCE00083EA101343EA002383EAC0031BB259409E
:10FCF00081EA0110C0B2C3F3072181EA101141EA81
:10FD0000002181EAC00109B24A4082EA0212D2B25D
:10FD1000C1F3072383EA121343EA022383EAC203EF
:10FD20001BB25E4086EA0616F6B2C3F3072383EAE7
:10FD3000161343EA0623607BA17BE27B277C94F8C1
:10FD400011C083EAC6031BB2584080EA0010C0B25B
:10FD5000C3F3072383EA101343EA002383EAC003B3
:10FD60001BB2594081EA0111C9B2C3F3072383EAE8
:10FD7000111343EA012383EAC1031BB25A4082EA0A
:10FD80000212D2B2C3F3072383EA121343EA022317
:10FD900083EAC2031BB25F4087EA0717FFB2C3F3CF
:10FDA000072383EA171343EA072383EAC7031BB237
:10FDB0008CEA030C8CEA0C1C5FFA8CFCC3F307235F
:10FDC00083EA1C1343EA0C2383EACC03A17CE27C84
:10FDD0005A4F1BB2594081EA0111C9B2C3F307233C
:10FDE00083EA111343EA012383EAC1031BB25A4099
:10FDF00082EA0212D2B2C3F3072383EA121343EA60
:10FE0000022383EAC2031BB283F0270686EA0612A6
:10FE1000D2B2C3F3072686EA121646EA022686EA1B
:10FE2000C20636B20EF10103B2B231204FF0FE0C21
:10FE30000C2184F86631C8234FEA122E5FFA86FA45
:10FE40002280E07184F802C0E170A371049E84F8FE
:10FE500014A084F815E07168B268F3683068B6F8E9
:10FE600010C00FC727F803CB84F8A3E184F8A2A140
:10FE700019F8011F2868F9F715F94F45F8D194F8DA
:10FE80005E71002F41F0DE802D4B94F866E1B3F9EE
:10FE90000010B3F90220B3F904309FED2A6A6771AC
:10FEA00007EE103ADBF800300C938EF06A0383EA19
:10FEB000031306EE901AD9B20B0983F0D50343EA77
:10FEC000012383EAC1031BB283EA03115242C9B280
:10FED00007EE902AC3F3072383EA111343EA0123B1
:10FEE000F8EEE77AF8EEE66AB8EEC77A83EAC1037D
:10FEF0001BB267EE867A66EE866A27EE067A0020E7
:10FF000083F0C80CCDED0E7ACDED0D6A8DED0F7A34
:10FF10001090119012908CEA0C160DF13009F6B287
:10FF2000C3F3072CB9E80F000EE000BFD61F002076
:10FF300087210020FC460020DC1F002064210020D7
:10FF40003046002088C3E43A8CEA161C4CEA062CA2
:10FF50008CEAC60CD04E0FFA8CFC0FC68CF01E0734
:10FF600099E8070087EA0717FFB2CCF3072383EA73
:10FF7000171343EA072386E8070083EAC707C82167
:10FF80004FF005094FF01E0CFE231C200EF101025C
:10FF9000A17184F85E9184F807C0A370E070A6F1A7
:10FFA000100184F804E00C36278084F8662111F8EB
:10FFB000013B7B4083EA0313DBB21A0982EA172272
:10FFC00042EA032282EAC3031BB29FB2B1422780F6
:10FFD000EDD183F0270383EA0313DBB24FEA131E4C
:10FFE0008EEA172E8EEA032E8EEAC30E0FFA8EFECD
:10FFF0001FFA8EFCA94FA4F800C05FFA8EFE4FEAEC
:020000040801F1
:100000001C2C84F825C084F824E007F5C77904F196
:10001000220A38687968BA68FB684E460FC61037FE
:100020005745B146F5D19E4E3B88A9F8003006F100
:10003000240784F8B2E184F8B3C116F8011F2868D8
:10004000F9F730F8B742F8D194F85F91B9F1000FA1
:1000500040F0F287934B1B68052284F85F219A06D3
:1000600041F11581904ADFED917AD18907EE101A9E
:10007000B8EEC77A13F0140F27EE277A01F07183D8
:100080008B4BDFED8A6AD3ED007AF8EEE77A67EE04
:10009000A67A94F866C1874B874AB3F90410B2F97F
:1000A0000620864E86488DED0D7A8CF0220383EA79
:1000B0000313DFB23B0983F0590343EA072383EAC2
:1000C000C703B2F5FA6F1BB2A8BF4FF4FA6283EA16
:1000D0000317FFB2B2F57A7FC3F3072383EA17133E
:1000E000B8BF4FF47A724FF0640E43EA0723A2F5CB
:1000F0007A720EFB02F283EAC70786FB02E680FBF8
:1001000001E03FB2C917D217C2EBA612C1EBA003A0
:100110004FF0000A0CA987F0C806CDED0E7AADF8B5
:100120004220ADF84030CDF830A0CDF83CA08E464E
:1001300086EA0616F6B20591C7F30727BEE80F0058
:1001400087EA161747EA062787EAC606524FDEF8FF
:1001500000E084F804C00FC736B286F04A0383EA91
:100160000313DBB2C6F3072181EA13113A4641EAD1
:1001700003210CF1010C81EAC303142042F810E9B9
:10018000FE264FF04A0E002184F866C14FF0C80CDD
:10019000E0702380043784F807E0A670617184F86A
:1001A00006C0184612F8011B414081EA0111C9B28C
:1001B0000B0983EA102343EA012383EAC10109B250
:1001C00088B2BA422080EDD181F0140181EA011198
:1001D000C9B24FEA111E8EEA102E8EEA012E8EEA67
:1001E000C10E2E4B0FFA8EFE1FFA8EF61F464FEAF7
:1001F000162C5FFA8EFE84F81CE084F81DC0386867
:1002000059689A68DB68B7F818A0049726803E46BC
:1002100007F5C7770FC73069716903C704F28F16F6
:10022000A7F800A0374684F8ABC184F8AAE104F22D
:10023000AB1A17F8011F2868F8F734FFBA45F8D150
:10024000204B214A1B781278013B12F00100DBB2EF
:1002500014BFC0214021172B03D81C4A134493F824
:1002600030901B4B1A8897071ABF002341F01001EA
:10027000012312F4027F18BF022312F0100F18BFDF
:10028000062312F0200F18BF1023002841F0088227
:100290004FF0030C1EE000BFDC1F0020D61F002023
:1002A000632100204C460020544600200AD7233CFE
:1002B0002C46002030460020DC5E0020D34D62102A
:1002C00067666666D4890020C18600205815040838
:1002D0004A9B002094F866E10C938EF0460383EA73
:1002E0000313DAB2130983F0920343EA022383EA89
:1002F000C2031BB283EA0310C0B2C3F3072282EA2F
:10030000101242EA002282EAC00212B282F0C8074A
:1003100087EA0717FFB2C2F3072282EA1712002307
:100320008DF837C0032042EA072C059A8DF83490E7
:100330008DF835308DF836108DF8380007CA8CEA04
:10034000C70C0FFA8CFCD04FE3718CEA0C1903C771
:100350005FFA89F9CCF3072C8CEA191C4CEA0921C5
:1003600081EAC90994F808C03A700FFA89F98CEA51
:10037000090C8CEA0C1C5FFA8CFCC9F3072282EA98
:100380001C1242EA0C22607AA17A94F80B906371F5
:1003900082EACC0212B2504080EA001C5FFA8CFC68
:1003A000C2F3072080EA1C1040EA0C2080EACC004F
:1003B00000B2414081EA0111C9B2C0F3072282EACA
:1003C000111242EA012282EAC10212B289EA02094A
:1003D00089EA09195FFA89F9C2F3072282EA191238
:1003E00042EA092294F80CC0607BA17B84F804E007
:1003F00082EAC90212B28CEA020C8CEA0C1C5FFA87
:100400008CFCC2F3072282EA1C1242EA0C2282EA26
:10041000CC0212B2504080EA0010C0B2C2F30722F0
:1004200082EA101242EA002282EAC00212B251406D
:1004300081EA0111C9B2C2F3072282EA111242EA2B
:10044000012282EAC102E17B94F8109013B281EAA2
:10045000030282EA0212D2B2C3F3072383EA121321
:1004600043EA022383EAC2031BB289EA030282EA57
:100470000212D2B2C3F3072383EA121343EA022320
:1004800083EAC2031BB283F0320282EA0212D2B2C2
:10049000C3F3072383EA121343EA022383EAC20366
:1004A0001BB29AB24FF0FE0C5FFA83FB0920C82101
:1004B0000EF1010E84F802C04FEA122CE070A17117
:1004C00084F866E1228084F812C084F811B0049B9D
:1004D000186859689A68B3F80CA007F5C07EAEE8B2
:1004E000070007F5C8778EF80290AEF800A084F8F0
:1004F000A0C184F89FB116F8011F2868F8F7D2FD53
:10050000B742F8D1039BC4F85031FEF78ABEDFF83A
:1005100098A15E4EDFF89491412015F0EBFCBAF9FA
:10052000023086FB0320DB17C3EBA00080B215F07E
:10053000C5FCBAF9003086FB0320DB17C3EBA00033
:1005400080B215F0BBFCBAF9043086FB0320DB1740
:10055000C3EBA00080B215F0B1FC99F80010386828
:10056000F8F7A0FD94F848A11AF0010600F0F7840E
:10057000474B06931B689A0673D5464B464E1B782D
:100580009B0741F15180337D042B8CBF4FF0030A50
:100590004FF0020A472015F0ADFC306815F05AFC08
:1005A000706815F057FC3D4AF3893868A2FB0323B5
:1005B000C3F3471319460493F8F774FD069B99F8A3
:1005C00000101A68049B12F0140F83EA010389F8E3
:1005D000003040F067863389642000FB03F015F09B
:1005E00039FC367D38684AEA8606F6B23146F8F7B5
:1005F00059FD99F8003038685E40314689F800604E
:10060000F8F750FD94F848A1BAF1000F29D1244E13
:100610004F2015F06FFC306815F01CFC706815F069
:1006200019FC504615F016FC01213868F8F73AFD20
:10063000184A99F800301678386806F001063146F5
:1006400083F0010389F80030F8F72CFD99F80030A9
:1006500038685E40314689F80060F8F723FD94F869
:1006600048A1039B0F4AC4F844310AF10103DBB2ED
:10067000A2FB0312D20802EB8202A3EB420384F82E
:100680004831FEF7B1BD00BFDC1F0020676666661B
:100690004C46002050460020544600201F85EB5158
:1006A000FC460020CDCCCCCC30460020CC450020F0
:1006B00094F8A432C24AC4F8A08202EB8302926C7E
:1006C00042B314AD04F2AB23BE4E45F8203D0021E9
:1006D00004F2BD2331800D9380211523A52784F8D2
:1006E000AA32284684F8A91284F8A87290472846AE
:1006F0003188FAF70FF80C9DB34804F52A716D1A8A
:10070000152DA8BF15252A462EF05CFBAF4A94F89C
:10071000A4321570AE4A013382FB0312A2EBE372DE
:1007200002EB42029B1A84F8A432FEF78ABDA94A62
:10073000A94BD4F81411DBF800001B88D77AA74A1C
:10074000401A4FF47A71DEB201FB07F11B0A96776B
:10075000167588424FF00006D37753759670167160
:1007600080F0D1849E4E9F4BD6F800C01B689E4EF1
:100770009E48DFF8989201688068DFF894E286FB73
:100780000376DB17C3EB661303F5FA739BB293761C
:100790001B0AD37689FB0173C917C1EBA30189FB3F
:1007A00000791177C0170912C0EBA90051778E4963
:1007B00082F820000CF5EA43001281FB0C71303303
:1007C00082F821004FEAEC701B12C0EB6110884EDA
:1007D0009EF800E082F823307830864B82F82400BF
:1007E0000CF13001307D03901EF0020F82F82210D0
:1007F000987600F08584D6F800E07F4AD6F804A009
:100800007E48DFF810C282FB0E194FEAEE7182FBC0
:100810000A72C1EBA9514FEAEA79C9EBA25200FB77
:1008200001E900FB02A009EB490900EB40004FEA97
:1008300049094000049207468CFB0920801405906A
:100840008CFB072CF089049A3689079702EB820209
:1008500006F5FA7600EBC00002EB8202B6B204960F
:100860000892059E8200099201EB81014FEAE9722C
:10087000B01A01EB8101624E06910246039906FB14
:100880001292069E40B2052900EB86004FEAE771FE
:100890004FEAAC4C5A4E0590ACEB0100014606FB0A
:1008A0001070089E504FDFF870C14FEADA7A49B2F3
:1008B00001EB86014FEADE7E87FB006983F80EA01C
:1008C00087FB026A099F83F809E0DFF850E13E46A2
:1008D0008EFB066EBCF8006003969DF810605E7596
:1008E000049EBDF814C083F80AC04FEA162689B2E8
:1008F00004964FEAE2724FEAE777424ED973C2EBB1
:100900006A12C7EBAE174FEA1C2A4FEA112E4FEAC4
:10091000E0700399368883F80BA0C0EB691083F868
:1009200010E04FEA22291A739DF810209A754FEAB9
:10093000202CC7F3072A4FEA112134BF4FF0320EA3
:100940004FF0330E9DF80C2083F80D90587483F807
:1009500012C0DF7183F808A0DA74197583F81BE000
:100960001E77C4F81081FEF7BBBBDFF8B490D9F84E
:100970000000F8F783FB00283EF441ACD9F80000F2
:100980000121F8F777FB0222002386F874203B70E0
:10099000FEF735BC94F82C1194F82D3138684A1CB8
:1009A000013384F82C2184F82D31F8F77BFBFEF716
:1009B000FABB154CDFF86C904FF0000A3FE000BF27
:1009C00058150408849B00201081002025810020F8
:1009D00056555555A8430020D4430020489C00207C
:1009E000204600202C4600201F85EB51C8430020E4
:1009F00054460020749C00206BCA5F6B806967FFBF
:100A000040420F0006470020D41F0020676666663C
:100A10005046002083DE1B4304470020D34D621064
:100A2000ECAB0020280000201B2B00F06F820D2B68
:100A300000F04B814FF0010389F801303868F8F776
:100A40002DFB002839D03868F8F720FB83B27E2BC5
:100A5000DBF800202AD099F801100029EED194F893
:100A60002E21002AE0D07D2B00F0368294F83CE164
:100A7000BEF1000F04D080F02003DBB284F83C11FB
:100A8000511CC9B22244092984F82E1182F8303150
:100A900000F016820829D1D8B4F83A21134403EBA8
:100AA000132303F0FF03A4F83A31C7E784F82EA11B
:100AB00084F82FA189F801A0C0E794F83D3133B143
:100AC00094F8313184F83D01302B00F0C18594F861
:100AD0002F21C54BC549DFF850A3DFF850E39146FD
:100AE0004A46002A3EF46FABDBF80020921B012A35
:100AF00024D894F83E21002A40F01E8294F83FC189
:100B000033F81C00F8B94FF0010284F83F210A685D
:100B10009706E5D59AF800209007E1D5B44EB5497F
:100B2000F2894FF4F36303FB02F381FB0321DB172C
:100B3000C3EB61114FF4036015F016FA002384F83B
:100B40002F31FEF740BB0CF1010C5FFA8CFCB0F5C5
:100B5000E06F84F83FC100F098801BD8B0F5047FA7
:100B600000F0238135D8B0F5887F00F0CD80B0F556
:100B7000007F00F0B380B0F5807FB1D10A685207E2
:100B8000AED59D4B196815F0EFF9002384F82F318D
:100B9000FEF719BBB0F5026F00F05A816AD8B0F5C4
:100BA000E46F00F08180B0F5006F00F0D680B0F502
:100BB000E26F95D1914BDA6B998A642303FB02F3C0
:100BC00093FBF1F115F0D0F9002384F82F31FEF7F3
:100BD000FABAB0F5826F00F05181B0F5C06F00F045
:100BE0002781B0F5806F7FF47BAF94F840310133FB
:100BF000DBB2032B00F2AD8142F2107184F8403178
:100C000001FB03F17E4B1B88002B40F0A0810131DA
:100C10007C4B1B78DB077C4B1B8848BF0431DF070C
:100C200048BF0A31980748BF14311A0648BF283117
:100C3000DF0548BF2831580748BF64311A0748BF4D
:100C4000C8319F0548BF01F5C871980648BF01F536
:100C50007A71DA0648BF01F5FA615F0648BF01F50F
:100C60007A614FF4806015F07FF9002384F82F310A
:100C7000FEF7A9BAB0F5046F1AD0B0F5116F52D0D3
:100C8000B0F5036F7FF42CAF41E75C4B91469A6B54
:100C9000998A642303FB02F393FBF1F115F064F9E5
:100CA00084F82F91FEF78FBA544B91461A6CEFE7F8
:100CB000564BB3F9041001EB81019146490015F040
:100CC00053F984F82F91FEF77EBA4FF0010184F8B2
:100CD0002E1184F83031A4F83A21AFE69EF80620B0
:100CE000002A3FF4FDAE4A4B4A491B6881FB0321B1
:100CF000DB17C3EBA1014FF4007015F035F90023A9
:100D000084F82F31FEF75FBA0A6852077FF5E8AE24
:100D1000414B4FF48870196815F026F9002384F8C8
:100D20002F31FEF750BA9EF80520002A3FF4D8AEC6
:100D30003A4A107800283FF4D3AE394B1B8803EBB6
:100D40008303590091FBF0F14FF4116015F00CF999
:100D5000002384F82F31FEF736BA0A6897067FF52C
:100D6000BFAE9AF8002090077FF5BAAE1CF0010FD5
:100D70001F4E204900F05C84726882EAE273A3EBA4
:100D8000E27303EB5303A1FB0331C908002AACBF94
:100D900041F0004141F040414FF4006015F0E4F8AB
:100DA000002384F82F31FEF70EBA9EF80520002AA2
:100DB0003FF496AE194A107800283FF491AE194BD3
:100DC0005B7B002B00F09484154B1B8893FBF0F0A9
:100DD00000EB800041004FF4047015F0C5F80023CB
:100DE00084F82F31FEF7EFB9581504084C4600205F
:100DF000544600201F85EB512C460020D84500208A
:100E0000789B0020C18600204A9B002030460020AD
:100E1000C843002067666666204600200B44002019
:100E2000D4430020A843002050460020384600202C
:100E30009EF80620002A3FF453AEC34B4FF4C06027
:100E4000996815F091F8002384F82F31FEF7BBB9AB
:100E50000F68BF067FF544AE9AF800C01CF0020F81
:100E60003FF43EAEB94E33896421914601FB03F154
:100E700015F07AF884F82F91FEF7A5B90A68900664
:100E800040F1F180B24BB14E1878317D00F0020391
:100E9000002B0CBF00234FF47A7340F6B83208BF22
:100EA0004FF4FA6210F0010F18BF134619444FF4C3
:100EB000826015F059F8002384F82F31FEF783B9CA
:100EC000B4F83A21C2F1FF0293427FF4B3AD4FF080
:100ED000010384F83D31ADE54FF0010384F83C3166
:100EE000ACE5FDF755FE9B4B1B68C01A40F6B833C6
:100EF000984200F21E81DFF89CA29AF804303A2B47
:100F000000F0BA8200233B70FEF779B93868F8F731
:100F1000C5F800287FF48EAD4FF0010384F82F311F
:100F20008CE5C4F8203184F818318B4F15F06AF83D
:100F300094F82431FEF71DB98849062014F0E6FD27
:100F4000002384F83E0184F82F31FEF73CB90231CA
:100F50005EE6012384F8403142F2107152E6804B84
:100F60001B88D80513D4D90600F17A839A0600F1BC
:100F7000F183580600F1F383190700F1F983DA07CA
:100F800000F1148413F0020F0CBF04260C26754BDD
:100F9000754A1B78D27803F001030AB143F00203CB
:100FA0005320049314F0A6FF704A128802EB8202C9
:100FB00002EB8202900080B214F080FF002014F057
:100FC0007DFF6B4A6B4912883868C2EBC21252002F
:100FD00081FB023111444FEAE27ACAEB612A5FFADF
:100FE0008AFA5146F8F75EF899F80020049B3868B1
:100FF0001E438AEA020A002189F800A0F8F752F895
:1010000031463868F8F74EF899F800303868734080
:10101000DBB2194689F80030F8F744F894F848A193
:10102000FFF7F2BA013B84F85631FEF717BB013BDC
:1010300084F85731FEF72BBC09F1FF3984F85F9132
:10104000FFF760BA013F84F85E71FEF7FDBF013B18
:1010500084F85A31FEF713BF47493A2014F056FD81
:101060002870FEF7E2B8454A1268120600F1FA82CB
:10107000434A127B002A3FF433AD94F8411103290F
:1010800000F28A83DFE801F0322819023D4B1B6829
:1010900059799A79DB7901F1407101EB022101EB79
:1010A0000341002384F841314FF4826014F05CFF67
:1010B000002384F82F31FEF786B8334B1A68137A71
:1010C000507992781B0403EB002313444A1C84F8E4
:1010D000412103EB0161E7E72B4B1A68D3791079C3
:1010E00052781B0403EB00231344EFE7264B1A68E6
:1010F0009379D07812781B0403EB00231344E5E7BF
:101100002D22DA762DE4214BDBF800101B78C4F891
:101110001411013B012B3FF625AB102102239170E6
:101120001371FFF71FBB14F05DFF01233370FDF750
:10113000F3BF174AB2F84A3100210133A2F84A310D
:101140003970FEF75CB800BFC84300205446002049
:10115000504600206CAB0020D0450020615F0208A3
:101160004A9B0020C1860020549B0020D4430020CD
:10117000489B002003082080915403089C630020B2
:10118000A8430020244A0020949F0020509B002068
:10119000D41F002054AB0020A64EA74B0093002480
:1011A000A6F13F01A54BA64A0A9106F8404CA54975
:1011B0000B960CA8F9F786FB0A9E731C0A933470F1
:1011C0000A9B2922591C0A911A700A9BEA22591C6F
:1011D0000A911A700A9BC822591C0A910CA81A700D
:1011E0002DF04CF8471C0CA93A460A982DF0EAFD60
:1011F0000A9AD31901330A93D4550A9B5A1C0A92AE
:101200001C700A9B5A1C0A921C700A9B5A1C0A9258
:101210001C700A9B5A1C0A921C700A9B5A1C0A9248
:101220001C700A9B5A1C0A921C700A9B5A1C0A9238
:101230001C700A9B5A1C0A921C700A9B5A1C0A9228
:101240001C700A9B5A1C0A921C700A9B5A1C0A9218
:101250001C700A9BFF22591C0A911A700A9B0122DA
:10126000991814A80A911A7050F8283D9B1B3370E6
:1012700024F0DEF82C70FDF7D8BF8C46894608466E
:1012800004910591069107910B46FEF719BA9FED5F
:101290006E7A13F0140F08BFF0EE477A7EF4F0AECA
:1012A000FEF7F7BE694B1868FFF799B9684A614BBA
:1012B00012680D93A3F14007002103F8401C21237D
:1012C000D100BB7040F13A8262490326624B1B8811
:1012D0005A0500F12982D80700F13E8203F002038B
:1012E0005E4A002B1CBF03261146DFF88891324668
:1012F00048462DF067FD06EB090314A80133A9F158
:10130000020140F8203D00225B1A06F809207B709C
:1013100024F08EF8FEF742B8C4F81C8186F80090DD
:10132000FDF7FABE434A4E4B0D9214AEA2F13D00BA
:1013300046F8200D19884B4FA2F1400300204FF0D2
:101340000A0E02F8400C082283F801E030469A7039
:10135000F9F7BAF93B684449DA1781FB0313C2EB8A
:10136000A30399B23046F9F7AFF90BF057FDBF6808
:101370000C9B3A0C591C0C911A700C9B3A0A591C84
:101380000C911A700C9B5A1C0C921F700C9B5A1CCF
:101390000C921870304624F04BF8FDF7FCBF334F29
:1013A0009FED338AB7F9022022480D9007EE902A6C
:1013B000F8EEE77A14AE67EE887AA0F13D01FDEE13
:1013C000E77A46F8201D00F8403C0823CDED037A6B
:1013D00000F83F3C1E23BDF80C1000F83E3C3046A0
:1013E000F9F772F9B7F9003007EE903AF8EEE77ABC
:1013F000304667EE887AFDEEE77ACDED037ABDF8E8
:101400000C10F9F761F9B7F9043007EE903AF8EEED
:10141000E77A304667EE887AFDEEE77ACDED037A1B
:10142000BDF80C10F9F750F9304624F001F8FDF73B
:10143000AFBF00BFC89B00208B9F0020C04804089E
:10144000C8480408D4480408000000002C460020C6
:10145000F4870020AC4804084A9B0020BC480408DC
:10146000D4430020C84300206766666630460020EB
:1014700058A08B418B9B00209AF80240C4B1013CDC
:10148000E4B2013454445146002211F8013B534068
:1014900083EA0313DBB2120ADE0042EA03228C4223
:1014A00086EA131382EA0302EFD1002A7FF42AAD01
:1014B000C04AC14EC14B1288C149C24CF261DFF82B
:1014C00038931A6809689B68F262B4F84A21F0669A
:1014D000F364D9F80000F163F265F6F74DFE03906E
:1014E00000287DF487AE0221D9F80000F7F7C2FD8D
:1014F00094F84C319AF803200492642B4FF00402C4
:1015000086F8742040F07C8194F84D31072B04BF9D
:101510009DF80C3084F84D3194F84D31079306EB6B
:10152000031ADAF80410039108462CF0A7FEDAF843
:10153000081006915FFA80FA08462CF09FFEC0B2B0
:1015400005900AEB0002079B9F480399039008321D
:10155000C27123F00F0286468272059803F00F03D2
:1015600000EBCA008EF80D3052468EF80E000EF1D8
:101570000F002DF027FC954B059A06990AF10900FA
:1015800018442DF01FFC0398C37903F1010ACBB175
:10159000013B5FFA83FC0CF1080CDFF860E2844445
:1015A0000023073010F8011B59408B00CA0883EA5A
:1015B000410302F018024B404EFA02F253408445B8
:1015C000DBB2EFD1814A04980AF8023018F06AFDC4
:1015D00094F84D310022013384F84D3184F84C21C8
:1015E000039BDDF80CA09B785BB11AF80510D9F8C5
:1015F0000000F7F757FD01359AF80230EDB2AB4223
:10160000F3D894F84C310322013384F84C3186F836
:1016100074203A70FFF7ABB902213868F7F72AFD5A
:1016200094F82431FDF7A5BD4FF0010AFEF7B2BFD3
:10163000326882EAE273A3EBE27303EB5303A1FB8C
:101640000331C908002AB8BF41F08041FFF7A4BBAD
:101650005F49881F14F0FEFA84F83E01FFF737BA9D
:10166000342694E410230026042218460CA98DF891
:1016700030308DF831208DF832608DF833608DF880
:1016800034608DF8356014F04FFC84F82F61FDF75D
:101690009ABD4B4B1E6806EB86067600FEF7EFB947
:1016A0004C4AD278002A0CBF4FF0040C4FF0050CC6
:1016B000FEF710BE012338683370F7F7E7FC0646E3
:1016C0003868F7F7E3FC72067DF426AD8A2851D01E
:1016D0008E287DF421AD94F81831002B7DF438ADBF
:1016E0003D4BC4F820312D2384F82431FDF71BBD78
:1016F000304B1888FFF76CBB0127FEF7E1B82D4986
:101700009A790B8803EB830303EB83039F00BFB23B
:10171000002A00F01181294B1B680FFA83FA0BF0A5
:101720007DFB40B2FDF7E0BE03262C49DDE59C467B
:101730009946184604930593FDF7C2BF284B294AE2
:101740001B68294903F48003002B16BF11460426A9
:101750000326BBE524261AE424490426C5E5102601
:1017600015E4138907EE903AF8EE677AFEF791BC1C
:1017700020260CE41E4B1B689B067DF5CDAC94F82F
:101780001831002B7DF4E4AC1A4BC4F820312D2322
:1017900084F82431FDF7C7BC4B1CDBB2042B84F862
:1017A00041314FEA01613FF47CAC7DE40826FFF74C
:1017B000EEBB00BFD443002028000020C843002017
:1017C0002C460020D41F0020A45A0020AA5A002032
:1017D0000C210020549B0020489C0020B0480408A5
:1017E0009C630020AC480408A4480408B4480408DA
:1017F0004C460020749C0020ECAB00200007090E32
:1018000096F875A0574905951AF00F0F04BF0AF115
:10181000010A5FFA8AFABAF1070F28BF4FF0010AEE
:101820004FEA0A1C06EB0C03187C4F4B03930A1873
:10183000002392F824104C4A93725FFA8CF31A46F4
:101840004A4B964606EB0C024EEA0000012918703E
:10185000D26803F101000CD90239C9B28D1C1D44B4
:10186000034603F8012BAB424FEA1222F9D10131B2
:101870000844B44422F060030AF1010A9CF81120E4
:101880005FFA8AFA1343BAF1080F037000F10103FB
:1018900040D04FEA0A1C06EB0C01344A087C31495F
:1018A00001449A1A91F8241055180EF1100E132DB8
:1018B0005FFA8EFEC6DD059D0398DFF8BCE0D2B26C
:1018C000931DDBB243F04001C17103F1010CCBB1B8
:1018D0000532D3B20833C31805930EF1010000237B
:1018E00010F8011B59408B0083EA4103CA084B40A2
:1018F0001F4902F0180241FA02F25340059A82424F
:10190000DBB2EDD104980CF80E3086F875A018F013
:10191000C9FB65E6154A059D9A1ACDE7154B64206B
:10192000B3F900A0FDF7E0BD9C4699461846049324
:1019300005930693FDF7C4BE4FF0FF33EDE69C46DA
:10194000FDF7BEBE9C469946FDF7BABE9C46994639
:101950001846FDF7B5BE9C46994618460493FDF718
:10196000AFBE00BF58150408A45A0020B15A002089
:101970000007090EC8430020AA5A00202DE9F04FA5
:1019800095B0B0F908500D81EDB2442D00AF0C4672
:10199000904600F04984064643D9812D00F08183AA
:1019A00000F29980542D00F0CD8040F2D7806E2D4A
:1019B00000F00884802D40F0D480774B93F800A08D
:1019C0000AF1020A1AF0FF0A00F09880734BDFF860
:1019D000FC81734EDFF8F8B19A4403F101090A253E
:1019E00016E0322D01F0F982A5F13C00C0B21328B7
:1019F00041F2FA8200232268511C2160157022688E
:101A0000D14502F101012160137077D019F8015B13
:101A10000A2DE6D1BBF80030FF2BA8BFFF23DBB2B5
:101A2000E9E7052D00F0EE8321D8022D00F0828039
:101A300040F21683032D00F0BB83042D40F091800B
:101A4000584920462A46F8F71DFE574B204619787C
:101A5000F8F760FE22680021531C01252360284608
:101A60002B46543711706381BD46BDE8F08F242D9D
:101A70005ED040F2AB82282D00F05C83382D70D10F
:101A80000A684A4B0125511C216015702268052106
:101A900050192060117022680A21501920601170BD
:101AA000226800215019206011702268197850199D
:101AB00020601170226859785019206011702268D6
:101AC0009978531923602B46117028465437638147
:101AD000BD46BDE8F08FA02D18D040F29682B82DFB
:101AE00000F06483FE2D3CD1314D05F1080635F838
:101AF000021B2046F8F70EFEB542F8D101252B4611
:101B0000284654376381BD46BDE8F08F294B08460F
:101B10001968F8F7E7FD284B20461968F8F7E2FD49
:101B2000264B196820460125F8F7DCFD2B46E7E730
:101B3000234BF6E70422234920460125F8F7A2FDAE
:101B40002B46C2E70B6800215A1C226019702268DC
:101B50000125531923602B461170B6E7522D3FF42F
:101B600079AF21462846FAF7C3FD03460028C5D1C0
:101B7000742D00F08882772D2CD1326871689142E3
:101B80001EBF531C336011780F4A08BF1946204608
:101B90002BF026FFB2E700BF11430020AC1504086C
:101BA000582600208B9F0020E5380020D98A00208D
:101BB00034430020107AFF1F147AFF1F187AFF1F8A
:101BC000248C00204049040849CF030867666666F4
:101BD00080260020F52D01F05F83762D00F02C8308
:101BE000472D01F09682292D336801F07982392D35
:101BF00001F02D82212D01F03D8271680B3DCA1A42
:101C0000EF2D00F2F98301A050F825F0492F0108CB
:101C1000F9230108F9230108F9230108F923010830
:101C2000F9230108F9230108F9230108F923010820
:101C3000F9230108F9230108F9230108F923010810
:101C4000F9230108F9230108F9230108F923010800
:101C5000F9230108F9230108F9230108F9230108F0
:101C6000F9230108F9230108F9230108812F01084C
:101C7000F9230108272F0108F9230108FD2E010887
:101C8000F9230108F9230108F9230108D52E0108D9
:101C9000F92301085F2E0108F92301082D2E010800
:101CA000F9230108072E0108F9230108F52D010881
:101CB000F92301089D2D0108F92301081D2D0108B4
:101CC000F9230108F9230108F9230108F923010880
:101CD000FD1A0108F9230108C72C0108F92301089E
:101CE000F9230108AD2C0108F9230108532C010840
:101CF000F9230108F9230108F9230108F923010850
:101D0000472C0108F9230108F9230108F9230108E8
:101D1000072C0108F92301087B2B0108F92301088E
:101D2000F9230108C92B0108F9230108F923010847
:101D3000F9230108F9230108F9230108F92301080F
:101D4000F9230108A72A0108F9230108252A010817
:101D5000F92301082F290108F92301088128010826
:101D6000F9230108592801083B280108F923010833
:101D7000F9230108F9230108F9230108F9230108CF
:101D8000F9230108F9230108F9230108F9230108BF
:101D9000F9230108F9230108F9230108F9230108AF
:101DA000F9230108F9230108F9230108F92301089F
:101DB000F9230108F9230108F9230108F92301088F
:101DC000F9230108F9230108F9230108F92301087F
:101DD000F9230108F9230108F9230108F92301086F
:101DE000F9230108F9230108F9230108F92301085F
:101DF000F9230108F9230108F9230108F92301084F
:101E0000F9230108F9230108F9230108F92301083E
:101E1000F9230108F9230108F9230108F92301082E
:101E2000F9230108F9230108F9230108F92301081E
:101E3000F9230108F9230108F9230108F92301080E
:101E4000F9230108F9230108F9230108F9230108FE
:101E5000F9230108F9230108F9230108F9230108EE
:101E6000F9230108F9230108F9230108F9230108DE
:101E7000F9230108F9230108F9230108F9230108CE
:101E8000F9230108F9230108F9230108F9230108BE
:101E9000F9230108F9230108F9230108F9230108AE
:101EA000F9230108F9230108F9230108F92301089E
:101EB000F9230108F9230108F92301081128010871
:101EC000F9230108F5270108F9230108F92301087E
:101ED000F9230108F9230108F9230108F92301086E
:101EE000F9230108F9230108F9230108F92301085E
:101EF000F9230108F9230108F9230108F92301084E
:101F0000972701080F270108D7260108F9230108A0
:101F100035260108C92501087B270108F923010896
:101F2000612701085D2501083525010823250108E1
:101F3000C7240108F923010897240108F92301089F
:101F4000F92301086D2401083F2401082B2401080E
:101F500003240108DB230108B123010885230108BC
:101F60006D230108F9230108F9230108F923010869
:101F7000F9230108F9230108F9230108F9230108CD
:101F8000F9230108F9230108F9230108F9230108BD
:101F9000F9230108F9230108F92301084D23010859
:101FA000F9230108F9230108F5220108F9230108A2
:101FB000F9230108F9230108F9230108F92301088D
:101FC000F9230108F923010889220108202D7FF453
:101FD000C8AD0B68B24D591C6A7821601A7023682D
:101FE0002A78591C21601A702368AA78591C21602C
:101FF0001A7029892046F8F78DFB23686A79591CE5
:1020000021601A702268A97926E5822D7FF4A9AD96
:102010000B68A44AA44D1178A14A581C206019707D
:1020200011892046F8F776FBA04B22681B88FF2B0E
:1020300002F10101A8BFFF2321601370A96881F399
:10204000100189B22046F8F765FB296801F30F01FA
:1020500089B22046F8F75EFB954B22681978FBE4BD
:10206000012D7FF47EAD0B680022591C21601A708F
:1020700023685A1C22601D7022682421531C23608F
:102080002B46117021E53268716891421EBF531CC6
:1020900033601178874A08BF194620462BF0A0FC10
:1020A0002CE5854B1E78033616F0FF063FF426AD6F
:1020B000824BDFF838821E4403F1010A4FF00A090F
:1020C00020E0B9F1500F00F08587B9F1320F00F030
:1020D000A187A9F13C00C0B2132840F29F870025D8
:1020E000294623685A1C2260204683F80090F8F79E
:1020F00011FB29462046F8F70DFB56453FF4FEAC90
:102100001AF8019BB9F10A0FDBD16D4B9D68196874
:1021100005EB85054FF6FF736D009D42A8BF1D4678
:102120009942A8BF194625EAE57521EAE171ADB2E9
:1021300089B2D6E70B68DFF8B891624E591C0222CB
:1021400021601A7023684FF006085A1C226083F839
:10215000008023680A22591C21601A702368012517
:102160005A1922601D70B9F800102046F8F7D2FA0B
:10217000B9F802102046F8F7CDFA23685A19226000
:1021800083F8008023685022591921601A7023684F
:102190000022591921601A7031882046F8F7BAFADE
:1021A00071882046F8F7B6FA2B468EE4464BB8E421
:1021B0000B685A1C0A601D700B680222591C2160B2
:1021C0001A7047E4394B0A681B88374DFF2BA8BFAC
:1021D000FF23511C21601370A96881F3100189B29B
:1021E0002046F8F797FA394B20461988F8F792FA03
:1021F000296801F30F0189B220460125F8F78AFA10
:102200002B4662E40B2232492046F8F73BFA0822BB
:1022100030492046F8F736FA012507222E49204694
:10222000F8F730FA2B4650E4002A3FF467AC2B4B0A
:10223000136001252B4648E43268511C3160127846
:10224000002A01F00E81102A07BF254B93E84200B7
:102250001E46314625686B1C236020462A70F8F71D
:1022600041FA31462046F8F73DFA1E4B20461968E0
:10227000F8F738FA20460021F8F74CFA00212046FA
:10228000F8F748FAFFF7E6BB174B1B78DB0700F1BE
:10229000B3800125FBF7FCFAFCF77EF92B4614E42A
:1022A000384600200B440020C8430020D4430020BF
:1022B000509B002081D8030811430020BC1504085E
:1022C0000C26002040260020AC3B0020489B00202C
:1022D00048490408544904086049040821C6000814
:1022E00084230020B0230020C18600205026002037
:1022F0009C8900205A1C32601A780F2A7CD8991CBD
:102300003160C2EBC202B74958788854D81C30609B
:102310000A4499785170191D3160D9789170591D0E
:1023200031601979D170991D316059791171D91DB8
:1023300031609979517103F108013160DB79937152
:10234000012529F0F9FB2B46FFF7BFBB3046F8F714
:1023500087F9DFF8A082A8F80E003046F8F780F978
:102360000125A8F80C002B46FFF7AFBB3046F8F765
:1023700077F99D4A00EB80004300012513802B462E
:10238000FFF7A3BB19465A1C3260984A11F8020B9A
:102390001070316059785170D91C31609978917002
:1023A000191D3160DB78D37001252B46FFF78DBBFB
:1023B0003046F8F755F9DFF86C82A8F8100030467F
:1023C000F8F74EF9A8F812003046F8F749F9012558
:1023D000A8F814002B46FFF778BB1A46591C316049
:1023E00012F8020B3260DA1C597832609A7823F0C6
:1023F000F1FB00287FF482AB4FF0FF352B46FFF74F
:1024000064BB1A46591C3160794912F8020B0870F6
:10241000326078495A788A70DA1C3260724A9B7846
:10242000937001252B46FFF750BB734B7349186817
:102430004E2201252CF0C6FC2B46FFF746BB194661
:102440005A1C32606E4A11F8020B107031605978D4
:102450005170D91C31609B7893703046F8F700F9C1
:10246000684B0125D8802B46FFF72FBB3046F8F785
:10247000F7F8DFF89081A8F800003046F8F7F0F898
:10248000A8F802003046F8F7EBF80125A8F8040098
:102490002B46FFF71ABBDFF8909199F80030002B1C
:1024A0003FF42CABDFF8848100253046F8F7D8F8EC
:1024B00010F050FB99F80030A8EC010A01359D425C
:1024C000F3DBFFF71BBB0D2A96D15A1C32601D7837
:1024D000072D91D8DFF8589130464FF00C08F8F7E7
:1024E000BFF808FB05F809EB0805A8803046F8F7A7
:1024F000B7F8E8803046F8F7B3F8336828811A4611
:10250000591C316012F8021BA97232605B78EB72C1
:102510003046F8F78DF8012549F808002B46FFF7FB
:10252000D4BA3046F8F79CF8374B012518802B4673
:10253000FFF7CBBA5A1C32601878060600F1E5871F
:10254000324B1B78DD073FF5D9AA032828BF0020AE
:102550000125FBF781F92B46FFF7B7BA5A1C326009
:10256000304693F800A0F8F763F881463046F8F754
:102570005FF805463046F8F75BF880463046F8F7D6
:102580006FF83046F8F76CF83046F8F775F8BAF19E
:10259000000F00F0C587BAF1100F7FF4AFAA1C4BF3
:1025A000C3F800905D60B8F1000F02D0194BC3F87A
:1025B00000801949194B0222081F01251A7025F0C5
:1025C00033FF2B46FFF781BA104B1B78D9073FF535
:1025D00095AA134B4FF4C87201251A802B46FFF7BA
:1025E00074BA00BF90AD0020BC890020D447002001
:1025F00078630020AC890020949F0020F42D04080B
:10260000A4890020903D0020D0470020C1860020F2
:1026100084230020B023002088230020BA46002015
:10262000444A00204860002011430020E83C00207C
:10263000B8B30020092A7FF7DFAEDFF8DC831A4643
:10264000591CD8F80050316012F8021B2970326012
:102650005A78AA70DA1C32609A78642A03F104016D
:10266000A8BF64226A713160DA78642A03F1050137
:10267000A8BF6422AA7131601A79EA719A1D32608A
:102680005A79642A03F10701A8BF64222A723160D3
:102690009A79EA7003F108023260DB792B713046D7
:1026A000F7F7DEFF726833686881D11A00290CDD04
:1026B000591CD8F800003160521A002A197841726A
:1026C00003DD9A1C32605B784370012516F00CFF25
:1026D0002B46FFF7FAB9C44A1068DA1C01462133C9
:1026E000951E356012F8035C0D70551E356012F8AA
:1026F000025C4D70326012F8015C8D7003329342BF
:1027000001F10301ECD129F005FEFFF7F7B95A1CDE
:1027100032601A78B549002A00F019870A7842F029
:102720000202981C0A70B24D30605B782B753046FF
:10273000F7F77EFF28603046F7F77AFF686030468B
:10274000F7F78EFF28813046F7F78AFFA94AE8811C
:102750001378012543F0020313702B46FFF7B5B938
:10276000A54B1B78D8073FF5C9A90125FBF76CF9E4
:10277000FBF712FF2B46FFF7A8B99F4B1B78DA0730
:102780003FF5BCA9994A1378012543F0040313705F
:102790002B46FFF79AB9C2F34705122D3FF62CAE30
:1027A000C5B107F1500307F12A0903EB450AC846F2
:1027B000AAF1260A3046F7F753FF28F8020FC24560
:1027C000F8D18E4B39F8022F23F8022FC845F9D1E2
:1027D000112D09D88A4A6B00023B13440021223292
:1027E00023F8021F9A42FBD1864A01231D4613702B
:1027F000FFF76BB9DFF8248200233046C8F80030B9
:10280000F7F716FF0125C8F800002B46FFF75DB962
:102810001A46591C316012F8025B3260DA1C587893
:1028200032609978002D00F0C486012D7FF466A9EE
:102830000AF0C4FA2B46FFF748B96F4A127812F033
:1028400001017FF4D9AD5A1C3260187801250AF0D5
:10285000F7F92B46FFF739B91A46591C31606A4916
:1028600012F8020BC870326068495A784A71DA1C53
:102870003260674A9B78D37001252B46FFF725B954
:102880003046F7F7EDFE3046F7F7EAFE3046F7F749
:10289000E7FE3046F7F7F0FE3368534D1946581CF3
:1028A0002A68306011F8020B82F82C0031605978E8
:1028B00082F83610D91C31609B7882F83730304668
:1028C000F7F7DAFE3046F7F7D7FE3046F7F7D4FED3
:1028D0003046D5F80080F7F7C3FEA8F83A00304636
:1028E000D5F80080F7F7BCFE33687268A8F83800A6
:1028F000D11A01290ADD591C2A6831601B7882F837
:102900002E303046F7F7B8FE33687268D31A032BBF
:102910000BDD3046D5F80080F7F7A2FEA8F83200AC
:1029200030462E68F7F79CFEB0862868EBE65A1C06
:1029300032602D4DDFF8E8801B7888F8053030468E
:10294000D5F80090F7F78CFEA9F820003046D5F8AE
:102950000090F7F785FE72683368A9F81E00D11A57
:10296000072919DD3046F7F77BFEA8F80A00304644
:10297000F7F776FEA8F80C003046D5F80090F7F788
:102980006FFEA9F822003046D5F80090F7F768FEF0
:1029900033687268A9F82400D11A03290BDD304688
:1029A000F7F75EFEA8F80E003046F7F759FE3368D9
:1029B0007268A8F81000D21A002A05DD591C2A688E
:1029C00031601B7882F82630FAF76CFF1AF0AEFA05
:1029D000104B1B68002B00F0E1852868012529F0C9
:1029E0003FF92B46FFF771B8949F00205046002016
:1029F00054460020B8460020C186002072AA00205C
:102A000074AA002098AA0020AC890020BC9D002058
:102A1000BC890020D0890020244A0020AC3B002043
:102A2000786300201A46591C3160DFF8E48212F8FE
:102A3000021B88F802103260AA495A780A70DA1C20
:102A40003260A94D9A782A711A1D3260DB78092B01
:102A5000A8BF09233046AB70F7F702FE33687268EF
:102A60002880D11A012905DD3046F7F7F9FD3368D2
:102A70007268E8819A4207D05A1C32601B78003392
:102A800018BF012388F80730FAF70CFF3368726823
:102A90009A423FF433A85A1C32601B78EB70012530
:102AA0002B46FFF712B83046F7F7DAFD054625F05A
:102AB000C9FDFF283FF422A83F2D00F20F8507F142
:102AC0005008002308F8243D4FEAD509414607F194
:102AD0002B0087F82B3009F1010925F093FD97F8B9
:102AE0002B305FFA89F905F007054B4505F1010523
:102AF00003D197F82C30AB4203D02946484625F045
:102B00008DFD33687268D21A012A7EF7F7AF5A1C1E
:102B100007F15000326000221D7800F8252D25F0C5
:102B200065FD97F82B30AB420AD0704B1B683BB168
:102B30009A79AA4204D31B681B690BB128469847AF
:102B400033685A1C3260404600221D7887F82C20DA
:102B500025F040FD97F82C30AB423EF4CFAF634BED
:102B60001B68002B3EF4CAAF1B685B69002B3EF468
:102B7000C5AF28469847FEF7C1BF5A1C326093F88C
:102B80000080B8F1110F3FF637AC9A1C3260584DF7
:102B90005B7805F818303046F7F762FD40F6CA0357
:102BA0009842A8BF184640F2EE23984205EB480130
:102BB000B8BF18460125A0F2EE222B46192092FB41
:102BC000F0F24A70FEF781BF4A4A1278012A3EF6B7
:102BD00095AF18465A1C3260DFF8388110F8022B86
:102BE00088F80220DA1C891A30600129587832608E
:102BF00040F3E5843046F7F733FD0125A8F80000DF
:102C00002B46FEF762BF1A46591C3B4D316012F845
:102C1000021B297132605B786B713046F7F720FD3B
:102C2000336828805A1C32601B78AB713046F7F746
:102C300017FD336868805A1C32601B78EB710125E0
:102C40002B46FEF742BF0125F8F7C2FB2B46FEF7E5
:102C50003CBF5A1C3260294A1B78DFF8BC801370D5
:102C60000023C8F800303046F7F7E2FC3368D8F8A4
:102C700000202349234D10435A1CC8F8000032603D
:102C80001B780B723046F7F7EBFC28603046F7F7FD
:102C9000E7FC68603046F7F7E3FCA8603046F7F7DA
:102CA000DFFC3046F7F7DCFCFEF728BF164A03F1DD
:102CB00008010133336013F8010C02F8010F8B4255
:102CC000F7D1FEF71BBF591C1A4631600F4912F8A5
:102CD000020B887032605B784B7001252B46FEF743
:102CE000F4BE00BFA089002048600020C89F0020DB
:102CF0003CAC0020078C0020AC3D0020D489002093
:102D0000146500208839002013650020C889002040
:102D1000786300200A8C0020248C00200721B2FB5D
:102D2000F1F1C1EBC105521B7FF466ABC9B201F1F1
:102D3000FF395FFA89F900293EF4E0AE09F1010993
:102D400015465A1C326093F900A0504611F034FE2B
:102D50000135804600283FF44FAB80F802A0304692
:102D6000F7F77EFC3268A8F800001346511C31606A
:102D700013F8021B88F803103360537888F8043086
:102D8000D31C3360937888F80630131D3360D278F3
:102D900088F80520A945D4D1FEF7B0BE5A1C326090
:102DA0001A780E2A3FF628AB991C31605D78032D06
:102DB0003FF622ABBF48062101FB02F1421803F1A6
:102DC000030E5571C6F800E09D784554191D316019
:102DD000D9785170591D316019799170991D316000
:102DE0005979D170D91D31609B79137101252B461A
:102DF000FEF76BBE5A1C3260AF4A1B785375012533
:102E00002B46FEF762BE591C31601D781F2D3FF620
:102E1000F3AA052A7FF4F0AA3046F7F709FCA74B7E
:102E200043F8250015F010F8FEF768BEA34D05F134
:102E300040083046F7F714FC3368A5F88000591CA9
:102E40001A46316012F8021B85F8821032605B78F6
:102E500085F883300435A845EBD1FEF74FBE5A1CE8
:102E60003260954D1B782B723046F7F7F9FBA8833B
:102E70003046F7F7F5FB28833046F7F7F1FB326869
:102E80006883531C33601278EA747268D31A032B78
:102E900000F365833368D11A05290EDD5A1C3260B0
:102EA0001B78EB723046F7F7C3FB3368E8605A1CB7
:102EB00032601B782B7433687268D21A002A7EF74E
:102EC0001DAE5A1C32601B7885F8213001252B4637
:102ED000FEF7FBBD581C3060794A1D781570091A41
:102EE00000297EF70BAE991C31605B78003318BF68
:102EF0000123012553702B46FEF7E7BD3046F7F757
:102F0000AFFBDFF8D481C8F800003046F7F7A8FB24
:102F1000C8F804003046F7F7A3FB0125C8F80800FD
:102F20002B46FEF7D2BDDFF8B4810023C8F800308D
:102F30003046F7F77DFBD8F8003001250343C8F889
:102F400000302B46FEF7C1BD5E49102A13464FF0F4
:102F5000000228BF10230A604A608A60CA600A74AF
:102F6000002B3EF4CBAD326801391344013232609C
:102F700012F8010C01F8010F9A42F7D1FEF7BEBD1D
:102F80005A1C32601D78132D3FF636AA9A1C326007
:102F900058787B622AF05EFD00283FF42DAA7B6AF8
:102FA000494A017802F82510D91C316002EB8502EC
:102FB00099785170191D3160D8789070581D306023
:102FC00042491B79D3700868012516F01BFA2B467D
:102FD000FEF77BBD3E4BFFF799B83388FF2BA8BFA8
:102FE000FF23DBB2FEF707BD12F090FC00283EF491
:102FF00001AD03780A2B28D8B0F9023088FB031200
:10300000DB17C3EBA2039BB2FF2BA8BFFF23DBB2EE
:10301000FEF7F1BC98E82200FFF77AB812F076FCD0
:1030200000283FF45CA803780A2B3FF658A8B0F9B3
:103030000430B0F9061003EB830383F3500521EA53
:10304000E171ADB289B2FFF74CB80023DFE75A1C3B
:1030500032601A780A2A00F0D5813046F7F70CFB67
:103060003046F7F709FB01253046F7F705FB2B46FD
:10307000FEF72BBD1A46591C3160164D12F8021B83
:10308000697032605A782A70DA1C32609B78AB70B3
:103090003046F7F7E5FA33682881591C1A46316043
:1030A00012F8021B697132605B78AB7101252B4607
:1030B000FEF70BBDB83B002014650020189A0020D5
:1030C000D489002088890020D8890020949F00207E
:1030D000442600203846002088390020248C002017
:1030E0005A1C32601B780A2B00F08681502B7FF42B
:1030F000D5AD3046F7F7B4FADFF84083A8F8000002
:103100003046F7F7ADFA0125A8F802002B46FEF786
:10311000DCBC726835687B623046551BF7F788FA6D
:10312000052D38627B6A00F25B818026B34601255B
:1031300094E80600521A103AB242B8BF1FFA82FB56
:10314000B84A396A92683A61521A9345396A7B6281
:103150002046FA6088BF1FFA82FBF7F7C3FA7B6A42
:10316000002B00F01C81002D40F0F3802368C7F88D
:1031700000D05D71C0B00533C7F808D0FB61BBF16A
:10318000000F00F0A7813B6A3A69934280F0E48126
:10319000AA463E6A7D627C6080255446FB681C1B03
:1031A000A04BB4F5807F28BF4FF480749B68A219B0
:1031B0009A4288BF9C1BF8F7A9F82246BC683046A3
:1031C0002146F8F723F9F969B86104EB000C0B7894
:1031D0007B6164452ED2DFF868920CF1FF3C04F16C
:1031E000FF3E1EF8013F09EB830219F82340568881
:1031F000ECB100234FF4004204F1FF3832424FEAB1
:10320000520202D00878284308706D0806D10AF1EE
:10321000010A4D701FFA8AFA01318025D34503D87F
:10322000E64533D3984531DC01339C42E6D1E6458F
:10323000D7D1F9617B6ABA6913449BB2DA457B62E4
:1032400006D27B6A3A6A1C46D6183B699E42A5D3D1
:103250007C68802D1CBF0AF101031FFA83FA0AF172
:10326000020189B22046F7F755FA2368796A0125E9
:103270005A19226020461D70F7F74CFA2368534410
:1032800023602B46D7F800D0FEF71FBCFB697C6893
:103290001A463B7D1370DCE7336872689A4240F04F
:1032A000E580614BFF221A704FF0000A5F4D0DF070
:1032B000C9FC514620225E4885F800A02EF001F896
:1032C00087F82CA097F82C30072B00F20181DFF84B
:1032D0007491574E524697F82C3003EB430309EB99
:1032E000C3035B7CE3B197F82C3003EB430309EB9A
:1032F000C30320215B699BB197F82C3003EB430398
:1033000009EBC303586946F82200F6F709FA2B784F
:1033100056F82300F6F752FB2A780132D2B22A700F
:1033200097F82C300133DBB287F82C3097F82C302B
:10333000072BD0D92368591C21601A70B8F1000FEF
:103340003EF4DCAB3B4BC8F8003001252B46FEF7C2
:10335000BCBB344B3A6A9B68D4F800905A44934201
:1033600074D23A6AA3EB0208F7F7D0FF4246494607
:10337000386AF8F74BF8236803442360002D3EF4C5
:10338000BDAB86427EF7BAAB002100E02368013076
:103390005A1CB04222601970F8D1FEF7AFBB002D65
:1033A000D7D159462046F7F7B5F923685A1C226051
:1033B0001D701C4B26689D683B6A0BEB030295420F
:1033C000C0F00A81F7F7A2FF5A463146386AF8F78B
:1033D0001DF823680125034423602B46FEF775BBC7
:1033E0003046F7F73DF9326871687B6A914283464F
:1033F00065D106461D469BE63046F7F731F9DFF802
:1034000048807BE69A1C32600B4A59781170D91CAF
:10341000316099785170191D3160DB789370FEF737
:103420006DBB00BFC0050020982200206FAC0020BB
:1034300070AB002079B40308D98A00204026002010
:10344000CC150408885F00209C890020F7F75EFFF8
:103450005A464946386AF7F7D9FF23680344236080
:103460008FE7644B93E84200FEF7F4BE5A1C1946FE
:103470003260614811F8022B027031605B78437052
:10348000042A03D9FF2A7EF4E5AA0DE75B490978EF
:10349000994205D8022A7EF4DDAAFF2B7EF4DAAA2F
:1034A000236801255A1922601D70B8F1000F3EF4FF
:1034B00025AB534BC8F800302B46FEF706BB511C1A
:1034C000316012781D46131C064618BF01232FE6F3
:1034D00052462FE7DA46C7F824B0C0E607F12C08B9
:1034E000404625F06BF8BB8DAB423FF40AAB454B31
:1034F0001B68002B3FF405AB1B689B69002B3FF456
:1035000000AB28469847FFF7FCBA00F07F0003287D
:1035100028BF0020012509F06DFC2B46FEF7D5BA27
:10352000344B1020C3F800905D6011F0A7FC364AC0
:10353000137843F001031370B8F1000F3EF4DEAAD4
:10354000324B0125C3F800802B46FEF7BEBA0A783D
:1035500002F0FD02FFF7E5B87D62AA467FE630463D
:10356000F7F77EF8A8843046F7F77AF83368726880
:10357000E884D11A03297FF78EAC1A46591C3160B2
:1035800012F8021BA97732605B7885F8203030464C
:10359000F7F766F83368726868847CE41C481D4954
:1035A0001D4A1E4B036001250B6013602B46FEF77E
:1035B0008CBA012528F01CFD2B46FEF786BA184A66
:1035C00099781288012512FB00F22B4692FBF1F24A
:1035D000A8F80020FEF779BA3B6AED1AF7F796FED5
:1035E0002A463146386AF7F711FF236803442360FF
:1035F000FEF784BAFC4600209822002011430020E8
:103600002DC60008C89F002050460020B02300208F
:1036100080AE0020D4AE0020D4B20020C1850008C6
:10362000068800202DE9F04F724B734A1C7893B046
:1036300000F59C412031814607911160002C00F07B
:1036400027856E4A1268904240F227826C4A6D4983
:103650001768DFF8E8B10492013C1C706A4C0391D2
:1036600007F48057002F40F02582039B5B7D002BE1
:1036700040F09B84049B1B681D0400F17787634B1B
:103680009945A37800F27383002B40F07383604B5D
:103690000693049B1F6817F4805940F0FA83039B3C
:1036A000BBF906605B8B9E42B4BF00260126594BD6
:1036B0001B6813F0805300F00782069A127812F00C
:1036C000010200F0088203985349408C91ED037A7F
:1036D00007EE900AF8EEE77AB4EEE77AF1EE10FA28
:1036E00081F20A80002E40F0FD814C4D95F8A0102B
:1036F000002940F0F7814A484A49056895F82D505D
:1037000000200860486088604749002D40F0EB8148
:103710000D70002A40F0EC81444B1A78002A50D1F9
:103720000399BBF900E04F8B898BBBF90200BE45C2
:10373000CCBF8025002545F040038E45A8BF2B4611
:103740009B0843F08005B842C8BF2B4643F04005B4
:103750008842A8BF1D46BBF904E0BBF90600AD08CE
:1037600045F08003BE45C8BF1D4645F040038E4569
:10377000A8BF2B469B0843F0800E284DB842C8BF17
:10378000734643F0400E95F8A2708842B8BF734666
:103790009F4201F04081A5F8A42085F8A620244985
:1037A00085F8A2300F78002F01F0B1805F2B01F077
:1037B00018816F2B00F0F887069B1B78D90740F122
:1037C000BA87049B1B4A1B68059203F00403002B75
:1037D00040F04A850DF14008174D0023C8F8043029
:1037E00005F15009109340F6330A192740F2833649
:1037F00029E000BFA886002028820020A48600209F
:103800009C63002014650020549B0020404B4C001A
:10381000C1860020F48700200C4400209C22002058
:10382000949F002058870020AC250020F19D0020A7
:10383000140300204C460020D8890020DC5E0020C4
:1038400004354D4520D0AA78EB789A4217FB0261E7
:10385000F6D26A78043217FB03633BF91220524513
:10386000A8BF5246B2F5617FB8BF4FF46172914272
:10387000E6DA9A42E4DC29782429E1D84046043586
:10388000F7F78EFA4D45DED1B04B98E803001F786C
:10389000AF4B83E80300002F00F03C840121AC48CB
:1038A000F7F78EFA002840F09A81E378002B40F079
:1038B0009681A84C23881DB225F00105AEB2B34213
:1038C000268000F0B286A44D02270E204FF0140986
:1038D0004FF0FF082F7085F8019085F8028011F0F5
:1038E0009DF939469A482688F7F76AFA002841F088
:1038F000458026F002039BB2B34223800AD0964B48
:103900001421FF2202250E201D7059709A7011F0AB
:1039100085F92688914BDFF884A21978DAF804003B
:103920000393B50708BF81F00201C1F34001F6F728
:103930004BF824218648F7F743FA30B9069A1378F2
:10394000590744BF23F004031370059B1B6813F051
:103950000A0F1DD005217E48F7F732FA002800F043
:10396000988625886F0740F1B58779480621F7F7D3
:1039700027FA002800F07A866E0640F18887072132
:103980007348F7F71DFA002840F03083059B1B6849
:103990009D0600F13B8327886D480C21F7F710FA4C
:1039A000002800F0388147F48073BB42238009D09F
:1039B000694B02251421FF220E201D7059709A7048
:1039C00011F02CF9664B1B78082B00F030810E2B80
:1039D00000F02D81049B1B685E0544D5614B1B796B
:1039E000002B00F0E18014215948F7F7E9F900288D
:1039F00040F0DF8021F08CFD012011F019F890B328
:103A0000DFF89C8100254FF0CC0902E0DDB2022DE9
:103A100029D809FB05F76B1C58F80760002EF5D173
:103A2000C378514A90F9020052F8233001960322DC
:103A30000092012132460FF061FF034605EB45007D
:103A400000EB0010049353B1314608EB8000CC2208
:103A50002DF037FC049B48F807300135EDB225F016
:103A6000E1FE0028D3D1069B1B78DD0740F1F280F0
:103A70003E493F4A01230B701370039BDAF80000A4
:103A8000197801F00101F5F79FFF059B1B685A07A4
:103A900000F1508113B0BDE8F08F364B364A1F68F5
:103AA000049307F480570392DFF8F8B0334C002FEB
:103AB0003FF4DBAD00212648F7F782F900287FF4B8
:103AC000D4AD0DF059FAD0E578023FF5F6AD069A7F
:103AD000127802F001022A4D002185F8A010002E74
:103AE0003FF409AE274901200870002A3FF414AEC4
:103AF000F9067FF511AE244A1278D2063FF50CAED6
:103B0000B9F1000F7FF408AE002B7FF405AE7B0205
:103B10003FF502AE1D4B1B78002B01F021841C4B9E
:103B20009B78002E41F059843BB11A4A1A4B126817
:103B30001B689B1A002BC1F28B841020104D11F0D2
:103B40006DF8012385F8A130E6E500BFC4490020E7
:103B5000F48700204A9B0020B43D0020ACBC00202C
:103B6000D4890020A8430020C8420408C28600204F
:103B7000C42300209C63002014650020549B002077
:103B80009C220020AC250020504600201403002079
:103B9000C88900208CB40020243B0020B0BC002049
:103BA000CC5A0020DC5E0020069B1B78D8077FF5EE
:103BB00021AF3C201AF0CAFC00283FF454AF09F0B2
:103BC000CDFB3C201AF05AFC00283FF44CAF09F022
:103BD000C5FB3C201AF052FC0028F0D143E7059BBE
:103BE0001B689A077FF565AEBF4C2688F3073FF543
:103BF00080AE46F001039E4223803FF47AAEBB4B79
:103C00001421FF2202250E201D7059709A7011F0A8
:103C100005F826886DE627F480739BB2BB422380AB
:103C20007FF4C6AEB24B1B78082B7FF4D0AE22884F
:103C300022F040039BB29A4223803FF4CBAEAB4BC1
:103C400002251421FF220E201D7059709A7010F069
:103C5000E5FFBFE6A74B93F80090B9F1000F5FD1E5
:103C6000DFF8E482A44F18F8030C3E784146A8F12F
:103C7000030515F097FB002800F0F083002E40F0BC
:103C8000428405F10801687915F08CFB002841F0A9
:103C9000E9819A49A87A15F085FB002800F0F183A4
:103CA000022E41F0E3819649E87B15F07BFB00286A
:103CB00041F0E0819349287D15F074FB002800F065
:103CC000F183042E41F0DA818F49687E15F06AFB9A
:103CD000002841F0D7818D49A87F15F063FB0028AB
:103CE00000F0F183062E41F0B981894995F823004F
:103CF00015F058FB002840F05887864995F82800B1
:103D000015F050FB002800F0F183082E40F03787B3
:103D1000814995F82D0015F045FB002840F0F1830E
:103D20007E4B01221A7015F0C0FD059B1B685A07D7
:103D30007FF5B0AE032015F05FFB002800F066862B
:103D4000238813F008047FF4A5AE082011F0AEF824
:103D50007348744D7449754A754BBBF8066000682A
:103D60002E80086014601C6013B0BDE8F08F0BB9A2
:103D70000123A3706F4B06931B201F7894F82160DA
:103D800015F03AFB012E07F00109824600F0258666
:103D900007F00203059394F82030DFF8B081664DF8
:103DA000052B69D8DFE813F05B004F000600DC004C
:103DB000FF008D00012E04BF052384F82030B9F1E7
:103DC000000F00F05281039B5C4FB3F91810B8F854
:103DD0000030002261F30F0263F31F42002361F3FE
:103DE0000F0361F31F43CBF8042039686269CBF8F5
:103DF00000308A42C0F06784012E41F0FE82032227
:103E000094F820300592CBE715F022FB012807D16A
:103E10004A4FB8F802303A68642101FB032323615A
:103E2000BAF1000F04D098F80630002B40F09080D3
:103E3000012E21D0414F22693B689A42C0F0318661
:103E4000012384F82030012E3BD098F80730012B55
:103E500000F014810FF0ACFB94F82030A0E7B9F12A
:103E6000000FD1D14FF48060BAF1000F00F0FB8356
:103E700011F01CF800232361059B002B3FF409ACD3
:103E8000059810F0CBFE049B1F6817F480593FF48F
:103E900006AC1D212A48F6F793FF00287FF4FFABFC
:103EA000284A039BD2881B8BBBF90660991A8E4265
:103EB00040F3018613449E42B4BF00260126FFF75B
:103EC000F6BB1E4F3A68B8F80230642101FB0323A9
:103ED0004FF480600022236184F82020E27010F00B
:103EE000CDFF94F820305BE74A9B0020B43D0020D2
:103EF000D4890020C28600209E000020AC3C002017
:103F0000B13C0020B63C0020BB3C0020C03C00205F
:103F1000C53C0020CA3C0020CF3C0020C423002028
:103F20002C460020A4230020B0230020A82300203A
:103F3000A0230020C1860020789B00208CB40020A4
:103F4000F4870020903D0020A23C0020AC3D0020E2
:103F50000FF02EFB03224FF47A7384F82020E361E4
:103F6000A74F2B8843F002032B800DF005F83A6829
:103F7000E36913440422A36184F82020012E40F059
:103F80009D853B68A2699A42BFF476AF9D4B187835
:103F900020B915F031FA00287FF46EAF2B8823F09A
:103FA00002032B808EE7964FE8E7039A013BD27D10
:103FB0003BF91330002A40F08183A3F57A73B3F5FF
:103FC0007A7FA8BF4FF47A7323EAE37307EE903A3F
:103FD0009FED8D7AF8EEE77A67EE877A8B4AFCEEF2
:103FE000E77A17EE903A1380FFF749BB884B894A6E
:103FF000B3F90430884982FB0302DB17C3EBA2024A
:10400000059B0A801B689D067FF5C5AC834B1B781A
:10401000980704D5824E337D042B00F255852788FE
:1040200017F0300F3FF4B8AC102010F027FF20201D
:1040300010F024FF7B4B278800221A707A4A7B48B5
:104040007B4E7C4D002111607B4A3160002329604A
:1040500041608161036083604361C36113605160AB
:10406000936053619161D36196E4654F3B6847F279
:1040700030520323E26184F8203072E70FF098FA9F
:10408000032240F6B83384F82020E3615C4F68E7F0
:104090006A4F3B78002B00F09887694BDFF8B481BA
:1040A000DFF8B4B1DFF8B4A1039345465E4604904F
:1040B00099460EE019F804109847032C28DC88B9BB
:1040C0003B782AF8020F01349C4205F1040580F286
:1040D000EF80072CE1B23046DBF80430EADD984788
:1040E00000B2EDE738F824206B88801A4FF47A711B
:1040F0009B1A01FB00F040F6CA0290FBF3F0084463
:10410000904240F2EE23A8BF10469842B8BF18462E
:1041100000B2D5E7DFF848A1DFF84881494D0AF140
:104120005A064FF0010951461AF8010C15F03AF9F8
:10413000F8B19AF804009AF802309AF803E000EB1C
:10414000400105EB8101013BD1F8B42003EB4303AF
:10415000434493420DD095F8E02081F8B0E009FA8D
:1041600000F022EA0000C1F8B430C1F8B87085F858
:10417000E0000AF1060A5645D5D13349204A334BAF
:10418000334D09681B78D2F8009008910793A5F188
:10419000B00A00266B685BB31F784FB3AA68A9EB1F
:1041A0000202002A0ADB9AF8E0200121B14022EA4B
:1041B000010209F5FA718AF8E020A960079ABAB1FC
:1041C0002A7859780432D2B2002940F09B820399B0
:1041D0003BF91220098B01F1C800824240F333847D
:1041E0009AF8E0109A7841FA06F3D80740F1C284B1
:1041F0000136042E05F10C05CCD1FFF74FBB00BFF3
:104200008CB4002014030020AAF1823F489B0020B8
:1042100030460020676666669823002050460020DE
:1042200054460020BA460020B047002060470020D6
:10423000802500202024002088470020F0AB0020AB
:10424000146500209C220020244A0020159B002099
:104250004C23002008AC0020BC9F00209A220020A4
:10426000B93B0020D0190408A84D95F8AA3053B1E5
:10427000069B1B78DE0706D5039BBBF906205B8BEC
:104280009A4200F34D841121A148F6F799FD0028C8
:1042900000F0208295F8AE302BB995F8A83013B90C
:1042A0003223A5F8AC30012385F8AE30FFF792BA7F
:1042B000DDF81090974A04921146974A0968A2FBCC
:1042C000092A42F201020A404FEA9A1A059200F0C6
:1042D000FD81924D9248934C934A95F800E0007806
:1042E00084F800E01070BEF1000F04D08E4A92F8FE
:1042F00000E08EF0010E854D0F2085F82400002B84
:1043000000F01283894B039E0C931B78B6F826C0ED
:104310000B931C463B78B78C039E854A368B0E96D2
:104320002646A2FB0442520802EB4202B21AD2B263
:10433000CDF824C001F48051089295F82580DFF86B
:1043400008B2DFF824C20A900AF5967276460F91F9
:1043500005F1280400200692CDF83490AE46002ED8
:1043600000F037823EF910201FFA82F9B9454FEA72
:10437000400103D3099DA94540F26F825CF82020DB
:10438000924580F02F823BF90120059D002D40F0E1
:104390004382013098422BF8012004F10604DEDB51
:1043A0000A98644ADDF834908EF825800F280CBFF7
:1043B000012100218EF82400117000F0BC825E4CB7
:1043C0005E4E5F4F35883868A1686268E06045F0EE
:1043D0000405401A9042524F3580534D4FF0010171
:1043E00088BF00223970297088BF84F82120002BF3
:1043F00000F0B382049A03991768524EB1F824C0B2
:10440000B1F818E0504817F48057354640F0C7829D
:1044100039460EE06A7802EB820202EB820202F277
:10442000EE2292B201318B4220F8022B05F10205F7
:104430000ED016F81120002A00F01382022AE9D0CB
:104440000131028820F8022B8B4205F10205F0D1E0
:104450000C9A137801331370FFF704B908F10501C2
:10446000687914F09FFF00283FF413AC012E40F050
:10447000F98505F10D01A87A14F094FF002840F0A9
:10448000F5853249E87B14F08DFF00283FF412AC2B
:10449000032E40F0EF852E49287D14F083FF00287D
:1044A00040F0EC852B49687E14F07CFF00283FF437
:1044B00012AC052E40F0E6852749A87F14F072FF64
:1044C000002840F0CB85254995F8230014F06AFFB9
:1044D00000283FF412AC072E40F06783204995F87E
:1044E000280014F05FFF002840F049831D4995F82B
:1044F0002D0014F057FF00283FF412AC092E3FF4B2
:104500000FAC4FF009094B463CE300BF9C22002052
:10451000F48700209C630020D34D621004820020A9
:1045200060030020159B0020610300209DAB00204C
:10453000ABAAAAAA0A4A0020549B0020789B00201C
:104540008CB400203CAC0020DC5E0020B13C00209C
:10455000B63C0020BB3C0020C03C0020C53C0020F5
:10456000CA3C0020CF3C0020A0AB0020CC4DD5F8A9
:104570008830A9EB0303002BFFF681A8C94A95F800
:104580008C30517C079AC5F888200133C64A039EB7
:1045900032F81120B17D03F00F0385F88C302B44E5
:1045A00092B292FBF1F283F8902095F8901095F872
:1045B000912095F8923095F89C000A4495F8931054
:1045C000134495F89420194495F895300A4495F8C9
:1045D0009610134495F89720194495F898300A449A
:1045E00095F89910134495F89A20194495F89B3042
:1045F0000A44134495F89D1095F89F20184495F8A7
:104600009E3001440B441A4442F30B12642AF17D9C
:10461000A8BF642213B209B1C2F1640307EE903A55
:104620009FEDA27AF8EEE77AD6E40221A048F6F7E9
:10463000C7FB00283FF45DA92580B7073FF56AA9AD
:1046400046F00203B34223803FF464A9994B022051
:104650001421FF2218700E2059709A7010F0DEFAA3
:104660002688FFF757B910F009FC03E425F0400352
:104670009BB2AB4223803FF482A98E4B02251421CA
:10468000FF220E201D7059709A7010F0C7FAFFF7C4
:1046900076B9238823F00405ADB2AB4225803FF400
:1046A00064A9844B02251421FF220E201D7059702D
:1046B0009A7010F0B3FA2588FFF757B9C3F53B633A
:1046C00008331BB279E403230593D0E47A4A92F8C5
:1046D00000E008E695F8A830002B3FF47BA8069B85
:1046E0001B7813F001037FF475A8012285F8A83028
:1046F00085F8A920FFF76EB8694D012185F8A01053
:10470000FFF7F0B9012900F002849AF8E0200123B4
:10471000B34001361343042E8AF8E03005F10C054E
:104720007FF438ADFFF7BAB8069B644A1B78106077
:10473000DF0700F1038295F8A61000297FF441A855
:10474000B5F9A430322B7FF73CA895F8A2200120C0
:10475000572A85F8A60000F09984049B1B6813F083
:10476000040302D05A2A00F0E8855D2A00F0E684AE
:104770005B2A00F026855E2A00F06C85562A00F040
:10478000CD85972A00F08785A72A40F09E844C4962
:10479000049B0A781B6842F004020A70494A059299
:1047A00003F00403FFF713B8B2F5FA7FFFF609A888
:1047B00095F8A620002A7FF404A8069B1B78012107
:1047C000D80785F8A61000F1C4840BF03BFDFEF776
:1047D000F8BF002F3FD05CF8202092454FEA4001FF
:1047E000FFF4D1AD384A384D525C05EB0109002A7F
:1047F00000F0B880022A47D199F8012002EB82022A
:1048000002EB820202F2EE2292B2032833DD059D12
:1048100012B2002D3FF4BDAD089D24F81520B8F16B
:10482000000F03D10B9D022D7FF6B3AD2288B4F8A3
:104830000290B4F804804A449044244A0FFA88F85D
:1048400082FB0852224DA2EBE87225F8018012B2D9
:104850004FF001089DE53A464100069D4CF8205076
:1048600093E5CAB2022A04D9032A7FF4E9AD62466D
:10487000D8E57246D6E5012505FA00F90A9D25EA34
:10488000090512B20A9580E53BF80120BDE745F025
:104890004003AB4223807FF4F0AEFFF770B800BF57
:1048A0009C22002058A0002074A0002014AE2341B8
:1048B000F4870020B43D0020159B0020283B0020F9
:1048C000504600204C4600203CAC00205655555523
:1048D0000C23002045F004039D4223800AD0B54BF1
:1048E00002251421FF220E201D7059709A7010F0BD
:1048F00095F92588B04BB14AB3F90430B04982FB31
:104900000302DB17C3EBA2030B80FFF72EB8394677
:10491000AC48F6F755FA00283FF406AF85F8A770C3
:104920000BF090FCFEF748BFA749A84A0C91DFF8AE
:10493000C0B2012111701B21A2480593F6F740FA7D
:10494000059B00287FF43BADA14CA24FE2683B6879
:10495000A3609B1AC82B00F25A83049B1F6807F4BC
:10496000805775E5C2B2022A40F2CF82032A8BD16A
:104970000E9A0F9D002D08BF3A4646E726F0010328
:104980009BB2B34223803FF458AE0E202F7085F8BF
:10499000019085F8028010F041F926884DE600214B
:1049A0000FE06A7802EB820202EB820202F2EE2250
:1049B00092B20131994220F8022B05F102053FF431
:1049C00047AD16F811201AB1022AEAD00288F0E7A2
:1049D000CAB2032AFAD87246EBE700230593FFF721
:1049E000DAB9B2F5FA7FFEF6ECAE95F8A630002BF8
:1049F0007EF4E7AE069B1B7801210B4085F8A610DC
:104A000000F0E7820CF0B8FAFEF7DBBE082010F0E9
:104A100035FAFFF73FB8704A70491068B5F9A4201D
:104A2000C76981FB07018911FF17781A00F5FF405C
:104A30007F3082423EF7B3AEC91B0A4412B2A5F8DA
:104A4000A420FEF7ACBEC8398A425CDA9AF8E010BE
:104A50009A7841FA06F3D9073FF5CAAB52420120D2
:104A6000099210F0F3F97B1E099A162B00F242818D
:104A7000DFE813F0E301F901CA0122020F02360256
:104A80009D01880171015A01430140012202300158
:104A900036029D0188011A010401EE00B201D60020
:104AA000C0000EF085FD032240F6B83384F82020C4
:104AB000E361FFF756BA0126FEF7F9BD3A68E369EC
:104AC0001344A361FFF7D8B90A2014F095FC278896
:104AD0008046002800F05882F90640F14483404D9A
:104AE00095F8F080B8F1000F7EF456AF0D2010F06D
:104AF00095F8012385F8F0302788B8F1000F7FF48E
:104B00009DAAFEF749BF9AF8E0300122B24023EA9D
:104B1000020309F5FA728AF8E030AA60FFF768BB71
:104B200000212848F6F74CF900287FF4ACAB32237B
:104B300085F8AA00A5F8AC30FFF7A5BB294B1B7878
:104B4000002B3EF43EAEE378002B7EF43AAE95F8AF
:104B5000A7300133DBB2032B85F8A7307EF631AEE8
:104B6000214B5B7813B9002E7EF42BAE0CF004FAC7
:104B7000FEF722BE002A0CBF0120022070E74FF092
:104B800008094B4603EB83031D4487F80090A9787E
:104B9000687823F043FD069B144A1B7801211170AD
:104BA000D9077FF5C0A8FEF768BF4FF007094B464D
:104BB000E8E700BFB43D0020304600206766666627
:104BC000D0470020F48700209DAB00200A4A002037
:104BD000549B00208CB40020D09D0020D34D621047
:104BE0009C220020159B0020C8890020C42300209F
:104BF000DC5E0020DAF8E400DFF81C8790F836105D
:104C000098F8023011446429A8BF642121EAE171B7
:104C100080F83610002B40F04B8427F07BFB74E5C6
:104C2000DAF8E400DFF8F08690F8371098F80230F0
:104C30001144FE29A8BFFE2121EAE17180F8371056
:104C4000002BEAD0162014F035FCDAF8E400E4E793
:104C5000DAF8E400DFF8C08681781144C829A8BFDB
:104C6000C82121EAE171817098F80230002BD4D07C
:104C7000142014F01FFCDAF8E400CEE7DAF8E400C0
:104C8000DFF8948641781144C829A8BFC82121EAD9
:104C9000E171417098F80230002BBED0132014F05F
:104CA00009FCDAF8E400B8E7DAF8E400DFF868862F
:104CB00001781144C829A8BFC82121EAE171017017
:104CC00098F80230002BA8D0122014F0F3FBDAF889
:104CD000E400A2E7DFF84086089898F802304179AE
:104CE00011446429A8BF642121EAE1714171002BBC
:104CF00040F09383DAF8E4008FE7DAF8E400DFF8B5
:104D00001886017A98F802301144C829A8BFC82132
:104D100021EAE1710172002B3FF47FAF0B2014F008
:104D2000C9FBDAF8E40078E7DAF8E400DFF8E885B0
:104D3000C17998F802301144C829A8BFC82121EAD6
:104D4000E171C171002B3FF468AF0A2014F0B2FB8F
:104D5000DAF8E40061E7DAF8E400DFF8BC8581798D
:104D600098F802301144C829A8BFC82121EAE1718E
:104D70008171002B3FF451AF092014F09BFBDAF84E
:104D8000E4004AE7DAF8E400DFF88C85417998F826
:104D900002301144C829A8BFC82121EAE17141713C
:104DA000002B40F04183112F7FF456AF35E7DAF83E
:104DB000E400DFF86485017998F802301144C829CD
:104DC000A8BFC82121EAE1710171002B40F0748372
:104DD000102F7FF457AF20E70898DFF83C85417823
:104DE0001144B1F5967FA8BF4FF4967121EAE171A5
:104DF000417098F80230002B3FF47CAF152014F07E
:104E000059FBDAF8E40008E70899DFF80C850F7918
:104E10001744642FA8BF642727EAE7770F7114F0BF
:104E200063FB98F80230002B3FF464AF032039464F
:104E300014F040FBDAF8E400EFE60898DFF8D884D5
:104E400001781144FA29A8BFFA2121EAE171017021
:104E500098F80230002B3FF44DAF012014F02AFBEC
:104E6000DAF8E400D9E60898DFF8AC8481781144D8
:104E70006429A8BF642121EAE171817098F80230A9
:104E8000002B3FF437AF022014F014FBDAF8E400F3
:104E9000C3E60898DFF88084C17998F8023011449D
:104EA00081F30801C171002B3FF424AF052014F0F9
:104EB00001FBDAF8E400B0E6089BDFF85C8499793E
:104EC00098F8020011446429A8BF642121EAE17125
:104ED0009971002840F0B0820D2F7FF4FDAE09E7F4
:104EE000DAF8E400DFF83084C17898F80230114431
:104EF000C829A8BFC82121EAE171C170002B40F088
:104F000084820F2F7FF4D4AE87E60E9A7DE43BF9BE
:104F100012209978B2F5617F4FF4966393FBF1F319
:104F20004ADB40F633019142A8BF11460C2FA1F590
:104F3000617191FBF3F100F08381182F7FF4E5ABF1
:104F4000C9B2C8290B46A8BFC823DAF8E400C27D5D
:104F5000DFB297423FF4D9AB9A1ADFF8BC83C7752A
:104F600048BF0732D71098F802300137FFB23BB97B
:104F7000002F3FF4CAAB38460FF068FFFFF7C5BB00
:104F8000182014F097FAF3E7FA0600F14F810B208E
:104F900014F032FA002840F01881BB0600F152816B
:104FA000C34D95F8F030002B3FF4A0ADB8F1000FE1
:104FB0007FF444A8FEF7F0BC0C2F00F0EA80182F15
:104FC0007FF4A3AB00210B46BFE7BA4A0392FFF779
:104FD00071B9B949096811F4003140F03F810B46BD
:104FE000B648C65C0F2E03F10C031ED00131152903
:104FF000F7D1049BB2491B680591FA3AA5F8A420A1
:10500000002203F0040385F8A620FEF7E0BBAD4ABA
:10501000049B1F68138823F004031380012307F403
:10502000805784F82130FFF713BAA74ED6F800E076
:105030004B00BEF1000F07D05F1800EB87079EF80A
:1050400001E07F787745D4D20B44A04FA04900EB14
:105050008300002330603B800B60CAE74FF00609F5
:105060004B468FE54FF001094B468BE54FF00209A7
:105070004B4687E54FF003094B4683E54FF00409A3
:105080004B467FE54FF005094B467BE5914B924936
:105090001A684FF47A73B3FBF2F3C3EB431203EBDA
:1050A0008203049A1268DB001206A1F8B43000F102
:1050B000E580834B05931B685F0700F1D680049B56
:1050C0001B6803F00403FEF782BB0021BB2A10918A
:1050D00000F08081B72A00F07981BE2A00F0748147
:1050E000BD2A00F04D81792A00F0DB817A2A00F098
:1050F000D1819E2A00F0C8819D2A00F0BE81AE2A8F
:1051000000F00182AD2A00F0F781EF2A00F0EE8175
:10511000FD2A00F0E581FB2A00F0DC81FE2A00F088
:10512000D381F72A00F08E817B2A7EF44AAB4FF4BC
:10513000FA61022007F084FDFEF743BB674B0022B3
:105140000120674D67492A700B600FF07FFEFEF764
:1051500038BB049B64491B680A60594A059203F0F6
:105160000403FEF734BB10200FF0A0FE20200FF048
:1051700085FE5E494E4D081F23F056F95C4B022216
:105180001A7095F8F030002B00F03B812788FEF76D
:1051900055BF00273946524B09915B78BB423FF41B
:1051A000B4AADFF87481384607F024FE98F802307C
:1051B00009991BB1C9B20C2014F07CF90137FFB278
:1051C000D6E64C4B01220220BBE74B4A4B4B52899F
:1051D00093ED007A07EE902AF8EEE77AB0EEC77A00
:1051E000B4EEE77AF1EE10FA7FF5D7AE93ED017ADF
:1051F000B0EEC77AF4EEC77AF1EE10FA7FF7CDAED3
:10520000BB063FF5CDAE2A4D20200FF04FFE2946BC
:105210007268336841F8EC2F05F1E800C5F8E83012
:1052200023F002F9324B01221A70AAE710200FF086
:1052300025FE2F4B278883F800804FF00108A6E653
:10524000CFB2A8E720200FF019FE294B184D0022FD
:105250001A7096E72A4B0222032072E7294909783F
:10526000032900F0C5801946BAE6049B264A1B684C
:105270000A21118003F00403FEF7A9BA234B1B781F
:105280009B077FF516AF224B1B7D042B7FF611AFDA
:1052900023F054F80DE7049B1E4A1B684FF4C871B5
:1052A0001180074A059203F00403FEF790BA00BF8D
:1052B0009C22002014650020AC3B00203C330408F5
:1052C0004C460020789B002058250020F625002021
:1052D000F82500208C630020C4B40020EE8A002052
:1052E000859F0020949F0020283B0020004700203D
:1052F000BA4600203C8B0020544700200C4400207C
:105300008A8B0020509B0020424A002050460020FB
:1053100054460020444A00200A8C00201BF04EF91D
:10532000F4F794FF1BF032F9F9F736F901200FF08A
:105330008DFD95F8A220FFF724BA95F8A820002A41
:1053400040F0938095F8AA3083F0010385F8AA30E5
:10535000002B40F085800C200FF060FCFEF731BA86
:10536000002E3EF4EAAB6B4D95F8A130002B3EF4D5
:10537000D3A90FF037FC002385F8A130FEF7CCB994
:105380004FF6FE73644A654896890590D089334488
:1053900001449381D1811BF011F9F4F757FF1BF001
:1053A000F5F8F9F7F9F801200FF050FD049BB5F876
:1053B000A4201B68FA3A0021A5F8A42003F00403F6
:1053C00085F8A610FEF703BA0223DBE70B464FF67B
:1053D000FE71D7E70B460221D4E7002BC3D050491A
:1053E000504A09684FF47A7000FB03131360BAE760
:1053F0000FF0F8FBB5F9A420FBE503230593FEF7B6
:105400003FBD4FF00108FFF771BB0F20099214F068
:1054100051F8DAF8E400099A73E50E2014F04AF81E
:10542000DAF8E400FFF7F9BB1120099214F042F812
:10543000DAF8E400099AB6E40D20099214F03AF87B
:10544000099A49E50021042007F0FAFBFEF7B9B9F3
:10545000304D0BF091FD002385F8A130FEF75CB9CB
:105460000B200FF0DBFBFEF7ACB92C4A85F8A81037
:1054700085F8A9000592FEF7AAB90021FF2029F0BE
:1054800057FC95F8A2203AE6012029F051FC95F846
:10549000A22031E6244A137A43F001031372FEF787
:1054A00090B9214A137A23F001031372FEF789B9E8
:1054B000172013F0FFFF1DE41020099213F0FAFFEC
:1054C000DAF8E400099A83E40021032007F0B8FB2E
:1054D000FEF777B90021022007F0B2FBFEF771B9A1
:1054E0000021012007F0ACFBFEF76BB90021084654
:1054F00007F0A6FBFEF765B9FF21002029F018FC94
:1055000095F8A22001E60121002029F011FC95F870
:10551000A220F7E59C220020AC8900204C46002008
:105520008CB40020243B0020F04900202DE9F047F6
:105530008C4B1B78DB07074644D58B4B8B4D1C7877
:105540008B4E012C59D01CD3022C07D189498A4A91
:1055500009881288914201D901241C70EB7AE3B1C9
:105560002B89D3B1854B1B78BBB107F057FC0028C2
:1055700000F09B802B7B83422CBF012100213170E6
:105580000CE07C497E4A098810886A7B801A884230
:10559000E2DAEB7A0024002BE2D131782A79632A0F
:1055A00006D8022C774E00F0BA803378002B5DD1FC
:1055B000754AAB7A8C4238BF0C461470002B4CD124
:1055C000BDE8F0876B4B694D19885B88E878CB1A8A
:1055D00083EAE3728142A2EBE3721DD32B788B4204
:1055E0001AD3614B1C78E01E012861D967490978FC
:1055F00002294FD0012C5E4EA5D15F4A5D49128829
:10560000687B0988121A914239DD5D4A12888A4204
:10561000A4D200241C70A1E7B1EB400FE1DC524B97
:105620001C78E11E012940F29480022ADEDC5749F1
:105630004F4E0878DFF84481DFF844C1DFF838E1E5
:1056400000210324022834701C7088F80010ACF884
:105650000010AEF8001081D11FE0012C71D0022C97
:105660000BD10720BDE8F0470FF0D8BA7068381AA0
:10567000474B984258DD72709AE7BDE8F0870224E4
:105680001C706BE7022AD2DD4049097802294FF0ED
:10569000040464D13949364E09783E48022ACCBF09
:1056A00000220122C28081804BE70221317075E720
:1056B000022A9BDC95F800C091FBFCFC0CF1010C6C
:1056C000BCF1080FDFF8B4A0304EA87895F801E0DF
:1056D00096F800802A4CDFF8A090254EA8BF4FF026
:1056E000080C8AF800C01FFA8CFA10FB0AF01EFBA7
:1056F0000AFE80B2DFF88CA02080A9F800E0002428
:105700004FF0640EB8F1020F34701C70CAF80440F8
:105710008AF801E07FF439AF0FFA8CF1BDE73078F9
:10572000A0B9012377603370C2F164021A4B00FB09
:1057300002F083FB0023C017A0EBA350643070700D
:1057400036E70820BDE8F0470FF068BA7368F81A2A
:105750008EE7032C96D10D49097802299AD0044E80
:10576000FCE600BFC1860020A826002038460020A5
:10577000AE260020D4430020AC2600200B4400209D
:10578000AA26002090230020509B002030430020B8
:105790007F969800344300206BCA5F6B2DE9F04F71
:1057A0002DED028BC54B1B7893B0072B0A9001F0AF
:1057B000218200230993C24B1B6807935E0500F109
:1057C000A987C04BD3F8008018F0080F40F040873D
:1057D000BD4B0893BD4C1B88DFF810B30593BC4B41
:1057E000BC491D68B1F906A06A89924580F2AC8176
:1057F000B94B4FF07E521A60B84FB1F900E03E8BC2
:105800009BF904209BF800009BF801C0AEEB060357
:1058100083EAE379002AA9EBE37914BF01224FF070
:10582000FF32B9F5FA7FA8BF4FF4FA79484580F204
:105830008881A9EB000307EE903AF8EEE77A764507
:10584000C4ED007A03DDF1EE677AC4ED007AB1F9B8
:1058500002E0AEEB060383EAE379A9EBE379B9F55D
:10586000FA7FA8BF4FF4FA79484580F28881A9EB06
:10587000000307EE903AF8EEE77A7645C4ED017A38
:1058800003DDF1EE677AC4ED017AB1F904108B1BE8
:1058900083EAE370A0EBE370B0F5FA7FA8BF4FF4A2
:1058A000FA706045CCBFA0EB0C0C4FF0000C02FB73
:1058B0000CFC07EE90CAF8EEE77AB142079BC4ED04
:1058C000027ABCBFF1EE677AC4ED027A13F480531A
:1058D000069300F01181BAF5FA6FDFF81492524680
:1058E000A8BF4FF4FA62B2F57A7F99F80030B8BFDA
:1058F0004FF47A72A2F57A72002B40F01781784942
:10590000DFF8F0E181FB0230D317C3EB6013581CC2
:105910006FF0630C3EF910003EF913E00CFB03231B
:10592000A0EB0E0003FB00F381FB0321DB17C3EBAD
:1059300061139E440FFA8EFE07EE90EA069BB8EEC6
:10594000E78A84ED038A002B40F01F86059B5906E9
:1059500000F1328518F0140F04D0059B13F4027F78
:1059600040F0E9865F4B1B781BB17B8B534580F27F
:10597000118599F82E601EB1059B9A0740F0DD87CE
:1059800099F83420002A40F0A785BE7F002E00F051
:105990000381022E00F0CA87032E40F0B18797F8EA
:1059A0002030C3EB431103EB8101C90089B2FB7FB7
:1059B0000233DBB2002A00F0AB87002900F0A88791
:1059C00049480668B1FBF6F10EB2A9F86460ABB3C2
:1059D00007EE906AF8EEE77AF7EE006A86EEA77AAD
:1059E000012BD4ED007AD9ED1E6A77EEE67A67EEE8
:1059F000877AC9ED1A7A21D0D4ED017AD9ED1F6AE0
:105A000077EEE67A022B67EE877AC9ED1B7A15D01E
:105A1000D4ED027AD9ED206A77EEE67A032B67EEB1
:105A2000877AC9ED1C7A09D0D4ED037AD9ED216AC1
:105A300077EEE67A67EE877AC9ED1D7A1F49097815
:105A4000092901F04985002E40F3AB8093B399ED0D
:105A50001E7AD9ED1A7A77EE877A012BC9ED1E7A74
:105A6000C4ED007A21D099ED1F7AD9ED1B7A77EE3B
:105A7000877A022BC9ED1F7AC4ED017A15D099ED12
:105A8000207AD9ED1C7A77EE877A032BC9ED207A3C
:105A9000C4ED027A09D0D9ED217A99ED1D7A77EE1D
:105AA000877AC9ED217AC4ED037A013B022BB8BF96
:105AB0000223DBB2002A18BF022373E03043002028
:105AC0009C6300204C4600204A9B00200C44002090
:105AD000244A0020DC5E00206025002014650020A0
:105AE0001F85EB5114030020D0890020A4890020D9
:105AF00090230020284A00207A8B9245C0F25984D6
:105B0000BAF5FA6FD4BFC2EB0A03C2F5FA634FF4D9
:105B10007A7101FB03F1DFF8789099F80000C2F583
:105B2000FA63B1FBF3F200283FF4E9AE99F80130D3
:105B3000144902FB03F281FB0213D217C2EB63127A
:105B4000DDE6DFED117A7AE6BAF5FA6F80F21D84B0
:105B5000287AAAEB020303FB00F3C2F5FA6293FB77
:105B6000F2F3C3F1640307EE903A9FED0A7A074B14
:105B7000F8EEE77A67EE877AC3ED007A3CE6DFED70
:105B8000027A7AE61F85EB510000000060250020B4
:105B9000902300200AD7233CA9F86460002A00F073
:105BA000728102232A785FED056AA97807EE902AB0
:105BB000F8EEE77AB0EE007A67EEA67ADB4AF4EE0A
:105BC000C77AF1EE10FA107840F38284DFEDD86ADC
:105BD00037EEC77AB0EE676AA7EE266AF0EE466A3D
:105BE00094ED007A9FEDD36ADFF870E3DFF870C3BD
:105BF00027EE066AF0EEC65ACEED005A8CED006A2A
:105C000099B107EE101AB8EEC75A9FEDCB7A66EE3F
:105C1000064A25EE075AB7EE007A37EE457A64EE6B
:105C2000A54AA4EE857A26EE076A9FEDC47A6A79C2
:105C300026EE877A27EE067AAAB1DFEDBF6A9FEDDE
:105C4000C06A65EEA65A06EE902AF8EEE66A66EE9F
:105C5000A56AF4EEC66AF1EE10FA40F324869FEDD1
:105C6000B96A27EE067A0C289FEDB78ADFEDB76A8E
:105C7000DFF8F08200F0EA85B4EEC87AF1EE10FAAF
:105C800098BFB0EE478AB4EEE68AF1EE10FAB8BFDC
:105C9000B0EE668A88ED008A002B00F0E680B0EE58
:105CA000007AF4EEC77AF1EE10FA05DD37EEC77A26
:105CB000DFED9F6AE7EE267A94ED017ADFED9D6ACB
:105CC00027EE267AF0EEC75A8CED017ACEED015A16
:105CD00099B106EE901A9FED986AF8EEE66A27EE03
:105CE000075A66EE866AB7EE006A36EE666A25EEF9
:105CF000255AA6EE856A27EE067ADFED906AAA7924
:105D000067EEA67A67EE877AFAB107EE102AB8EE48
:105D1000C77A9FED896ADFED8A6A27EE257A27EE3A
:105D2000067AB4EEE67AF1EE10FA00F3B885B5EE35
:105D3000C07AF1EE10FA01F11780B7EE006A36EE84
:105D4000477AC6EE076A67EEA67A0C2800F05F85F0
:105D5000DFED7D6A9FED7D7AF4EEE67AF1EE10FAE2
:105D600088BFF0EE667AF4EEC77AF1EE10FAB8BFAB
:105D7000F0EE477A012BC8ED017A76DD6B78DFED26
:105D80006E6A07EE903AF8EEE77AB0EE007A67EEC8
:105D9000A67A6B7AF4EEC77AF1EE10FA05DD37EEEB
:105DA000C77ADFED636AE7EE267A94ED027ADFEDDB
:105DB000616A27EE267AF0EEC75A8CED027ACEEDB4
:105DC000025A9BB106EE903A9FED5B6AF8EEE66AE6
:105DD00027EE075A66EE866AB7EE006A36EE666A06
:105DE00025EE255AA6EE856A27EE067ADFED536A80
:105DF000EB7967EEA67A67EE877AFBB107EE103A89
:105E0000B8EEC77A9FED4C6ADFED4D6A27EE257A32
:105E100027EE067AB4EEE67AF1EE10FA00F33B854F
:105E2000B5EEC07AF1EE10FA00F19A87B7EE006A8B
:105E300036EE477AC6EE076A67EEA67A0C2800F0BF
:105E40002285DFED416A9FED417AF4EEE67AF1EECC
:105E500010FA88BFF0EE667AF4EEC77AF1EE10FA27
:105E6000B8BFF0EE477AC8ED027A092800F0C68480
:105E700097F82140002C40F07B84354BD3F800800C
:105E8000002389F8343018F0200F06D0089B1B88B7
:105E900003F03003002B40F009822E4C2E4E94F874
:105EA0002420DFF8C480DFF8C4A0531E082B00F2C2
:105EB0000981DFE813F022018101AA0007015D00DA
:105EC000090096010701830198F80030002B40F08B
:105ED000F2842368207A4FF4807203EB00200021C3
:105EE00026F03AFC237A0133DBB2022B237240F016
:105EF0005281002026F06CFC002026F069FCFF2077
:105F000026F066FC00F01F00052801F0998321F0BF
:105F1000BFF8E568002D00F00A840022236961685B
:105F20000120A84794F82420BFE700BF3043002099
:105F3000D7A368416F12033B0AD7233C00004843B4
:105F4000A4707D3F0000C84200C0F94400C0F9C4FD
:105F50004C460020305D00208CB4002090250020AD
:105F60008425002068250020845F0020886002408E
:105F70004FF40071206821F03DF8012800F04485BD
:105F8000C0F00F86022840F0068121F0ABF821F026
:105F90007FF8E568002D00F0CA83002210462369CF
:105FA0006168A84794F824207FE71021B64821F0C3
:105FB00021F88346002840F0EC8001217F2014F076
:105FC0006BF90128074640F0E4805846022114F09E
:105FD00063F9002801F0DB81012840F0DA80162106
:105FE0003A2014F059F9431C9B02A36221F07AF87D
:105FF0002868F3F7DDFC00210A2021F019F80028B9
:1060000040F04386032384F8243010210EA820F0AA
:10601000F1FF002840F0BF809DF842209DF841002C
:106020009DF844109DF845309DF84350120442EA13
:1060300000620A431B019DF846109DF83900DBB24F
:1060400043EA111342EA052203F5FA6362636387A8
:106050009DF83A209DF8403042EA002201F00F01FD
:10606000180903F00F0384F83C10A2859DF838103E
:106070009DF83B2084F839309DF83C3084F82E1090
:1060800084F82F209DF83D109DF83E2084F8303094
:106090009DF83F3084F8333084F8380084F83110AC
:1060A00084F8322021F01EF8A37E002B00F0DB8064
:1060B00004217648F3F722FE00230422236284F8A9
:1060C00024200323DBB2022B6BD9042A00F0A58025
:1060D000082A00F0A2806E4B1B7823B96D4DAB7877
:1060E000002B40F072856C4B1B78072B00F0E88486
:1060F00013B0BDEC028BBDE8F08F684D2868F3F754
:1061000057FC0021084620F093FF074620F0EAFFE5
:10611000012F40D128684FF0000B84F819B0F3F735
:1061200047FC40F2AB11082020F082FF052800F068
:106130007884012800F08C8520F0D4FF637E002B4A
:1061400001F09282022384F824302868F3F730FCAF
:10615000637E022B14BF00274FF0804700213720B9
:1061600020F066FF3946292020F062FF074620F024
:10617000B9FF87B9637E022B00F07785A776286880
:10618000F3F716FC0021092020F052FF00283FF40D
:106190000CAF20F0A7FF94F82420531EDBB2022B93
:1061A00093D83F4B61691B685B1AC82B90D920F0CC
:1061B0006FFF94F8242088E7384DC6E70825FF20B4
:1061C00026F006FBFF2800F08684013DF7D16369C5
:1061D0003268FA339342DED220F05AFF94F824203A
:1061E00063E6FF2026F0F4FAFF284FF0080506D0FA
:1061F000013DECD0FF2026F0EBFAFF28F8D1236A0E
:106200000022012B227641F27984E269013B0132BE
:1062100023620823E26184F82430224C16F046F908
:106220006378022B00F06384032B7FF454AF41F2B8
:10623000B813E35C002B41F0CB8041F2A403E35C94
:10624000002B41F0C08041F2E803E35C002B41F0F9
:10625000C48041F22C13E35C002B3FF43CAF1248A6
:1062600016F018F837E70D4D2868F3F7A1FB4FF447
:106270000071102020F0DCFE054620F033FF002DD9
:106280003FF416AFA8E700BF705D0020003C00405F
:10629000C44900200A8C002030430020805F002089
:1062A0008CB40020B86D0020E47E0020CD4B1B781C
:1062B000D8077FF5F2ADCC4BCC4AB3F90430DFED13
:1062C000CC7A82FB0312DB17C3EBA2031BB208EEEE
:1062D000103AB8EEC88A28EE278AB0EE480AF4F7DA
:1062E00099FCF0EE408AB0EE480AF4F719FCC14B75
:1062F000D878002800F08A85BF49B9F99220B1F911
:10630000023044F250649B1AA34241F38D80A3F5FE
:106310000C43A03B44429C4201F383808342A8BFCC
:106320000346B1F90010B9F9905013444A1B44F2E6
:1063300050611BB28A42A9F8923041F36A80A2F5FB
:106340000C42A03A944203DC9042A8BF1046044697
:106350002A1912B207EE902A07EE103AF8EEE77A01
:10636000F8EEC76A27EEE87A60EE277AA0EE267A82
:10637000A249A9F89020E8EEA67ADFEDA16A27EEFF
:10638000267A67EEA67A00F05DBD2B7AC3F164032E
:10639000FFF7E9BB9B4B1B78012B00F08683192B81
:1063A00000F083830E2B3FF4E4AA082B3FF4E1AA0C
:1063B00080E31946FFF7AFBB8B4B8C49B3F9043030
:1063C000B9F80820DFED8A6A9FED8F7A81FB03011F
:1063D000DB17C3EBA1039B1A1BB207EE903AF8EE52
:1063E000E77A67EEA67A77EE876ABDEEE66A16EE82
:1063F000103A2033402B40F28D83DFED846ABDEEEE
:10640000E77A17EE103A2033402B00F280839FED9D
:10641000807AF4EEC77AF1EE10FA40F3F687DFEDFA
:106420007D5A9FED7D6A01E0F0EE477AF4EEC67A80
:10643000F1EE10FA37EEE57AF6DCDFED787AB4EEBD
:10644000E77AF1EE10FA40F1DC87DFED725A9FED4A
:10645000746A01E0B0EE677AB4EEC67AF1EE10FA33
:1064600077EE257AF6D49FED687AF4EEC77AF1EEEE
:1064700010FA00F3D1829FED6B7AF4EEC77AF1EE59
:1064800010FA44BF9FED657A77EE677A67EEA75AF8
:106490009FED655A9FED656A9FED657AA5EE856A69
:1064A00027EEA55AA5EE867AE5EE077A94ED016A05
:1064B000D4ED005A27EEC67A65EEA77AA5EEA67A45
:1064C000E6EE267A84ED007AC4ED017AFFF742BA4F
:1064D000F0EE676AFFF784BB5649574BD1F8EC10D2
:1064E0001B6844F620608142A8BF0146B1F57A7F5F
:1064F000B8BF4FF47A7189B2DB06A9F8361040F1C3
:106500009382069B002B40F033844C4BD3F800E081
:10651000BEF932604A48D9F83830D4ED037AA0FB8E
:1065200001018809642191FBF0F11429BDEEE77A9D
:1065300009EB430CA8BF142101338B42C9F8383052
:1065400017EE10AAA4BF0023C9F8383009EB4303A3
:10655000ACF83CA0B3F93C3007EE103AB8EEC77A7D
:1065600077EEC77AFDEEE77ACDED057ABDF9141026
:1065700081EAE173A3EBE173B34200F33387314B5C
:106580004FF07E511960FFF700BA1D212A48F4F739
:1065900017FC00283FF4DAA92B4BDB78002B7FF4A3
:1065A000D5A9DFED2A7A264938EE678AC6F5FA6260
:1065B000FDEEC87A12B2CDED0B7ABDF92C301B037B
:1065C00081FB0301DB17C3EBA11302FB03F343F3CE
:1065D0000F33334407EE903AB8EEE78A84ED038A2E
:1065E000FFF7B4B950460020304600206766666663
:1065F00035FA8E3C54470020B0470020802500200B
:10660000CDCCCC3DD4890020DB0FC93F0000000079
:10661000DB0F4940DB0FC940E4CB1641DB0F49C01B
:10662000E4CB16C1DB0FC9BF92E741B99730083CF4
:1066300015A82ABE300A0020F4870020949F00206D
:10664000D34D6210A4000020549B002000007A4427
:10665000D44CD54BD4ED027A0893B2EE0E7AF0EE1C
:10666000E76AF4EEC76A1B880593F1EE10FA42D58B
:106670005D0740D5CD4BCE4AB3F90430CD49DFF8A4
:1066800080B3098882FB0302DB17C3EBA2035B1A0A
:106690009BB21AB212F1B30FBCBF03F5B4731AB2B6
:1066A000B32AC8BFA2F5B473C349C8BF1AB29BF8D6
:1066B00004300978002B4FF6FF7318BF0123080739
:1066C0007FF58DA8BD49096812FB03F3097EBC4A1A
:1066D0009BB211FB03F382FB03121A44DB17C3EBDB
:1066E000221307EE103AB8EEC77A77EEC77AC4EDF8
:1066F000027AFFF774B8AD4BAD49B3F90430AD4A37
:10670000DFF8FCB281FB0301DB17C3EBA1031380AD
:10671000FFF765B8AB488368002B3FF452A800F13F
:1067200050019847A84B1B680793FFF74AB894F8A5
:106730002420FFF7BABBA04B1B7813F0100300F026
:10674000838199F80C20D9F8103094ED017A002A51
:106750000CBF01224FF0FF3203FB02F307EE903A29
:10676000F8EEE77A77EE877AC4ED017AFFF7FAB8A8
:106770001E219648F4F724FB00283FF47EAB089BCB
:106780001B885D063FF579AB99F88830A34240F04D
:10679000C5868F4BD9ED237AD3ED006A98ED025A66
:1067A000DFED8C5A9FED8C6A27EEC57A68EE277A6A
:1067B000A8EE267AE5EE267AB4EEE57AF1EE10FA46
:1067C00088BFB0EE657AB4EEC67AF1EE10FAF4EE58
:1067D000E57AB8BFB0EE467AF1EE10FA88BFF0EE77
:1067E000657AF4EEC67AF1EE10FAB8BFF0EE467AAA
:1067F00088ED007AC8ED027AFFF73FBBFDEEC87A5C
:10680000764A17EE903A9680D380FFF731BB9FED22
:10681000717ADFED716A7149F4EEC77AF1EE10FA20
:1068200098BFB0EE677AFDEEE77AB4EEE67AF1EE65
:1068300010FA17EE902AB8BFB0EE667A012B88EDF9
:10684000017A4A803FF79AAAFFF712BBB4EEC87AE2
:10685000F1EE10FA98BFB0EE478ABDEEC77AB4EEFB
:10686000E68ADFF878A1F1EE10FA17EE102AB8BF29
:10687000B0EE668A88ED008AAAF80020002B7FF42B
:106880000EAAFFF7F5BABDEEE77A544B17EE102AC1
:106890009A80FFF7D6BADFED526AFFF7CDBADFED87
:1068A000506AFFF750BAF7EE005A75EEE66A85EEC9
:1068B000A66AFFF7D6B94B4B596809057FF508ACB6
:1068C0004FF40062DA60DAF80020474B22F0010250
:1068D000CAF800201A89D20700F1AC8022F096FF96
:1068E0000028FBD1404A938823F002031B041B0CB1
:1068F000938098F80030002B7FF4FBAAFFF7E9BAE9
:106900003A4B5988FB7F0233DBB2002A7FF455A84B
:10691000B9F86460013E36B2002EA9F864603FF712
:1069200095A8002A7FF43DA9FFF7ADBAB9F8361053
:1069300001F57A7189B2FFF73AB82D4BDFED2D7A68
:1069400093ED080AB4EEE70AF1EE10FA40F2FE8188
:1069500028F042FCD9ED0C7A20EE270A28F0A6FB9D
:10696000B0F5617F00F30C8207EE900AF8EEE76A5B
:10697000DFED217A66EEA76A07EE906AB8EEE77A55
:10698000FDEEE67A17EE903A2033402B40F2728605
:106990009FED1A0A28F08AFB00B207EE900AB8EEC3
:1069A000E77AD5E10C4400204A9B002030460020C5
:1069B00067666666D047002050460020949F0020FE
:1069C00089888888C4B400209C630020F487002054
:1069D000A000002000C0F94400C0F9C434430020E6
:1069E0000000C84200600240003C0040BC9F002004
:1069F000383B00208FC2753CD06D393A0000000052
:106A0000A4890020DB0F49406369326864339342F4
:106A1000FFF4BBAAFFF7BFBB1FED067A77EE677ADC
:106A200034E56776FFF788BB079BDE003FF569AD6D
:106A3000FEF7ABBF9A891A89D207FBD422F0E6FE93
:106A400000287FF44BAF4DE79BF80320002A40F06D
:106A50000582B9F914609BF80210AAEB060383EAD9
:106A6000E370A0EBE370884240F3048503EBD3733B
:106A700001225B10C9F8243089F8282089F81C20ED
:106A8000D9F810301E44B6F5FA6FA8BF4FF4FA6675
:106A9000B6F57A7FB8BF4FF47A7607EE906AF8EED3
:106AA000E77AC4ED037AFEF75DBFC24B9B7B002BF8
:106AB0007EF45FAFC04A0023A3609360FEF759BF26
:106AC000F8F766F8099ABD4B801A988013B0BDECB0
:106AD000028BBDE8F08F20F005FB042384F82430FE
:106AE000B74C15F0E3FC6378022B7FF49DABA378E1
:106AF0004FF0010A072B3FF6EEAADFE813F09E03E2
:106B0000240492031904B703780382038E03DFED94
:106B1000AD7ACBE4F4EEC77AF1EE10FA40F3888553
:106B2000DFEDA95A9FEDA96A01E0F0EE476AF4EEA5
:106B3000C66AF1EE10FA36EEE57AF6DCDFEDA46A0D
:106B4000B4EEE67AF1EE10FA40F17685DFED9E5A6A
:106B50009FEDA06A01E0B0EE667AB4EEC67AF1EE7F
:106B600010FA77EE256AF6D49FED9B7AF4EEC76AA9
:106B7000F1EE10FA40F39A809FED987A77EE666A0C
:106B800066EEA65A9FED965A9FED966A9FED967A0D
:106B9000A5EE856A26EEA55AA5EE867AE5EE076A89
:106BA0002DE420F09FFAE5680423002084F82430C7
:106BB0002076002D3FF431AB236922686168A84735
:106BC00094F82420531EFFF7E9BA884E3278013A30
:106BD0000D2A28D8DFE812F07600D0019F017E014F
:106BE000610185027002CA024C021300FA01F00131
:106BF000E701DE01F7F7CCFF0990FEF7DCBD7C4B27
:106C00001B78002B00F0BF851A2012F0F5FB00283E
:106C100040F0B98599F89430002B40F0B4850923F1
:106C200033701BF0CFFB1FF0FDFD00285BD03378E5
:106C30000C3B022B7FF657AA99F894300122327050
:106C4000002B3FF450AA002389F89430FFF74BBA89
:106C5000584604220EA925F07FFD9DF83B30AB2B52
:106C600004BF02236376FFF767BA2868F2F7A0FE35
:106C700039463A2020F0DCF9042283460EA9384632
:106C800025F06AFDBBF1000F07D020F02BFA20F0B1
:106C9000FFF994F82420FFF708B920F023FA0E9B9F
:106CA0001BBAC3F38073A376FFF769BA9FED517ADD
:106CB000F4EEC76AF1EE10FA44BF9FED457A77EE25
:106CC000666A5DE74C4B1B78DF0700F12A871F20BF
:106CD00012F092FB0028A6D00C2333701FF0A2FD07
:106CE00000287FF400AAEB78002B3FF4FCA9424B6C
:106CF0001B78D90704D40CF0D3FB002840F07D8426
:106D00003E4CD9F8982023689A4200F27D8433786B
:106D1000012B3FF4E8A999F89420002A3FF4E3A955
:106D20000B2B0DD801229A4040F6030112EA01050F
:106D300089D112F4C06F03D0093B012B40F2D187F7
:106D40002F4B22685A600B2333707CE79FED1D7A2E
:106D5000D4ED037A77EE877AC4ED037AFEF710BE9E
:106D6000F7EE006AFFF768B8F7EE006AFEF7EBBFD0
:106D7000244BD3F800E0BEF832607608FFF7CABBB8
:106D800007EE906ADFED206AB8EEE77A66EEA65A63
:106D90009FED135A9FED136ADFED137AA5EE856A16
:106DA00026EEA55AE5EE867AE5EE276A26EE870AF4
:106DB000F0E500BFA0A70020682500203443002094
:106DC000B86D002000000000DB0FC940E4CB164185
:106DD000DB0F49C0E4CB16C1DB0FC93FDB0F4940D5
:106DE00092E741B99730083C15A82ABE078C0020CD
:106DF000288A0020DB0FC9BFC18600208CB4002088
:106E000080890020949F002084F9223FC24B9FED8F
:106E1000C36AB3F90020B3F90230C14907EE902AE2
:106E200006EE903AF8EEE77AF8EEE66A27EEE87AB0
:106E300060EE277AA0EE267AE8EEA67A27EE067AAA
:106E400067EE867ABDEEC77AFDEEE77A17EE102A76
:106E500017EE903A0A804B80FFF71FB8B9F914205B
:106E60009BF80210AAEB020686EAE670A0EBE67039
:106E7000884240F3E1829245C8BF494207EE901A2A
:106E8000F8EEE77A012037EE888AC9F8183089F8D9
:106E90001C0084ED038AFEF765BD1FF07FFCA14B4B
:106EA000002102208DE80300A3F10802029148208E
:106EB0001BF0B4FF00287FF4B6AE9B4B4FF0FF31C0
:106EC00006221860596032701FF0ACFC00287FF475
:106ED000B3AE08E71FF062FC944A0292A2F10C03E1
:106EE000292101930091A2F10A035021163A492069
:106EF0001BF094FF00287FF496AE8D4B1B6813F0B7
:106F0000800300F02786884B4FF0FF310522186080
:106F100059603270D8E7844C1FF040FC854A6368A2
:106F2000126864339342BFF47EAE40201FF008FC29
:106F300000287FF478AE2368DFF828A2DFF8F88114
:106F400040270CE01FF04EFDD8F800202368013ADE
:106F50000133013FC8F80020236000F0A8861AF82A
:106F600003301846002BEDD100234FF0FF32236091
:106F7000042362603370A7E7022B00F089846D4B15
:106F8000694A1B6853606C490023136003220B603D
:106F9000327099E71F2012F02FFA00287FF49EAE7E
:106FA0000123337090E7012B00F048840E23132057
:106FB00033700DF033FE36E6012B01D1F4F708FAF9
:106FC0000D23132033700DF029FE2CE6022B33D154
:106FD0005A4BDFF894811B78002B40F04086D8F89C
:106FE00000401CB323780BB394F82820002A7FF4C8
:106FF0006BAF237EA26384F83C20042284F828200F
:1070000013F00803626AE262226303D04C4A41F241
:107010009413D358636300276762A760E760204634
:1070200013F0F6F80523276484F82830002204239F
:10703000C8F8002088F814303B4B3E4A5B68126861
:10704000C833934204D31FF00DFC00283FF4EBAD8E
:10705000AB78032BA4D13B4C20680CF01DFC3A4BC1
:107060001B780022022B22609AD106F08FF997E755
:107070001A2012F0C1F900283FF4D3AD334B1B881E
:10708000002B7FF4CEAD324B45201C681FF0AAFCCC
:107090000E201FF0A7FC20461AF026FD0A9C204671
:1070A0001AF022FD2B4A2C4B12681A6020460A2344
:1070B00033701AF029FEB4E51FF070FB274B002156
:1070C00005208DE80300A3F10802029153201BF074
:1070D000A5FE00287FF4A7AD134A08231060337083
:1070E000F2E61FF05BFB1E4A0292A2F10C0307249A
:1070F00001930094A2F108030021143A47201BF0E9
:107100008DFE00287FF48FAD074B34704FF0FF32B7
:1071100083E80500D8E600BFB0470020CDCCCC3DC9
:10712000802500205C1C0408808900207E1A040849
:107130009C6300208CB40020709E00206C8900208D
:10714000B86D0020749E0020CC89002000880020AB
:10715000FC870020E8870020E4870020C01C04088A
:10716000781C0408181A0408D49D00201FF016FB90
:107170001BF05EF900283FF456AD1FF073FB0028AA
:107180003FF451ADC34AC44B12681A600A233370EE
:107190009AE623690622652BA27032D92278032A47
:1071A00014BF6FF0FF026FF07F02A3F1650303EAE3
:1071B000020303F1010314BF4FF4807280229A424C
:1071C00023611ED23268E66802329F19974280F02E
:1071D000B284B24A6660D16FA760490203FB01F333
:1071E0000521166042F81C3C42F8183CA170A268C8
:1071F000AB49012014F0B6FA012840F0A18406231F
:10720000A3700021A74814F0EBF9012840F09884FE
:10721000A3780133DBB2A3706CE403236370FEF741
:107220005ABFA14B00930320A070302305229F4931
:107230009C4815F0A9F8FEF74EBF0EAB1946059312
:1072400000231846092214F01FF801287EF443AFEA
:107250000E9B93F8FE21552A00F0528241F2B4129F
:1072600002210123A1546370FEF735BF2278237DEC
:107270008F4EDFF82C82032A14BF4FF480778027CB
:10728000002B41D0012BFBD18A4B62681968306812
:1072900000234FEA412E4FF0FF31B1FBFEF112EB1C
:1072A000010B43F1000C0021614500F1020008BF11
:1072B000584538BF83465A467F49022014F084FB64
:1072C000032800F2D58101A353F820F0D76001080C
:1072D000DD720108D7600108DD7201086268A368E9
:1072E0002569991AA94284BFE260216103283FF40D
:1072F00050AF0133B3FBF7F207FB12320AB13B4444
:107300009B1A0022636022753268414602320020D7
:1073100014F05AFB032800F2AB8101A353F820F0CC
:10732000D760010883730108D760010893710108D1
:1073300041F27013E35C002B3EF4CDAE594814F0DB
:10734000A9FFFEF7C8BE0EAB0593194641F2FC1526
:1073500000236059092213F097FF01287EF4BBAE89
:1073600000230E9A2370B2F80B30B3F5007F00F0C3
:10737000178441F2B41203210123A1546370FEF774
:10738000AABE636884F814A00133A3607CE70421DB
:107390002C2012F081FF032183464E2012F07CFF47
:1073A0000C210590362012F077FF059B421C02331A
:1073B0009A4007FA0BF7A2FB0701420A42EAC152C0
:1073C000A262FEF713BE3D4814F064FFFEF73BBF18
:1073D0003B4814F05FFFFEF730BF3A4814F05AFF05
:1073E000FEF737BFBEF834309FED377A07EE903A9C
:1073F000F8EEE77A354B67EE877AC3ED007AFEF751
:10740000C4BAF0EE477AFFF72EB8B0EE677AFFF70E
:1074100014B82F498A42BCBF02F50C42A032FEF7D5
:1074200091BF2346FEF77DBF294CA342BCBF03F5A5
:107430000C43A033FEF76EBF99F81C1029B1254903
:1074400089F81C300B68C9F82030D9F81030134483
:10745000B3F5FA6FA8BF4FF4FA63B3F57A7FB8BFFC
:107460004FF47A7307EE903AF8EEE77AC4ED037AB8
:10747000FEF778BA99F81C30002B3FF401AB154B9E
:1074800089F828201B6889F81C20C9F82030FFF7EC
:10749000F7BA00BFE8870020E48700204C7F002077
:1074A000BC6D0020287F0020FDAE02086C49040856
:1074B000C07F0020C87F0020C06D00205C7E0020BF
:1074C000707F0020A07E00206F12833AA40000206D
:1074D000B0B9FFFF2C46002094ED000A06930592F8
:1074E00027F0E4FDD949DFF8A0E3D1F8EC10DFF88C
:1074F0009CC3059AACF800008EFB013EC917C1EB96
:10750000AE1107EE901AF8EEE77A069BFDEEE77AE9
:1075100017EE901AACF80210FEF795BA07EE904AF3
:10752000DFEDCB6A9FEDCB7A89F88840F8EEE77AF9
